:1000000000400020A9740000E9740000EB740000B7
:1000100000000000000000000000000000000000E0
:10002000000000000000000000000000ED7400006F
:100030000000000000000000EF740000F1740000F8
:10004000F37400009155000055780000F37400002F
:10005000F374000000000000F3740000F37400006B
:10006000F3740000297C00004D340000F37400009C
:10007000F3740000F3740000F3740000F3740000E4
:10008000F3740000D9780000F3740000F3740000EA
:10009000F3740000F3740000F3740000F3740000C4
:1000A000F3740000F3740000000000000000000082
:1000B0000000000000000000000000000000000040
:1000C00010B5064C2378002B07D1054B002B02D02E
:1000D000044800E000BF0123237010BD640200202B
:1000E0000000000024E80000044B10B5002B03D0F2
:1000F0000349044800E000BF10BDC04600000000F6
:100100006802002024E80000164B002B00D1144B9D
:100110009D46402292029A1A924600218B460F4633
:100120001348144A121A0BF0B3FB0F4B002B00D0EC
:1001300098470E4B002B00D0984700200021040068
:100140000D000D48002802D00C4800E000BF0BF065
:100150005FFB2000290007F0CFFB0BF033FBC0460C
:100160000000080000400020000000000000000027
:1001700064020020C42F00200000000000000000E6
:1001800002000120104011D1042A0ED91368180969
:1001900080B2002809D001388000031D11180979A8
:1001A000002902D001309842F8D170470020FCE7C6
:1001B0000378002B03D05AB2002A01DB01307047CC
:1001C0003F229343C03B59424B41C01803789343AD
:1001D000802BF4D10130F9E710B500240378002B0F
:1001E00001D1200010BDFFF7E3FF0134F6E770B541
:1001F000002204000D00411C092003F051FC0028DE
:1002000006D001236200134343600023A34200DBB6
:1002100070BD9A00A958821891600133F6E770B555
:10022000012803DC1C2001F0CFF870BD01230D680C
:1002300011201D42F7D04868184206D1042804D97D
:100240000F2302681340042B01D00E20EBE703F0CC
:1002500085FA6D100400002D03DDFFF7BDFFA842F5
:1002600006DA1220DFE72000FFF7A2FF0400013DBD
:10027000012DF8D120787F2809DDDF280BDCF82359
:100280003F22DB00800118406378134018430123AC
:1002900040001843C9E7EF280BDCFC226378120109
:1002A0009B0113403F220007000C0343A07810403D
:1002B000ECE7F72812DCFC22637892021B03134060
:1002C000E0228004520310403F221843E378134099
:1002D000FC220343A07812018001E8E7012040429C
:1002E000D5E7F8B54D680F00EB0706D4042D04D907
:1002F0000F232E683340092B03D00B2001F064F844
:10030000F8BD6B683609B6B25C10731EA3420FD8F5
:100310000321200009F078F96421642803DC01003E
:10032000032800DA03212800891903F0EBFB0500FC
:100330002B6800201B099BB2013B9C42E0D23A682B
:10034000A31C9B005A510123013464001C436C60C0
:10035000D6E7F0B585B0012803DC1C2001F034F8A5
:1003600012E001274B683A000093022806D08B6800
:100370003B4203D05F10002F00DC17000125009BDB
:100380002B4203D00120404205B0F0BD009B042B5E
:10039000F8D91B680C680F261900314004292AD1AE
:1003A0002C4205D1042C03D923681E40042E01D011
:1003B0000E20D3E70098FFF7E3FEB842E2DB009897
:1003C00003F0CCF90600200003F0C8F90100781E04
:1003D00030180BF013FE041ED4D03378002B01D05C
:1003E000A64202D36800012521E03000FFF7E0FEBD
:1003F00001350600F1E709293ED1009B5B685B10DF
:1004000001939F42BEDC2C422ED1042C2CD92368B0
:100410003340042B28D1200003F0A0F9039602906A
:100420007E1C009AB300D058844202D17800284341
:10043000AAE728420ED104280CD90368039A134076
:10044000042B07D103F08AF9010002980BF0A0FDFC
:100450000028EBD0019B37009E42E1DD92E71F00B0
:10046000019B9F4200DD8DE77B1C00999A008A5812
:10047000A242F4D17800B6E7032900D082E71A0936
:1004800092B25B0F92000B40D31A01939F4200DDA2
:1004900078E72C4229D1042C27D922681640032E54
:1004A00019D1100980B2520F80003240251D801AE8
:1004B000019B2E181B1A0193009B781E0433019A8E
:1004C000904200DD5EE72A001918B2420FD316D120
:1004D0000130400087E7042E07D1200003F03EF9E9
:1004E00005002000FFF74CFEE2E70F2036E70C780E
:1004F000A4461478A44502D101310132E5E7013068
:10050000DDE710B503F00EF943000120184310BDDC
:10051000C30711D404280FD90F2302681340032BFB
:100520000AD119400133591AC0234907DB05194084
:10053000024B1A40114301607047C046FFFFFF9F06
:10054000F7B507000E001C20012F06DD4C680123C3
:1005500022001A40009203D10D2000F035FF53E035
:10056000022F02D08A681A42F6D0012335681D4254
:1005700000D0A9E0042D00D8A6E01C41002C00DC2E
:100580001C000F2029680840092828D16B685B10DF
:100590000093022F05D0B368009A5B109A4200DDE9
:1005A0000093009B01221D1B0135EB43DB171D400F
:1005B000691C092003F074FA071E09D001236D009D
:1005C0001D4303003268083345600099A14201DAF7
:1005D0003800FEBD0134A100515802C3F5E70428DC
:1005E00045D1280003F0BAF8FFF7F6FD0190022F7D
:1005F00004D0B3685B10984200DD0193019BA342D5
:1006000004DA002003F0BEFA0700E1E7280003F057
:10061000A5F80700009BA34221DB2800009703F008
:100620009DF805003800FFF7C3FD019B013407006A
:10063000A342F7DA009BC41A200003F0A3FA071EB6
:10064000C6D003F08BF80190306803F087F82200E1
:10065000009B591B411801980BF0FEF8B8E73800D1
:10066000FFF7A6FD009B070001330093D2E70328A4
:100670002AD10B099BB2490F9B000140591A022F46
:1006800004D0B2685210914200DD1100A14205DA97
:1006900000220320110003F003FAB5E703200E1B2C
:1006A000331DD9170140C9188910002203F0F8F949
:1006B000071E00D18CE7013631000334FFF728FF15
:1006C000381D29193200C7E7212046E7F8B5002870
:1006D00005DC1C2000F078FE05002800F8BD01268E
:1006E0000C6826400FD06410E343DB171C40E11C6C
:1006F00089100022032003F0D3F9051EEDD021005C
:10070000FFF706FFE9E7042C01D80025E5E70F23F2
:1007100022681340042B1BD12000FFF731FDC31CBE
:1007200007000320D9170140C9188910320003F0CF
:10073000B7F9051ED1D03900FFF7EAFE200003F01B
:100740000DF82B1D01003A0018000BF085F8C4E7E6
:10075000092BDAD10320636832005F10FB1CD91724
:100760000140C918891003F09BF9051ECDD039004E
:10077000FFF7CEFEFF20BE42AFDA0122B300E3183E
:100780009B68134208D01341FF2B00DD0300D943BF
:10079000C917AA190B4013710136ECE710B57F2970
:1007A00002DC0170013010BD1A4B99420CDC402371
:1007B0008A115B42134303703F230B40802149425F
:1007C000194341700230EEE7134B994210DC2023AD
:1007D0000A135B4213433F24802203708B11524261
:1007E0002340214013430A43437082700330DAE709
:1007F0000A4B9942D7DCF0230370603B4370113BF6
:100800008A11FF3B1A4382703F2211401943C17085
:100810000430C8E7FF070000FFFF0000FF0F0100E2
:10082000F0B50D0085B0002803DC1C2000F0CCFDE5
:100830000DE009680122080010400AD002AC114105
:100840002000FFF7ABFF011B200003F0A7F9040015
:100850001AE004293FD90F230C682340092B3AD111
:100860004B685B10019303239C46019B9A420EDD6B
:1008700003F088F9041E07D02E68012502F06EFFF0
:100880002F00019B9D421DDD200005B0F0BD01320F
:100890009300CC580123234001D10D20C6E76410FA
:1008A0007F2C0DDD0D4E0223B44209DD0C4E634654
:1008B000B44205DD00270B4EE30FA6427B419B00AF
:1008C000C018D2E70135AB00F1583942E5D04910E4
:1008D000FFF764FFD5E72120A8E7C046FF07000027
:1008E000FFFF0000FF0F010010B5040001200840C9
:1008F00010D104290DD90F230A681340042B08D105
:10090000080002F02BFF010020000BF041FB4342E6
:10091000584110BD0020FCE7F7B50F00012803DCAB
:100920001C2000F051FDFEBD01264D682E4006D171
:10093000042D04D90F222B681A40092A01D00B205C
:10094000EFE76A681B099BB25410A34200D85C1EF3
:1009500039681E48FFF7C8FF01230190002813D112
:1009600039681B48FFF7C0FF002811D0002C0DD0BC
:100970000123621C013C9C409200535123436B6055
:1009800004E00136B200AB50B442FADA0020CAE704
:100990003B680D20DA07C4D55B10002B11DD9C42AB
:1009A0000FDB9B00A200291DEB1889180433994224
:1009B00009D10123013C9C40AA181C4353606C6080
:1009C000E4E71220ADE758681860EFE723CF000096
:1009D00027CF0000002310B50C000B70C30705D50E
:1009E0000D49421020000BF097FA08E00B4900284F
:1009F00002D0042804D10A4920000BF0ADFA10BD42
:100A00000428FCD90F2302681340042BF7D102F00D
:100A1000A5FE04490200E5E7ACD900002CCF000098
:100A200032CF000037CF0000F0B593B0060002913E
:100A30001C20012E1DDD029B01251B681C002C4083
:100A400000D0ADE0042B00D8E6E01A680F231A406E
:100A5000092A4AD10394039A029992008A581700EE
:100A60002F4005D1042A03D910681840092806D060
:100A7000222000F0A9FC0190019813B0F0BD52684B
:100A80005210A418039A013203929642E3D1611CDA
:100A9000012203F005F80190002802D10023019300
:100AA000EAE7019B6400190025435D600831029A62
:100AB000BB00D05802684368120992B25B109A4298
:100AC00000D8531E0022934209DCDA43D2171340A8
:100AD0009B00C918039B01379F42E8DBCCE79400D9
:100AE0000519AD6801320D51EDE72700032A59D1F0
:100AF0000193029ABB00D3582B42B9D1042BB7D92A
:100B0000186801990140032939D1020992B2430FB3
:100B100092000B40D31A1C190137BE42E9D10320C1
:100B2000E31CD9170140C9188910002202F0B8FF50
:100B300001900028B2D000252100FFF7E9FC019BBD
:100B40001E1D029AAB00D45801231C421FD1042C55
:100B50001DD90F2123681940032918D1180980B223
:100B60005B0F80000B40C01A0023834213DBC3439A
:100B7000DB17184001353618BD42E2DB7CE704295B
:100B800000D075E71800FFF7FBFA2418C4E720002F
:100B9000FFF7F6FAE8E7E2181279F2540133E4E7D6
:100BA00000273C000F25029ABB00D35801221342B4
:100BB00034D1042B32D9186801002940042935D1D9
:100BC0001800FFF7DDFA24180137BE42EBD12000F0
:100BD00002F0D8FF0190002800D15FE7029FB60025
:100BE000BB19041D029301233D681D4229D1042D28
:100BF00027D90F262B681E40042E37D12800FFF777
:100C0000BFFA0600280002F0A9FD01002000320012
:100C10000AF022FEA41922E02700C3E7180005A964
:100C2000FFF7D8FE05A80BF0BDF9CCE7032900D0EB
:100C30001EE7020992B2430F92000B40D31A1C190F
:100C4000C2E705A92800FFF7C5FE05A80BF0AAF921
:100C500005A90500020020000AF0FEFD6419029BB0
:100C60000437BB42BFD10023237005E7032EF6D122
:100C70001A0992B25B0F92001E40961B291DC5E710
:100C8000F0B50D0097B0002806DC1C2000F09CFB9E
:100C90000700380017B0F0BD0C68012123000B409D
:100CA000009306D1042C04D922680F331A40092A74
:100CB00001D00B20EAE7626852100392002A03DC9D
:100CC000009802F05FFFE3E7504A019201280BD041
:100CD0006868084208D1042806D902681340042B2A
:100CE00002D102F03BFD019001980BF05BF9060088
:100CF0000F27039B0834013B05935E43039B02903F
:100D00009B00E318049301232068184273D1042840
:100D100071D901680B003B409C46042B03D1FFF7BF
:100D20002FFA861909E0032B6CD162460B099BB29E
:100D3000490F9B0011405A1A9619049B0434A34290
:100D4000E1D1300002F01EFF071EA2D02B680793EE
:100D5000029B002B03D0686802F000FD0190380070
:100D600002F0FCFC0400009B079A9B00D3189E68CD
:100D7000300002F0F3FC0123334005000693002B02
:100D800001D1042E04D809A93000FFF723FE09ADD4
:100D900028000BF007F9069B0490002B0ED1042EBF
:100DA0000CD90F2133681940032907D11A0992B2CF
:100DB0005B0F92000B40D31A351D04932000049A58
:100DC00029000AF049FD049BE418029B002B0AD07D
:100DD000059B009A934206DD2000029A01990AF0D1
:100DE0003BFD029BE418009B01330093009A039B98
:100DF0009342B8D14DE709A9FFF7ECFD09A80BF024
:100E0000D1F88EE702F0AAFCF9E7C046CBD3000088
:100E100010B50024A04207DD0B6801341C4003D04C
:100E20005C10E343DB171C40611C0122092002F027
:100E300037FE002803D0012364001C43446010BD2A
:100E40000A6870B510000125284034D1042A32D92F
:100E50000F24136849681C40092C17D154681B09DA
:100E60009BB22C41A34200D85C1E844205DC0220C8
:100E70000133984206DB00200FE085005519A96078
:100E80000130F2E7840011510130F2E7032C12D156
:100E9000294203D1132000F097FA70BD4910FF29B1
:100EA000F8D81B099BB204329B00D3189342E2D9B5
:100EB00011700132FAE70B2000F086FADBE7000040
:100EC000F8B5012700254E680C003740AF420ED11F
:100ED0003D00042E0BD90F2233681A40092A10D185
:100EE00072681B099BB25510AB4200D85D1E216889
:100EF000CB0716D54C10002C01DDA5421CDA1220C0
:100F000030E0042A04D13000FFF73AF90500EEE79B
:100F1000032AECD11D09ADB25B0FAD001340ED1AF1
:100F2000E5E72748FFF7E0FC002813D00AF090FF20
:100F3000290008F04FFC4C1C002F3ED1042E3CD958
:100F40000F2332681340092B10D10134A400A45997
:100F50002000F8BD21681B48FFF7C6FC2C000028C4
:100F6000EAD1113000F030FA0400F1E7042B1CD173
:100F7000300002F0F3FB0500012C0EDCFFF718F93E
:100F8000461B300002F0FEFD041EE1D002F0E6FB3D
:100F9000320029000AF060FCDAE72B78013C002BD4
:100FA000ADD02800FFF704F9E5E7032B05D134198C
:100FB000E37801245B001C43CAE70B20D2E7C0465C
:100FC0001CCF000027CF0000F7B54D680F002A00A6
:100FD00001210A402FD1042D2DD90F242B68BE6882
:100FE0001C40092C14D169681B099BB24C1001925A
:100FF000A34200D85C1E39682A48FFF775FC002818
:101000002DD00F232A681340092B1DD1012317E08F
:10101000032C10D10E4203D1132000F0D5F9FEBDF0
:1010200072100192FF2AF7D81A0992B25B0F920050
:101030001C40141BDFE70B20EFE701339A00AE5092
:101040009C42FADA0020EAE7032BFBD12B000133A4
:101050005A1BA242F6DC6A461279DA70F7E7396861
:10106000CB0706D54910002901DD8C4209DA122090
:10107000D3E70D48FFF738FC2100002801D11130DB
:10108000CBE70F232A681340092B03D101318900D4
:101090004E51D7E7032BD5D16B461B796D18EB70FA
:1010A000D0E7C04623CF000027CF000070B5012451
:1010B0000868204207D1042805D90F2501680D4092
:1010C000092D02D14468200070BD032D08D10A0902
:1010D00092B24B0F92002B40D31A5B001C43F2E7F5
:1010E000042DF0D102F03AFBFFF776F840000443FC
:1010F000E9E7000010B5034A0B21034804F01CFB8C
:1011000010BDC046C4CE0000BCCE00000020704719
:10111000042070470120704710B5002002F032FD16
:1011200010BD00207047002070470020704700204D
:101130007047002070470020704700207047002053
:101140007047000010B5034A0C21034804F0F4FA7C
:1011500010BDC046ACCF00000CD000007047037833
:10116000002B03D05AB2002A01DB013070473F2226
:101170009343C03B59424B41C01803789343802BA3
:10118000F4D10130F9E70000F8B50127060014009A
:101190000800394227D104293FD90F230A681A4091
:1011A000042A3AD13C4213D1042C11D922681340AD
:1011B000042B0DD102F0D2FA0500200002F0CEFA85
:1011C000010028000AF0E4FE00282EDB1FD127E0F2
:1011D000E30722D502F0C2FA0A2200210AF0AAFF90
:1011E0000500601010E0174015D1042A15D90F230F
:1011F00012681340042B10D120004D1002F0AEFAFB
:101200000A2239000AF096FF85420EDB08DD002E27
:1012100009DC00200CE04D10E3E70F22054B1A70AB
:101220000136022EF5D8042002E004207617304063
:10123000F8BDC046A402002010B50124044002D02D
:101240004410200010BD042810D90F230268134059
:10125000042B07D102F082FA21000A220AF06AFF69
:101260000400EEE7032B01D10430F5E70D22014B1A
:101270001A70E6E7A4020020012210B5024018D13E
:10128000042802D903681A0992B201230B4012D133
:10129000042902D90B681B099BB20024934206D192
:1012A00004309B000431C318984206D30124200067
:1012B00010BD0022E9E70023EFE704780A78002C4C
:1012C00001D1002AF2D0013001319442ECD0002447
:1012D000EDE70000F7B50700009101933049314B6D
:1012E000002A02D002220A70013A00261A601B6806
:1012F000CE54BE4200DBF7BD009AB300D058294B54
:10130000274D1C68C8239B0065191C1B012318422C
:1013100006D0254A4310210028000AF0CBFD09E041
:10132000224A002802D004281BD1214A210028008B
:101330000AF0C0FD1A4C20000AF034FE194A019B45
:101340001060002B0BD07B1EB34208DD194B984276
:1013500005D8431C1360202222540022E254013697
:10136000C7E7042819D90F2301680B40042B04D1C7
:1013700002F0F4F9104A0300CDE7092B03D14368CA
:101380000E4A5B10C7E7032B08D10A0992B2490F36
:1013900092000B40D31A0A4ABDE70123094ABAE773
:1013A000A5020020C8050020ACD900002CCF000009
:1013B00032CF00001F030000D7DF00007CD2000006
:1013C0008BD2000096D20000014B187000207047AD
:1013D000A402002070B501F01DFF094C0100251D7D
:1013E0001F2228000AF0F6FD28000AF0DBFD042386
:1013F00004308008000118432060200070BDC04602
:1014000080020020C368F0B59D00836889B05D1933
:101410000300183306930369069A9F00069B039006
:10142000DF19436901939B00D3180293CD4B1B78BE
:10143000002B26D17F222B68CB491C1213409B0026
:101440005B58043501929F46039B587804F0AEFD2B
:101450000023039A137027E0C24B1B78002B10D196
:101460002B68019A1C121340BF4A9B009B580435FD
:10147000E9E7069B3A1DD11ABA4BD82928DD1A2272
:101480001A70039BB74C9B6821780193EA1A039B5F
:1014900092109B7812021A43039B587804F08EFD39
:1014A0000023039A23701370039B069A9B68019391
:1014B000ED1A039BAD10DD60069BFE1A039BB61070
:1014C0001E61029B9B1A039A9B10536109B0F0BDE9
:1014D0001B783C60002B01D01700D2E72B680199E4
:1014E0001C120B40A0499B005B5817000435AAE76B
:1014F000069B3A1DD11A9B4BD82902DD1A221A707D
:10150000BFE728681B78291D3860002B02D0170020
:101510000D00B6E76B6801991C120B4092499B00C5
:101520005B58170008358EE7069B3A1DD11A8D4B84
:10153000D82902DD1A221A70A3E7A4001B782C19FF
:101540003C60002B01D017009BE72B6801991C120F
:101550000B4085499B005B581700043573E7069BD9
:101560003A1DD11A7F4BD82902DD1A221A7088E75A
:101570007E48A40021581B783960002B01D0170049
:101580007FE72B6801991C120B4077499B005B5841
:101590001700043557E7043F744B3A68A400E25043
:1015A000704B1B78002B00D06BE72B68019A1C1244
:1015B00013406D4A9B009B58043544E76B4BA400D5
:1015C000E058FFF739FE043F06003868FFF734FEA5
:1015D00036180120654B76000643E650614B1B78B8
:1015E000002B00D04DE72B68019A1C1213405E4A75
:1015F0009B009B58043526E7069B3A1DD11A594B90
:10160000D82902DD1A221A703BE70698029C0121B4
:10161000A04202D221000C3909681B783960002BE6
:1016200001D017002DE72B6801991C120B404E4981
:101630009B005B581700043505E7069B3A1DD11A3D
:10164000484BD82902DD1A221A701AE70699029827
:1016500081420FD203000C3B1968454B4910E41836
:10166000641AA40023583B603E4B1B78002B05D026
:10167000170006E7182119700023F4E72B68019979
:101680001C120B4038499B005B5817000435DAE602
:10169000069B029A934219D213000C3B1968344BF3
:1016A000043FE41813004910611A3A688900CA50CF
:1016B0002C4B1B78002B00D0E3E62B68019A1C1200
:1016C0001340294A9B009B580435BCE61822254B41
:1016D0001A70EDE7069B029A93422DD2244B3E1FCF
:1016E000E31814000C3C04932368049A5B10D31A8B
:1016F000029A9B009858FFF79FFD07903068FFF70C
:101700009BFD2468049B64101C1B079BA4001F18EE
:1017100001207F00029B0743E7503700114B1B78E5
:10172000002B00D0ADE62B68019A1C1213400E4A24
:101730009B009B58043586E618220A4B1A70EDE789
:10174000069B3A1DD11A074BD82902DD1A221A70BE
:1017500097E60299A40061581B783960002B09D0E4
:1017600017008EE6A40200207CD00000902D0020FF
:10177000FDFFFF3F2B6801991C120B40CF499B00D6
:101780005B58170004355EE6043F029B3A68A400EC
:10179000E250CB4B1B78002B00D072E62B68019AED
:1017A0001C121340C54A9B009B5804354BE6029B14
:1017B000A4001C192368043F38685E10FFF73CFD45
:1017C00036180120BE4B76001B7806432660002B9E
:1017D00000D056E62B68019A1C121340B74A9B00B2
:1017E0009B5804352FE6069BA4003F1BB44CBB421C
:1017F0000CD82378002B00D043E62B68019A1C12EA
:101800001340AE4A9B009B5804351CE6AD4801F0DE
:1018100095FF2378002B00D033E62B68019A1C1229
:101820001340A64A9B009B5804350CE6A300ED1814
:10183000002C00DA38E6A24B1B78002B00D020E603
:101840002B68019A1C1213409C4A9B009B5804353C
:10185000F9E5043F3B68042B04D1A300ED18002CEC
:1018600000DA21E6964B1B78002B00D009E62B68A6
:10187000019A1C121340914A9B009B580435E2E5E3
:10188000043F3B68042B04D0A300ED18002C00DAC1
:101890000AE68B4B1B78002B00D0F2E52B68019AEF
:1018A0001C121340854A9B009B580435CBE53E1F14
:1018B0003068C3070AD540100138002809DB01232E
:1018C0004000A40018432D193060EDE5FFF7B4FC8B
:1018D000F2E77B4B37001B78002B00D0D1E52B685B
:1018E000019A1C121340754A9B009B580435AAE5C7
:1018F0003A00069B0C32D31AD82B03DD1A22704B08
:101900001A70BEE5FF2361005B001940FE3BFF3B00
:1019100019433960039906988968241204916D1A55
:101920000399AD1089782D020D4302999D40091A43
:10193000891099401D430B43BB60039B7D609C70E5
:10194000E4B2614BE4000292E358039A93605C4A6C
:101950001278002A03D008331D00029F91E51D0074
:10196000019A9B680C351C121340544A9B009B58EB
:10197000029F68E53B1F1C68029A069B934232D186
:101980000A20E30711D4042C18D90F23226813402E
:10199000042B16D1200001F0E1FE0AF003FBC8235E
:1019A0009B00984200D918000630643003F0FEFE18
:1019B00000280FD1043D069B029375E50720042CF7
:1019C000F3D02000431E9841FA234042FF331840D1
:1019D0000730EAE7039B2100587804F001FB00235D
:1019E000039A1370E7E7029B029A0C3B1B6803996A
:1019F0005B109B00D31A0C3B1C601F1D1300083B9F
:101A00001B685A108A70D2B22F49D2005B00555819
:101A10009B0A039A9B009560ED18029B069A043B73
:101A20001B685B109B00D3180293254B1B78002B7F
:101A300000D026E52B68019A1C1213401F4A9B0018
:101A40009B580435FFE43B1F1868FFF7F5FBA40023
:101A500006003F1B1E2827DC00280DDC184B1B78D6
:101A6000002B00D00DE52B68019A1C121340134A7D
:101A70009B009B580435E6E401F0B8FB033E3618A2
:101A800001F0B4FB114B801B9842F9D80C4B1B782A
:101A9000002B00D0F5E42B68019A1C121340074A72
:101AA0009B009B580435CEE40123039A137001F088
:101AB0009DFB039B0A3886195E60F5E47CD000002C
:101AC000A4020020A8D20000982500203F420F0069
:101AD0003B1F1868FFF7B0FBA40006003F1B00285F
:101AE0000DDCD14B1B78002B00D0CAE42B68019A87
:101AF0001C121340CD4A9B009B580435A3E4CC4BE9
:101B0000984203DD1D22C84B1A70BAE40123039AE0
:101B1000137001F06BFBFA239B005E430A3E301802
:101B2000039B5860C0E4A300FF1A002320001A00A2
:101B30003900FFF7CFFBBF4EBF4C3168200002F0E9
:101B40002DF8BE4B31681860200004F0EBF83168C6
:101B5000200004F04CFAB44B1B78002B00D090E42A
:101B60002B68019A1C121340B04A9B009B58043505
:101B700069E4AD4BA4001B783F1B002B00D080E430
:101B80002B68019A1C121340A84A9B009B580435ED
:101B900059E4039803F06EFEA34B1B78002B00D092
:101BA0006FE42B68019A1C121340A04A9B009B58BB
:101BB000043548E43B1F1B68002B49D13B000C3B1C
:101BC0001868012303401E1E1FD046103A0001234F
:101BD0007100083A0B431360002E00DC94E00123EF
:101BE00072001A43391F0A603A00083A12681A4113
:101BF000921B04923A000C3A106818422BD0049AB7
:101C0000A400D2189A40134331E004281BD90F23B3
:101C100002681340092B02D143685E10D6E7042BFB
:101C200008D101F09BFD0378002BCFD0FFF797FA86
:101C30000136F8E7032B06D11609B6B2520FB600EB
:101C40001340F61AC2E71922774B1A70FFF719FCF6
:101C50005B105E1EC0E7042851D90F2102680A40BC
:101C6000092A16D1049BA40002339B001B58029A38
:101C7000A3506D4B1B78002B01D0FFF702FC2B68A3
:101C8000019A1C121340694A9B009B580435FFF7C8
:101C9000DAFB042A2BD1029BA4001B19079301F045
:101CA0005DFD0600049C0134012C10DC3000FFF7C0
:101CB00056FA831B1800049301F064FF041E0ED033
:101CC00001F04CFD049A310009F0C6FD07E03178BF
:101CD000013C002906D112220C00534B1A70079BBD
:101CE0001C60C6E73000FFF73AFA0600DCE7032A7B
:101CF00005D1049AA40082181279520083E71922B0
:101D0000494B1A70FFF7BDFB0435B2E7A300069AF2
:101D1000FB189B1AD82B12DC0123002C14DC424B3D
:101D20001B78002B01D0FFF7ACFB2B68019A1C122B
:101D300013403E4A9B009B580435FFF784FB1A2250
:101D4000394B1A70FFF79DFB3B60013C0437E4E719
:101D5000069A3B1D9B1A344ED82B03DD1A23337091
:101D6000FFF78FFB069B029AA40093422AD23B1FE7
:101D70001868FFF761FA011E21DD029B0C3B1A680F
:101D8000521082421BDB9007801A2D4B4018C0185E
:101D9000029B8000C2583B1B1A60234B3F1B1B78E1
:101DA0000437002B01D0FFF76CFB2B68019A1C1243
:101DB00013401E4A9B009B580435FFF744FB202329
:101DC0003370EAE71823FBE71C4BA4001A683B1B9F
:101DD0001F001A60144B04371B78002B01D0FFF74B
:101DE00050FB2B68019A1C121340104A9B009B5811
:101DF0000435FFF728FB3B1F1A68042A11D1A40001
:101E00002D19094B1B78002B01D0FFF73AFB2B68EB
:101E1000019A1C121340054A9B009B580435FFF79A
:101E200012FB1F00EDE7C046A40200207CD000009A
:101E300080EE3600C8050020A50200200800002022
:101E4000FCFFFF3F3A1F1368042B04D000231360EC
:101E50003A00A4002D19D54B1B78002B02D0170097
:101E6000FFF70FFB2B6801991C120B40D0499B0018
:101E70005B5817000435FFF7E6FAA3009C46F81AF2
:101E8000002C17DC1C22C94B1A7000230360634628
:101E9000FF1AC64B04371B78002B01D0FFF7F1FA6D
:101EA0002B68019A1C121340C14A9B009B580435B1
:101EB000FFF7C9FA036804005A1063461E1801238D
:101EC00021680B4003D10D21B84A1170DEE749109B
:101ED0008A4200DD0A000434B442F0D101235200EA
:101EE0001343D3E7A3009C46F81A002C17DC1C22EE
:101EF000AE4B1A70002303606346FF1AAB4B0437E6
:101F00001B78002B01D0FFF7BCFA2B68019A1C123A
:101F10001340A74A9B009B580435FFF794FA0368C7
:101F200004005A1063461E18012321680B4003D198
:101F30000D219E4A1170DEE749108A4200DA0A003C
:101F40000434B442F0D1012352001343D3E73B00E1
:101F50000122083B1968A40011421DD03B1F1B68D9
:101F6000134219D0114113410022994200DA043280
:101F70003B1B1A608D4B3F1B1B780437002B01D095
:101F8000FFF77FFA2B68019A1C121340884A9B00C6
:101F90009B580435FFF757FA02203B1F1A6840424E
:101FA000FFF7F2F83E1B3060E4E73B00083B19689E
:101FB0000123A40019421ED03A1F12681A421AD0F7
:101FC00019415010CB0FD217884253413A1B9B0046
:101FD0001360764B3F1B1B780437002B01D0FFF7B3
:101FE00050FA2B68019A1C121340714A9B009B58AF
:101FF0000435FFF728FA01203B1F1A684042FFF71B
:10200000C3F83E1B3060E4E73B00083B18683B1F09
:102010001968A600BE1B0423814202D0042802D8FE
:102020000023336018E001239C461842F8D10F23A7
:1020300002681A40042AF3D163461942F0D10429F8
:10204000EED90B680B321340042BE9D1FFF714F9DA
:10205000431E984180003060544BA4001B783F1B06
:102060000437002B01D0FFF70CFA2B68019A1C12E1
:1020700013404F4A9B009B580435FFF7E4F93B009F
:10208000083B18683B1F1968A600BE1B002381424D
:1020900002D0042802D80423336018E001239C46B0
:1020A0001842F8D10F2302681A40042AF3D163467C
:1020B0001942F0D10429EED90B680B321340042BDE
:1020C000E9D1FFF7D9F84342584180003060374BDF
:1020D000A4001B783F1B0437002B01D0FFF7D1F978
:1020E0002B68019A1C121340314A9B009B580435FF
:1020F000FFF7A9F93B000122083B1968A40011422F
:102100001ED03B1F1B6813421AD05B104A10D80F19
:10211000C9179A4241413B1B89001960234B3F1B61
:102120001B780437002B01D0FFF7ABF92B68019A1D
:102130001C1213401E4A9B009B580435FFF783F97D
:102140003B1F1A680120FFF71FF83E1B3060E5E7D0
:102150003B000122083B1968A40011421DD03B1F1F
:102160001B68134219D0114113410022994200DD2E
:1021700004323B1B1A600D4B3F1B1B780437002BAE
:1021800001D0FFF77EF92B68019A1C121340084A10
:102190009B009B580435FFF756F93B1F1A68022035
:1021A000FEF7F2FF3E1B3060E5E7C046A4020020C8
:1021B0007CD000003B1F1B68A400043B5A1E9341C7
:1021C0003A1B17009B001360F44B04371B78002B5D
:1021D00001D0FFF756F92B68019A1C121340F04A00
:1021E0009B009B580435FFF72EF93B00083B18680D
:1021F000FFF722F83B1F06001868FFF71DF832189A
:102200000120A4003B1B1F00520002431A60E34B55
:1022100004371B78002B01D0FFF733F92B68019AA4
:102220001C121340DE4A9B009B580435FFF70BF944
:102230003B00083B1868FEF7FFFF3B1F06001868CD
:10224000FEF7FAFF321A0120A4003B1B1F005200C8
:1022500002431A60D14B04371B78002B01D0FFF7E3
:1022600010F92B68019A1C121340CD4A9B009B5811
:102270000435FFF7E8F83B00083B1868FEF7DCFF81
:102280003B1F06001868FEF7D7FF02000120A400DC
:102290003B1B1F007243520002431A60BF4B0437BE
:1022A0001B78002B01D0FFF7ECF82B68019A1C1269
:1022B0001340BB4A9B009B580435FFF7C4F83B1FF3
:1022C0001868FEF7B9FF061E17D11F23B34A137013
:1022D000A4003B1B1F001E60B04B04371B78002B73
:1022E00001D0FFF7CEF82B68019A1C121340AC4ABC
:1022F0009B009B580435FFF7A6F83B00083B186885
:10230000FEF79AFF310007F07FF9012640000643EF
:10231000DEE73B1F1868FEF78FFF061E17D11F234D
:102320009E4A1370A4003B1B1F001E609B4B04378A
:102330001B78002B01D0FFF7A4F82B68019A1C1220
:102340001340974A9B009B580435FFF77CF83B00ED
:10235000083B1868FEF770FF310007F03BFA0126D2
:1023600049000E43DEE73B1F1868FEF765FFC21702
:10237000801850400122A4003B1B1F004000104366
:102380001860864B04371B78002B01D0FFF779F8D3
:102390002B68019A1C121340814A9B009B580435FC
:1023A000FFF751F8A300FE1A07943068012C23D1DF
:1023B000FEF742FF049009F04BFD0499002900DC70
:1023C000012107F007FA0C190121079B64000C4357
:1023D00034609E00714BBF1B1B780437002B01D06B
:1023E000FFF74FF82B68019A1C1213406C4A9B00B0
:1023F0009B580435FFF727F8FEF71EFF04007068AE
:10240000FEF71AFF0130031B0493D4E7A300FE1A62
:1024100031002000049301F047FD049B3060FF1A57
:102420005E4B04371B78002B01D0FFF72AF82B688E
:10243000019A1C1213405A4A9B009B580435FFF71F
:1024400002F83B00083B1868FEF7F6FE3B1F06004B
:102450001868FEF7F1FE02000120A4003B1B1F00DC
:102460003240520002431A604C4B04371B78002B59
:1024700001D0FFF706F82B68019A1C121340484A56
:102480009B009B580435FEF7DEFF3B00083B1868B5
:10249000FEF7D2FE06003B1F1868FEF7CDFE3200A5
:1024A00002430120A4003B1B1F00520002431A609C
:1024B0003A4B04371B78002B01D0FEF7E2FF2B6864
:1024C000019A1C121340364A9B009B580435FEF7B4
:1024D000BAFF3B00083B1868FEF7AEFE06003B1F44
:1024E0001868FEF7A9FE320042400120A4003B1B01
:1024F0001F00520002431A60284B04371B78002B40
:1025000001D0FEF7BEFF2B68019A1C121340244A2B
:102510009B009B580435FEF796FF3B1F1868FEF79B
:102520008BFEC0430122A4003B1B1F004000104350
:1025300018601A4B04371B78002B01D0FEF7A1FF5F
:102540002B68019A1C121340154A9B009B580435B6
:10255000FEF779FF3B00083B1868FEF76DFE0600AA
:102560003B1F1868FEF768FE3200824051000122CE
:10257000A4003B1B1F000A431A60084B04371B785A
:10258000002B01D0FEF77DFF2B68019A1C1213402F
:10259000034A9B009B580435FEF755FFA402002018
:1025A0007CD000003B00083B1868FEF745FE0600A3
:1025B0003B1F1868FEF740FE320002415100012225
:1025C000A4003B1B1F000A431A60DE4B04371B7834
:1025D000002B01D0FEF755FF2B68019A1C12134007
:1025E000D94A9B009B580435FEF72DFF3B000C3B5E
:1025F0001868FEF721FE3B00083B06001868FEF74E
:102600001BFEF1170200C317300007F035F93B1F1E
:10261000049005911868FEF70FFE020004980599D2
:1026200007F0DEF843000120A4003E1B37001843EA
:10263000C44B30601B780437002B01D0FEF721FF1C
:102640002B68019A1C121340BF4A9B009B5804350B
:10265000FEF7F9FEA300FE1A310020000493FEF7F6
:10266000D7FB049B3060FF1AB64B04371B78002B56
:1026700001D0FEF706FF2B68019A1C121340B24AE4
:102680009B009B580435FEF7DEFEA300FF1A3900BD
:102690002000FEF7D5FBAB4B1B78002B01D0FEF7DB
:1026A000F0FE2B68019A1C121340A74A9B009B580E
:1026B0000435FEF7C8FEA300FE1A31002000049383
:1026C000FEF7FEFB049B3060FF1A9E4B04371B781D
:1026D000002B01D0FEF7D5FE2B68019A1C12134087
:1026E000994A9B009B580435FEF7ADFEA300FF1AE4
:1026F00039002000FEF768FC924B1B78002B01D0BC
:10270000FEF7BFFE2B68019A1C1213408E4A9B00F5
:102710009B580435FEF797FEA300FE1A31002000F7
:102720000493FEF7C3FC049B3060FF1A854B04370B
:102730001B78002B01D0FEF7A4FE2B68019A1C1217
:102740001340814A9B009B580435FEF77CFE3B1FDB
:10275000186801F003F83A00083A12680300A40070
:10276000D10729D4042A0CD910680F22104001384F
:1027700008280FD806F0B4FE052026220E0E0E0EF5
:1027800024007249180009F003FC434258413B1BE6
:10279000800018606B4B3F1B1B780437002B01D067
:1027A000FEF76FFE2B68019A1C121340664A9B00CD
:1027B0009B580435FEF747FE6549E3E76549E1E7C5
:1027C0006549DFE76549DDE7069B3E1DF31A5D4C71
:1027D000D82B03DD1A232370FEF753FE00F010FD03
:1027E00043000120184323783860002B02D03700C3
:1027F000FEF747FE2B68019A1C121340524A9B00B9
:102800009B5837000435FEF71EFE069B3E1DF31A4B
:102810004C4CD82B03DD1A232370FEF732FE00F058
:10282000E5FC4F4B400018400123184323783860E3
:10283000002B02D03700FEF724FE2B68019A1C12F1
:102840001340414A9B009B5837000435FEF7FBFDBF
:10285000069B3E1DF31A3B4CD82B03DD1A23237035
:10286000FEF70FFE00F0CCFC3E4B1A68831A904234
:1028700001D23D4A9B1801205B0003433B60237853
:10288000002B02D03700FEF7FCFD2B68019A1C12CA
:1028900013402D4A9B009B5837000435FEF7D3FDAB
:1028A00000F0AEFC2F4BA4001860264B3F1B1B789A
:1028B000002B01D0FEF7E5FD2B68019A1C12134096
:1028C000214A9B009B580435FEF7BDFD00F0A0FC9B
:1028D000A300002810D1FF1A1A4B1B78002B01D03F
:1028E000FEF7CFFD2B68019A1C121340164A9B007D
:1028F0009B580435FEF7A7FD3E00FF1A0123200078
:102900001A003900FEF7E6FC184C2068643002F02B
:102910004DFF002803D1043D3700FEF7C5FD039BA2
:1029200021685A78124803F074FB0123039A13704C
:1029300000F05CFC0F4B22681B68063253431818EA
:10294000FFF7EEF8A40200207CD00000B8D200000F
:10295000C0D20000C7D20000CED20000D3D2000007
:10296000FEFFFF7FD005002037894100C805002009
:10297000A50200200400002000F04AFCA30000286B
:1029800010D1FF1AF24B1B78002B01D0FEF779FD16
:102990002B68019A1C121340EE4A9B009B58043589
:1029A000FEF751FD3E00FF1A2000012300223900EE
:1029B000FEF790FCE84C2068643002F0F7FE002837
:1029C000A9D0E64803F09EF8AFE7A4003E1BFEF74F
:1029D00001FD3700DE4B30601B780437002B01D03F
:1029E000FEF74FFD2B68019A1C121340D94A9B0039
:1029F0009B580435FEF727FDD54BA4001B783F1BE1
:102A0000002B01D0FEF73DFD2B68019A1C121340EC
:102A1000D04A9B009B580435FEF715FDA4003E1BD1
:102A2000300000F022FC3700C94B30601B780437BF
:102A3000002B01D0FEF725FD2B68019A1C121340D4
:102A4000C44A9B009B580435FEF7FDFCA4003E1BC6
:102A5000300000F00CFC3700BD4B30601B780437B1
:102A6000002B01D0FEF70DFD2B68019A1C121340BC
:102A7000B84A9B009B580435FEF7E5FCA300FE1AFC
:102A800031002000049300F0F5FB049B3060FF1A36
:102A9000AF4B04371B78002B01D0FEF7F2FC2B68FC
:102AA000019A1C121340AB4A9B009B580435FEF759
:102AB000CAFCA4003F1B380000F012FCA44B1B789A
:102AC000002B01D0FEF7DDFC2B68019A1C1213408D
:102AD000A04A9B009B580435FEF7B5FCA300FE1AE4
:102AE00031002000049300F023FC049B3060FF1AA7
:102AF000974B04371B78002B01D0FEF7C2FC2B68E4
:102B0000019A1C121340934A9B009B580435FEF710
:102B10009AFCA4003F1B380000F04CFC8C4B1B7847
:102B2000002B01D0FEF7ADFC2B68019A1C1213405C
:102B3000884A9B009B580435FEF785FC0121200044
:102B400000F020FC824B1B78002B01D0FEF799FC93
:102B50002B68019A1C1213407E4A9B009B58043537
:102B6000FEF771FC0021200000F00CFC784B1B7874
:102B7000002B01D0FEF785FC2B68019A1C12134034
:102B8000744A9B009B580435FEF75DFCA4003E1B75
:102B9000300000F031FC37006D4B30601B7804379B
:102BA000002B01D0FEF76DFC2B68019A1C1213401C
:102BB000684A9B009B580435FEF745FCA4003E1B69
:102BC000300000F02DFC3700614B30601B7804377B
:102BD000002B01D0FEF755FC2B68019A1C12134004
:102BE0005C4A9B009B580435FEF72DFCA4003F1B5C
:102BF000380000F0EFFB564B1B78002B01D0FEF79E
:102C000040FC2B68019A1C121340524A9B009B58AF
:102C10000435FEF718FCA4003F1B380003F044FD08
:102C20004B4B1B78002B01D0FEF72BFC2B68019A35
:102C30001C121340474A9B009B580435FEF703FCC7
:102C4000A4003E1B300003F0DFFD3700404B306036
:102C50001B780437002B01D0FEF713FC2B68019A78
:102C60001C1213403B4A9B009B580435FEF7EBFBBC
:102C7000A4003F1B380003F0BBFC354B1B78002B36
:102C800001D0FEF7FEFB2B68019A1C121340314A5B
:102C90009B009B580435FEF7D6FBA4003E1B30007A
:102CA00003F0BCFC37002A4B30601B780437002B44
:102CB00001D0FEF7E6FB2B68019A1C121340254A4F
:102CC0009B009B580435FEF7BEFBA300FF1A39009A
:102CD000200001F04BFC1E4B1B78002B01D0FEF7AF
:102CE000D0FB2B68019A1C1213401A4A9B009B5878
:102CF0000435FEF7A8FBA300FF1A3900200001F0FD
:102D000049FA134B1B78002B01D0FEF7BAFB2B6856
:102D1000019A1C1213400F4A9B009B580435FEF782
:102D200092FBA300FF1A3900200001F057FB084B6B
:102D30001B78002B01D0FEF7A4FB2B68019A1C1214
:102D40001340044A9B009B580435FEF77CFBC046A9
:102D5000A40200207CD00000C8050020A5020020AD
:102D6000A300FF1A3900200001F060FB894B1B789B
:102D7000002B01D0FEF785FB2B68019A1C12134033
:102D8000854A9B009B580435FEF75DFBA300FE1AA5
:102D900031002000049303F097FD049B3060FF1A7C
:102DA0007C4B04371B78002B01D0FEF76AFB2B68A5
:102DB000019A1C121340784A9B009B580435FEF779
:102DC00042FBA300FE1A31002000049303F084FDAF
:102DD000049B3060FF1A6F4B04371B78002B01D027
:102DE000FEF74FFB2B68019A1C1213406A4A9B00A6
:102DF0009B580435FEF727FBA300FE1A3100200084
:102E0000049303F071FD049B3060FF1A614B04379B
:102E10001B78002B01D0FEF734FB2B68019A1C12A3
:102E200013405D4A9B009B580435FEF70CFBA30042
:102E3000FE1A31002000049303F05EFD049B306015
:102E4000FF1A544B04371B78002B01D0FEF719FBF7
:102E50002B68019A1C1213404F4A9B009B58043563
:102E6000FEF7F1FAA300FF1A3900200001F0CAF9B9
:102E7000484B1B78002B01D0FEF703FB2B68019A0F
:102E80001C121340444A9B009B580435FEF7DBFAA2
:102E9000A300FF1A3900200001F0F0FA3D4B1B7827
:102EA000002B01D0FEF7EDFA2B68019A1C1213409B
:102EB000394A9B009B580435FEF7C5FAA300FE1A59
:102EC00031002000049301F055FA049B3060FF1A92
:102ED000304B04371B78002B01D0FEF7D2FA2B6859
:102EE000019A1C1213402C4A9B009B580435FEF794
:102EF000AAFAA300FF1A3900200001F003FA254BBB
:102F00001B78002B01D0FEF7BCFA2B68019A1C122B
:102F10001340214A9B009B580435FEF794FA069B08
:102F2000039AFB1A9B101361A300FF1A39002000BB
:102F300002F026FE174B1B78002B01D0FEF7A1FAFA
:102F40002B68019A1C121340134A9B009B580435AE
:102F5000FEF779FA069B039AFB1A9B101361A300F4
:102F6000FE1A31002000049302F00AFE049B306038
:102F7000FF1A084B04371B78002B01D0FEF781FAAB
:102F80002B68019A1C121340034A9B009B5804357E
:102F9000FEF759FAA40200207CD000000023F7B508
:102FA0005A1E0192002B07DA01F0F6FA02F018FF20
:102FB00003F08EF81923019300263000194B19688D
:102FC000B14212DD184B1A6801328A420FDAF0243E
:102FD0001A601D68154F6C43E35D002B1FD0E41988
:102FE000022B06D12000FEF70DFA019BD8E7002244
:102FF000EDE7012B0DD1002801D100F0F7F8F02208
:103000006A43BB185B680A49C31A8B4201D8022382
:10301000BB54F0235D43054BEB5C022BE2D0013641
:10302000CCE7C046CC05002000000020381C002062
:103030003F420F00012200210A4B0B481A61195030
:1030400004301950A2210420C9005850C121C020C9
:103050008900800258501A60044BFC311960044BFF
:103060001A70704700A000400405000000E100E075
:10307000F505002004207047F8B550C9012322004F
:103080001A40101E2DD03340181E2AD06410002084
:103090001A2C26D81D4B761035009E4200DD1D00EF
:1030A0001B4F3B5D012B05D00121200004F008FEE1
:1030B00001233B55174B1B78002B01D1FFF7BAFFBB
:1030C0000023154A9E420DDCFF2514491448D65CA6
:1030D000B44202D15E007052D5540133042BF6D1B4
:1030E0000420F8BDD15C8C4203D10C4A5B009D5298
:1030F000F6E70133042BF5D10023D15CFF2901D180
:10310000D454F2E70133042BF7D1E9E78813000028
:10311000D8050020F50500201C0000200E0000202E
:10312000DC05000070B530C9012322001A40101ED2
:103130001BD02B40181E18D064101A2C00D919244B
:10314000174E335D012B05D00121200004F0B8FD9E
:103150000123335569100800124A1038124B90426F
:1031600004D9012252421A60042070BD1C600F482D
:1031700006F04AFA0E4B18800E4B1B78002B02D13A
:10318000FFF758FFF0E701220B4B9A64A922D20007
:103190009A588018A82280B2D2009850E4E7C0461E
:1031A000D8050020908601001800002020A107000B
:1031B0000C000020F505002000A00040030010B521
:1031C0000120002B02DC1B30FEF7FEF810BD0420AE
:1031D000704710B5002803DC1C20FEF7F5F810BD81
:1031E0000B680020DB07FAD40D30F6E70122034B11
:1031F0001A64A822D20098587047C0460080004048
:1032000010B5FFF7F3FFFA21890006F073F910BD3E
:10321000012070470048704738D300001B207047DA
:1032200070B5054E0400335C0D008B4202D004F0F3
:1032300047FD355570BDC046D805002070B5002447
:10324000084D635D012B09D10021200004F056FDDB
:103250000021200004F034FD0023635501341B2CB1
:10326000EED170BDD805002070471120704737207F
:1032700070470000F8B501240B6806000D002342DA
:1032800004D10D20FEF7A0F82000F8BD5B1004D19A
:1032900003F0D2F940002043F7E72000072BF4D8D1
:1032A0000D4A9B009C580D4F3B5D002B05D0002123
:1032B000200004F005FD00233B55012E06DD6B6860
:1032C000042B03D10221200004F0FAFC200004F0BA
:1032D000A5FB01244000DEE718D30000D80500203C
:1032E000F8B501260568354202D04468344203D15E
:1032F0000D20FEF769F8F8BD6D101A2DFBD80A4FA6
:103300007B5D012B04D03100280004F0D9FC7E55F0
:10331000064964108C4202DCE143C91721402800B1
:1033200004F002FCE7E7C046D8050020FF030000D8
:1033300070B501240D68254204D10D20FEF744F834
:10334000200070BD6D101A2D17D80024012804DD4F
:103350004C68043C63425C416400094E735DA342C7
:1033600004D02100280004F0ABFC7455280004F0C0
:10337000DBFC03000420012BE3D00020E1E7C04682
:10338000D805002070B504000D001A280ED8084E8C
:10339000335C012B04D0012104F092FC012333554E
:1033A000290020004D1EA94104F0A8FC70BDC046B4
:1033B000D8050020036810B5DA0703D40D20FEF706
:1033C00003F810BD4168581004394A425141FFF7D3
:1033D000D9FFF6E737B569460A00064B30CB30C255
:1033E00003680220042B02D100F0F8FF37BD01F082
:1033F0001DF8FBE7E0D2000010B5084C237D002B40
:1034000005D00021142004F05BFC00232375142058
:1034100004F08AFC43425841800010BDD8050020CA
:1034200010B5084CA37D002B05D00021162004F018
:1034300047FC0023A375162004F076FC4342584154
:10344000800010BDD805002070470000F7B5304D52
:10345000304E6B6C002B15D0A8240023E4003759A4
:103460006B642D4B186800280CDB2C4B19784A42F2
:103470005141C9B2197004F041FC294B1B88DF1976
:10348000BFB23751AB6C002B39D00021254B264FF2
:10349000F458A9643A780C340193244D8A4206D03A
:1034A0002B68032B03D8224AD05C04F027FC2B683E
:1034B000204A0133134004D50422013B52421343F6
:1034C00001331B4900228C462B60042B18D0604628
:1034D000C05C591CFF2802D10B000122F5E7002A2D
:1034E00000D02B60012104F009FC01233B702B6804
:1034F000114A5B009B5AE418019BA4B2F450F7BD3B
:1035000001235B422B6000233B700C4BF3E7C0466A
:10351000FCA0004000A0004018000020F40500209E
:103520000C00002044050000F3050020D405002015
:103530001C000020030000800E0000205046000008
:10354000084B094AFF201A805A809A80DA800023AB
:10355000064A07491370074A087048708870C87097
:10356000136070470E000020DC050000F30500200A
:103570001C000020D40500200122024B52421A6098
:103580007047C0461800002010B5034A06210348C2
:1035900002F0D2F810BDC046E8D20000DEDA00002A
:1035A000E12170B54902194803F0AEFF0024012261
:1035B0000320174B17491A615C500431585080188A
:1035C000083158501A60063004F022FAFF21124ADE
:1035D000A15401341B2CFBD1012200200F4B010010
:1035E0001A6004230E4A0F4D1468002CFCD02C687E
:1035F0000002013B20431160002BF5D101220A4B50
:103600001A6004F03DF901F013F970BDC01B0020F1
:103610000080004004050000D805002000D00040D4
:1036200000D1004008D5004004D00040F8B50B4E52
:10363000070030000D0003F0AFFF0400A84200DDDA
:103640002C003D00EB1B9C4205DD300003F0AEFF7B
:1036500028700135F6E72000F8BDC046C01B0020E9
:1036600010B50100014803F057FF10BDC01B00203A
:1036700010B5054C200003F05DFFE1212000490258
:1036800003F042FF10BDC046C01B0020C3070CD48E
:10369000064B1B68834208D8054B1B68984204D828
:1036A000031F1B68002B00D0180070470006002085
:1036B000FC0500200023012210B50A4899000133BF
:1036C0004250642BFAD1084C084B00211A602000AC
:1036D000074A08F0DDF8074B074A6360074B1A609A
:1036E00010BDC046902D00200406002008000020D8
:1036F000D40900003027000008060020F80500204B
:1037000010B5044B044A1A60044B054A1A60FFF7CF
:10371000D1FF10BD0006002004060020FC0500209B
:10372000D80F0020044B1B681868000980B20238CB
:10373000C343DB1718407047F805002000B59BB065
:103740000200054901A808F0E7FB01A802F0F6F91C
:1037500002F0BEFCFCE7C046BBD300000B4BC20727
:1037600004D4042804D80A4B00D00A4B1800704730
:103770000F2203681A40031D042AF7D0064B092ABA
:10378000F4D0064B032AF1D0054BEFE795D30000A8
:1037900032CF00002CCF00009FD30000AFD3000039
:1037A000A6D300000020064A0649131F18601368BC
:1037B0001B099BB202339B00D2188A42F5D3704793
:1037C00008060020D80F0020F7B50F240126314B42
:1037D000314A1968314B324D186813681F00274071
:1037E000072F26D813681B099BB202339B00D218FF
:1037F000AA42F2D300242B4EA500AD192868FFF78A
:1038000045FF01342860642CF6D1274C2068FFF76F
:103810003DFF2060254C2068002802D0FFF736FFCE
:1038200020600025224B1B680093009B9D4214DB07
:10383000F7BD1B099BB29B00D3189A42D2D01F68D8
:10384000374208D1B94206D2B84204D3043F3F6898
:10385000002F00D01F60043BEFE7F0236B43154AB5
:103860009B181A78002A01D10135DEE71F693C2335
:1038700000266B43DB199B0001930136BB1BF3D47D
:10388000019BB4001C1B0B4B1C19A069FFF7FEFE2B
:10389000A061F2E70006002008060020FC050020D9
:1038A000D80F0020902D002008000020D80F002005
:1038B000CC050020381C0020F7B50124204246D159
:1038C000234B1B689C46984241D3224B1B680193B3
:1038D00098423CD8031F1B68002B38D102000368B4
:1038E00000941B099BB2002B0FD10099131F196084
:1038F00090422CD015682B1F1B68990069180C6822
:10390000013B14600A602A00EDE79D005519296803
:10391000009C214219D18C4517D8019C8C4214D3AC
:103920000E1F3468002C10D10F680F343C40072C58
:1039300008D92F60151F2B600B680A601B099BB20A
:103940000A00D0E700993160CDE7013BCBE7F7BD36
:1039500000060020FC0500200D4970B50A000D4D41
:103960001368141F1B0926689BB2981C002E0BD0ED
:1039700000238A4200D00B0023608300C918800016
:103980001218AA42ECD370BD1B011360F7E7C046C2
:1039900008060020D80F0020F8B5124C27000F228F
:1039A0003B681D09ADB213420DD06E1CB600A74294
:1039B00004D032003900200007F057FF0022A3197D
:1039C0000436A4191A600235AD00074B7F199F42D7
:1039D000E5D31B1B9B10013B1B012360034B1C60A9
:1039E000F8BDC04608060020D80F0020F8050020CA
:1039F000F0B59BB0FFF7FAFB00240700214AA300B3
:103A0000D0580134FFF758FF642CF7D11E4B1868CB
:103A1000FFF752FF1D4B1868002801D0FFF74CFF3D
:103A200000261B4B1B689E4217DBFFF795FFFFF735
:103A3000CBFEFFF7B1FFFFF7D9FB164BC21B1B688C
:103A400015491B6801A81B099BB2023B08F064FAE8
:103A500001A802F073F81BB0F0BDF02575430F4BC1
:103A6000ED182B78002B01D10136DAE72B695C1EAB
:103A7000002CF9DBA300EB189869FFF71DFF013C50
:103A8000F6E7C046902D002008000020D80F002047
:103A9000CC050020F805002075D30000381C00205C
:103AA000F7B5174D4F1C2B6806001B680C001B094F
:103AB0009BB201929F420BDBFFF79AFF2B681B68BA
:103AC0001B099BB29F4203DB0A20FDF77DFCFEBD74
:103AD0002868A71CBA00DB1B81181B010B6029603A
:103AE0000021031F19600F231E40030024012643F9
:103AF00040C3083A9A189A42E9D9019902C3FAE7F1
:103B0000F8050020F7B503000122134004000D0062
:103B10000193002B2BD1174B1B68834227D8164BE0
:103B20001B68834223D90F23144F38600068184064
:103B3000FFF7B6FF019B3C68061E3B6017D0236869
:103B400004301B099BB29D4200DD1D00AA00211D0F
:103B5000251F07F081FEFFF725FE2E60FFF734FEDC
:103B600000232B602268064B1340236034002000A2
:103B7000FEBDC04600060020FC050020D80F002036
:103B8000F0FF0F000323043010B5C11719400918C6
:103B9000891000220420FFF783FF10BD70B50500D7
:103BA00008000C00FFF7EEFF0023002804D170BDD1
:103BB000E95CC21811710133A342F9DBE343DB175F
:103BC0001C40002304192371F1E7F0B50C009BB0F1
:103BD000022804DC1C20FDF7F7FB1BB0F0BD01231D
:103BE0000868184206D1042804D90F26016831401C
:103BF000042901D00E20EEE761680D001D40F9D1C7
:103C00000429F7D90A683240042AF3D1A2681A427B
:103C100001D10D20DFE7FFF7A1FD06006068FFF787
:103C20009DFDA768010001AC7F103000257003F0F6
:103C300078F839006423220003F0D8F8200008F057
:103C4000B1F901002000FFF7A9FFC6E710B51C4C31
:103C5000A544041E02D1FFF795FF0BE002F07AFFA6
:103C60000138062828D805F03BFC09091118290459
:103C7000240000208023DB009D4410BD200002F0C2
:103C8000E5FF011B2000FFF789FFF3E7200002F0AA
:103C90008BFF430001201843ECE780226946D200E5
:103CA000200002F098FF684608F07CF901006846A1
:103CB000E9E704210348E6E70020CCE70420D9E740
:103CC00000FCFFFF04D4000070B50C00022803DCE8
:103CD0001C20FDF779FB70BD01230868184206D14E
:103CE000042804D90F2501682940042901D00E2099
:103CF000EFE761681942FAD10429F8D90A682A4025
:103D0000042AF4D1A2681A4201D10D20E1E7FFF79D
:103D100025FD05006068FFF721FDA468010064101F
:103D2000280002F0FEFF210003F03BF8FFF78EFFB2
:103D3000D1E770B50D00012803DC1C20FDF744FB22
:103D400070BD01240868204206D1042804D90F213F
:103D500002680A40042A01D00E20EFE76A68224276
:103D6000FAD1042AF8D913680B40042BF4D1FFF7D9
:103D7000F5FC06006868FFF7F1FC0100300002F076
:103D8000D0FF03F052F840002043D9E7F8B5070010
:103D90000C001C20012F0BDD01250868284206D1EC
:103DA000042804D90F2102680A40042A03D00E20F7
:103DB000FDF70AFBF8BD62682A42F8D1042AF6D959
:103DC00013680B40042BF2D1FFF7C8FC06006068B3
:103DD000FFF7C4FC0100022F14D0A4682C4211D0BC
:103DE0006410300002F09DFF050002F0B3FE0128D0
:103DF00011D1002C02DD0135012C06D12800FFF77E
:103E000025FFD7E701246442EBE7280002F02AFFF0
:103E1000013C0500F0E70228F0D1002CEEDD013571
:103E2000012CEBD000222800110002F04DFF02F01F
:103E300019FF013C0500F3E710B5012408680440B0
:103E400016D04410200005F073FE154905F03EFD24
:103E500007F024FC04F076F80022124B06F0D8FD9F
:103E600004F018F807F0AAFB43000120184310BD26
:103E7000042810D90F2302681340042B07D1FFF741
:103E80006DFC21000A2208F055F90400DAE7032B43
:103E900001D10430F5E70D20FDF796FAD2E7C046D0
:103EA000D30237390000D040086870B501240500FE
:103EB000254006D1042804D90F2302681340042B9F
:103EC00003D00E20FDF780FA70BDFFF747FC0378A2
:103ED0002900233B5A4253411022C01808F02AF906
:103EE00080239B05C218044B9A4201D91420E9E7AC
:103EF00040002043E8E7C046FFFFFF3F10B5034AFC
:103F00000621034801F018FC10BDC046D4D30000C0
:103F1000CCD300000020704710B51E20FDF754FAE6
:103F200010BD10B51E20FDF74FFA10BD10B51E20B4
:103F3000FDF74AFA10BD10B51E20FDF745FA10BD79
:103F400010B51E20FDF740FA10BD10B51E20FDF77C
:103F50003BFA10BD10B51E20FDF736FA10BD10B5A6
:103F60001E20FDF731FA10BD10B51E20FDF72CFA0A
:103F700010BD10B51E20FDF727FA10BD10B51E208C
:103F8000FDF722FA10BD10B51E20FDF71DFA10BD79
:103F900010B51E20FDF718FA10BD10B51E20FDF754
:103FA00013FA10BD10B51E20FDF70EFA10BD10B5A6
:103FB0001E20FDF709FA10BD10B5034A1121034870
:103FC00001F0BAFB10BDC04640D40000C8D40000C8
:103FD0000120034B1860034B1B6883401843704754
:103FE000FC0F0020DC0F0020F0B5EFF3108101235F
:103FF000194083F31088134C134AA4461268134ED9
:10400000013A9340124F134A002B17D01468034211
:104010000FD03D682C60C046C046C046C046C04672
:10402000C046C046C0460C4C1568246825605B0835
:10403000EAE765462C6014683460F8E781F310887D
:10404000F0BDC04608050050200000200C050050BF
:10405000E80F0020F00F0020E40F002030B585B0FD
:1040600001AD0C220649280007F0F6FB0024285D6C
:1040700001210134FFF7D4F80C2CF8D105B030BD84
:10408000B1D50000F7B56A463B4B01AE138006235D
:1040900093703A4B33800F23B370FFF7A7F8384B78
:1040A000384DC0182B68984201D200232B602C6831
:1040B000002C41D1375D01213800FFF7B1F8013400
:1040C0000021380003F01AFE032CF3D1002401274D
:1040D0006B461E5D39003000FFF7A2F8013439004D
:1040E000300003F00BFE032CF2D1C8200138C0468B
:1040F000C046C046C046C046C046C046C046C04690
:10410000C046C046C046F1D16B4600211878FFF783
:1041100087F86B4600215878FFF782F86B4600213C
:104120009878FFF77DF8FFF761F8FA2300241B0168
:10413000C01828602000FEBDFFF758F82B68002447
:104140009842F7D3042003F069FC0600052003F031
:1041500065FC3618062003F061FC0B4B9B1B181AFC
:104160000A4BA04206DB18600023094A2B6013604B
:104170000124DFE71C60F7E7040500000D0E0000D6
:1041800010270000F40F002043030000DC0F002084
:10419000FC0F00200022054B10B51A60044B1B6871
:1041A000934201D002F076FC002010BDF80F0020F1
:1041B000E41A002010B5041E10DA1A240A4BA400D9
:1041C000E25801239340094A09491360094A1160E2
:1041D000094A0A4911600A4A136010BDFFF71EF828
:1041E000A042EADDEAE7C046ECE20000F00F002062
:1041F00008050050E80F0020E40F00200C050050D7
:1042000018050050F0B53B4B85B01B680C00002B27
:1042100003D101204042FFF7CDFF2468012227008F
:10422000174028D0FF2360121840334967146610E6
:1042300040431F401E4005F0E7F9050438002E49B1
:10424000784305F0E1F90002054330002A49704344
:1042500005F0DAF9294B28431B68202B06D16400AE
:10426000A40E274BA400E35800021843FFF7BCFE3E
:10427000002005B0F0BD042CFAD90F2321680B40B3
:10428000092BF5D1636803925B100193019B9F4258
:10429000EEDABB00E3189E68039B1E4228D0FF2382
:1042A0007012184072101A401349751440431D4093
:1042B000009205F0A9F9030428000F49684302930E
:1042C00005F0A2F9029D0002054300980A49404307
:1042D00005F09AF9094B28431B68202B06D176007C
:1042E000B60E074BB600F55800022843FFF77CFED8
:1042F0000137CBE7F00F0020590600002000002016
:1043000098D700000200086810B5C3070FD5401009
:104310001823012A03DD4A68042A00D10833054A1C
:104320001360FEF7A1FFFFF745FF002010BD01203D
:104330004042EDE72000002010B50124044002D0E7
:104340004410200010BD042810D90F230268134028
:10435000042B07D1FFF702FA21000A2207F0EAFE38
:104360000400EEE7032B01D10430F5E70D20FDF743
:104370002BF8E6E70868F8B5C3071AD5FFF7DCFFA6
:104380000300203B5E2B25D80520434301221D1846
:104390000020114E9D4219D005211024F75C3C42AB
:1043A00000D080180139520064100029F7D1013380
:1043B000F0E704280ED90F2203681A40042A09D115
:1043C0001B099BB2002B05D00379DAE701234000DB
:1043D0001843F8BD0120FCE7BDD5000070B50868A2
:1043E0000D00FFF7A9FF04006868FFF7A5FF621E34
:1043F0000100042A14D8451E042D11D805236B434F
:104400009B18012215009D402B00064805682B4390
:104410000360054B1B68002B02D0200002F03BFB21
:10442000002070BDF80F0020E41A002070B5086865
:104430000D00FFF781FF04006868FFF77DFF621E33
:104440000100042A13D8451E042D10D805236B4300
:104450009B1801229A400748036893430360064B68
:104460001B68002B03D00022200002F014FB002068
:1044700070BDC046F80F0020E41A0020F0B505001A
:1044800089B008680C00FFF757FF0690022D36DD53
:104490006068FFF751FF0190A068FFF74DFF04002F
:1044A0000127231D661E0793731C0293079B9E42E0
:1044B00035D0052373430593019B019D0533049378
:1044C000049BAB421ED0042E16D86B1E042B13D8AF
:1044D0000122059B2349013B5B199A409446224ADD
:1044E0000B681068069A3A4003920DD062461A4350
:1044F0000A60012200280DD17F000135E0E7012488
:104500000194CDE7029ECFE7624693430B600028FB
:10451000F2D0039A0299280002F0BDFAECE7019B61
:104520001E1D042E1AD8012C18D1002505273B008A
:1045300021006B439B1999400B000A4A0135116811
:104540009943094B11601B68002B05D0019B002289
:10455000581D290002F09FFA052DE8D1002009B06E
:10456000F0BDC046F80F0020E41A0020086810B51E
:10457000C30703D5FFF7E0FE054B1860054B1B682A
:10458000002B03D0024B186802F086FA002010BD01
:10459000F80F0020E41A00207FB5A04C2368002B00
:1045A0000AD19F4A1268002A06D19E4B1B68002B35
:1045B00001D0FFF767FD7FBD9B4D2A68002A26D1F9
:1045C000984A1268002A1BD0FFF75CFD0028F2D041
:1045D000FFF744FD924B24681A681C60002A16D02D
:1045E000002C14D101AD0C229049280007F034F9B9
:1045F000285D00210134FEF713FE0C2CF8D1DAE718
:10460000874A1268002AE5D1002BE3D0E0E70021B9
:104610000D2003F073FB00210E2003F06FFB00213F
:104620000F2003F06BFB2E68012E5DD0022E00D10F
:10463000A2E0002E51D101363100794C04202368CC
:10464000994303F05BFB04212368052019404B428A
:10465000594103F053FB10212368062019404B42B7
:10466000594103F04BFB80212368090119404B425B
:1046700059410C2003F042FB8021236809021940B4
:104680004B4259410B2003F039FB8021236849023A
:1046900019404B4259410A2003F030FB8021236826
:1046A000890219404B425941092003F027FB802120
:1046B0002368C90219404B425941082003F01EFBF0
:1046C000802321681B0319404B425941072003F006
:1046D00015FB31000D2003F011FB2B680321581C42
:1046E00005F078F8296066E702214D4C0720236821
:1046F00019404B42594103F001FB08202168014059
:104700004B42594103F0FAFA80212368C90019404D
:104710004B425941052003F0F1FA802123684901F9
:1047200019404B425941062003F0E8FA80212368E2
:10473000C90119404B425941042003F0DFFA80219E
:104740002368890319404B4259410A2003F0D6FAE5
:10475000802321681B0419404B425941092003F072
:10476000CDFA31000C2003F0C9FA31000B2003F020
:10477000C5FA31000E20AEE72021294C072023681E
:1047800019404B42594103F0B9FA402123680820EF
:1047900019404B42594103F0B1FA802123680920A6
:1047A00019404B42594103F0A9FA8021236849007E
:1047B00019404B4259410A2003F0A0FA8021236896
:1047C000890019404B4259410B2003F097FA802190
:1047D0002368890119404B4259410C2003F08EFA9D
:1047E00080212368490319404B425941062003F0B8
:1047F00085FA80212368C90319404B42594104209E
:1048000003F07CFA802321685B0419404B42594134
:10481000052003F073FA01210F205CE7F80F002058
:10482000EC0F0020FC0F0020E00F0020B1D50000AD
:10483000012010B54042FFF7BDFC0020FFF7D4FB7C
:1048400010BD000010B5034A0921034800F074FFB1
:1048500010BDC04698D80000E0D800008023F0B515
:1048600002255B051A690A4C0A4BA1261D51032734
:104870008025F600ED00BA43884202D300221A5187
:10488000F0BD5F59002FFCD098518018F4E7C04666
:104890000405000000E0014010B5002806D1C0204A
:1048A000B02140028902FFF7D9FF10BDB02080215E
:1048B0008002C902F7E7000043425841064B4042DC
:1048C0001840B0239B02C018036800201A0E532A18
:1048D00001D11B02180A704700C0FEFF30B5012449
:1048E0008025054B054AED009C505C59002CFCD0FE
:1048F00001600021995030BD00E001400405000036
:1049000043425841074B40421840B0239B02C01815
:10491000A62310B50902DB05090A1943FFF7DEFFDC
:1049200010BDC04600C0FEFFF0B5012480260D4B2F
:104930000D4DF6005C51002902DC00225A51F0BDF9
:10494000577814783F022743947824042743D47877
:10495000043224063C439F59002FFCD010C001397B
:10496000E9E7C04600E001400405000070B505001D
:104970004B680A009C1C2100A400FFF7D5FF2819F2
:1049800070BD0000134B1B68002B0CD08022B0239D
:10499000D2029B0200280BD11A1D5B681B0E522B02
:1049A00000D110007047B022C02392025B02F1E7F1
:1049B00082420DD903681B0E522B09D14368023382
:1049C0009B00C018824203D903681B0E522BE9D00A
:1049D0000020E7E700110020F0B50020B7B0002468
:1049E000FFF7D0FF270005002600002D2ED1284D0F
:1049F0002868FFF761FF32003B00019000942549D1
:104A000004A807F089FA04A801F098F8224B642062
:104A10001C682B68A0215A425341204A5B42134034
:104A2000B02292029B18E41A6043490204F0ECFDA4
:104A3000A0225202030000921949220004A807F0A4
:104A40006BFA04A801F07AF837B0F0BDFF226B686A
:104A500029689C460233FF180B12013613409C4212
:104A600000DA1C00FF200A14024003926246014053
:104A700001920091039A0B4904A807F04DFA04A88B
:104A800001F05CF82800FFF77DFF0500ADE7C046A8
:104A900000110020EAD900000411002000C0FEFF30
:104AA00094D90000D6D9000070B50020FFF704FFAC
:104AB00004000120FFF700FF844200DA04000A4BE3
:104AC0001D686A42554128001D60FFF7E5FEA022DF
:104AD0006B4252021340054A28009B18044A611C8D
:104AE0001360FFF70DFF70BD00110020048001006E
:104AF00004110020F8B50020FFF7DEFE07000120BA
:104B0000FFF7DAFE3E00204D0643204C0DD18021F8
:104B1000C020C9024002FFF7A1FE01213000FFF7CB
:104B2000EFFE1B4B2E6023601DE0874209DD002352
:104B3000B0212B60164B89022360236800200125D9
:104B400017E0012380212B60124BC9022360F4E798
:104B5000120E522A08D0002800D023600E4800F020
:104B6000EDFFFFF7A1FFF8BD28005A68023292005E
:104B70009B188B4205D21A68561CE9D10028F2D046
:104B8000D1E72160EFE7C0460011002004110020AA
:104B90000480010004C00200AFD9000070B50020FD
:104BA000FFF7F0FEFF260500002801D1280070BDA8
:104BB00003681C143440FFF7E5FEDA2CF4D105003D
:104BC000F2E700008022F0B55200A1B00021674852
:104BD00006F05EFE802200215200654806F058FE75
:104BE000644BFF271B681A00049353425A4110007C
:104BF0000592FFF751FE049C0020631E9C415E4B12
:104C000064421C405D4BE418FFF7C8FF0600002E0D
:104C10002DD10498FFF750FE411C0598FFF770FE58
:104C2000059A574D534B2C601A60FEF721FD514BEE
:104C300064201B68A0215A4253414F4A5B421340F3
:104C4000B0222C6892029B18E41A6043490204F0D7
:104C5000DBFCA0225202030000924A49220007A86E
:104C600007F05AF907A800F069FF21B0F0BD3268DB
:104C7000131412123A403B4003921A000A3A092ACE
:104C800049D83A4B039A995C002931D110223E4809
:104C900006F0FEFD35002B6803991A123A40914246
:104CA00009D11A143A400B2A27D0132A2DD00A2AE8
:104CB00001D1354B1D602800FFF764FE051EEAD1C7
:104CC000314B196800290FD02000FFF74FFE040078
:104CD0002D4B5B195968002903D02000FFF746FED1
:104CE000040004350C2DF3D1204B0121039A995473
:104CF0003000FFF747FE060089E73B40022BDADC75
:104D0000214A9B00D3185D60D5E7102200211E4880
:104D100006F0BEFDCFE71A00153A082AE8D8144A73
:104D20000399525C002AE3D13500152B00D0150001
:104D3000300003681A143A40152A0FD01D2A00D1FA
:104D40000025FFF71FFE0028F3D1002D04D020001E
:104D50002900FFF70BFE0400054BC6E7039A1B1260
:104D60003B409A42EDD10500EBE7C0460010002021
:104D7000081100200011002000C0FEFF04C0020046
:104D80000411002079D90000202F002010B5FFF772
:104D900019FF10BDF0B585B0039203220333DC1771
:104DA000294D1440E4182B68284F5A425341802261
:104DB0005B42D202A4103B409B18A21C0291244EDD
:104DC000910000910190316800980A18934215D221
:104DD000FFF7F8FE2B685A42534180225B421F4086
:104DE000D202BF183368009A9B189F4206D2194816
:104DF00000F0A4FE0025280005B0F0BD029B356838
:104E000019066B461A7BA423DB051343FF222F00F0
:104E1000090C1943019B12041B0413401943280079
:104E2000FFF75CFD0837281D21003760FFF756FDAE
:104E3000002C04D00A9A21003800FFF775FD009B72
:104E4000083BFF183760D6E70011002000C0FEFFC6
:104E50000411002053D9000070B59AB0FFF74AFE44
:104E6000FF221E4CD2000021200006F011FDFF257C
:104E7000FFF794FE0026002814D10200C300E35877
:104E80000130591E8B41D218FF28F7D1144901A8CF
:104E900007F042F801A800F051FE124800F04EFE63
:104EA0001AB070BD03681A142A400A2A0AD11A12CD
:104EB0002A40FF2A03D0D200A1180B71A050FFF79F
:104EC00061FDD8E7132AFAD11B122B40FF2BF6D035
:104ED000DB00E2181671E650F1E7C0469825002085
:104EE0001FDA000033DA00000021094B094A59603B
:104EF0000131516059680029FCD00021196101235A
:104F000093600222044B8131FF315A501A6070477E
:104F1000FC1000400010004000E100E00222064BBF
:104F20000121DA670022054B5A61054A11615A696D
:104F3000002AFCD07047C04604E100E0FC100040AD
:104F40000010004010B5044C2378002B01D0FFF76F
:104F5000E5FF0020207010BD0912002080230120F1
:104F60005B055B6E5B001843704700000120024B3D
:104F70001B685B00184370478C1200200120024B15
:104F80001B685B0018437047240000200120024B7F
:104F90001B685B00184370479012002070B5040036
:104FA0000D001600FEF72CF9802301215B055A6ED7
:104FB0002670002653006170E1706272010A5A0A7D
:104FC0006071A171A272010C5A0C000E5B0EA670EA
:104FD0002571E1712072E272237370BD10B5044C2B
:104FE000200006F0DFFF01002000FEF7D7FD10BD16
:104FF000951200200E4B10B51B680E4C5A1C0FD09A
:105000000D4C002B0CD00D4C012B09D00C4C022B5D
:1050100006D0094C042B03D00A4C052B00D1074CB9
:10502000200006F0BFFF01002000FEF7B7FD10BD15
:1050300028000020C4DA0000C0D20000CFDA00004F
:10504000C7D20000C9DA000070B5214C2278002ACE
:105050003DD1204B01215A608022D20511605A684F
:10506000002AFCD0002207201B4B1C4901255A5066
:105070000439585008315A5019481A4958501A4999
:105080001A485A501A495A50A622D2009D50082256
:1050900018495A500431585002201749585017499E
:1050A0001748585017480439585018201649585076
:1050B000C12189005A500539FF39585892180243C6
:1050C0005A501249124A9950FFF70EFF257070BDD1
:1050D00009120020FC000040001000400C050000F8
:1050E000746962751C05000024050000200004029C
:1050F0002C05000014050000340500003C050000EC
:10510000FFFF000021100100540500000A120020DA
:105110000405000070B50E4B06001B78002B01D172
:10512000FFF792FF00200B4D2C7884420ED00A4BE3
:10513000202219780323091B1940084B4901C9187B
:10514000300006F089FB0120013C2C7070BDC04688
:105150000912002094120020081200200A120020D8
:10516000002370B588B0984235DD0D6801262C000B
:1051700034409C422FD12300042D2CD90F222B68C0
:105180001A402300092A26D16A683F2A23DD68468F
:10519000FFF7C0FF230000281DD06B4619783300AD
:1051A000A14203DB6B461B5D5B003343A200AA18E0
:1051B00001349360202CF2D1092169444A780B789C
:1051C00012021A438B781B041A43CB781B06134335
:1051D000024A13600423180008B070BD901200202A
:1051E00070B5454B8AB01B78002B01D1FFF72CFF1F
:1051F00002AC2000FFF78EFF002802D100200AB089
:1052000070BD23780B2BF9D96378012BF6D1E378A5
:10521000012BF3D100231120384E394D33602B7010
:1052200068442379374A41781360027809021143B0
:10523000827812041143C27812060A4332490A6086
:10524000002B0ED1152169444A780B7812021A43BB
:105250008B781B041A43CB781B061343336000235F
:1052600018E0012B1AD1152169444A780B781202F3
:105270001A438B781B041A43CB781A211B0613435D
:1052800033600E23627C6944934200DD13000022E8
:105290009A422CD100220420EA54B0E7022B03D119
:1052A000627B10331621EEE7042B0DD11521082265
:1052B0006944684606F0D0FA0098019902F05AFD58
:1052C00006F07CF93060CAE7052BC8D11521082209
:1052D0006944684606F0C0FA0098019902F04AFD58
:1052E00006F06CF93060627D0A231E21CBE7885CF2
:1052F000A8540132CCE7C046091200208C120020CD
:1053000095120020280000209012002010B5134BA9
:1053100004001B78002B01D1FFF796FEFFF7FEFD7E
:1053200000200F4A0F49104B545058600130106054
:1053300058680028FCD0002018610130906018697E
:105340000028FCD0094B0A481B785B011B185350FE
:10535000FFF7E4FDFFF7C8FD10BDC04609120020AD
:105360000010004004050000FC100040081200205E
:105370000A12002010B588B000281DDD0A6801213E
:1053800013000B4018D1042A16D90F2014682040AE
:10539000092811D150683F280EDD98001018806848
:1053A0000024084201D04010C4B26846C4540133FE
:1053B000202BF2D1FFF7AAFF002008B010BD00009B
:1053C00010B5002813DD0C68E30710D56410532CCA
:1053D0000DD8084B1B78002B01D1FFF735FEFFF7E6
:1053E0009DFDA123044ADB00D450FFF77DFD002082
:1053F00010BDC046091200200010004010B5002862
:105400000EDD0C68E3070BD56410FF2C08D8054BA4
:105410001B78002B01D1FFF717FE034A034BD45032
:10542000002010BD091200200010004024050000DB
:1054300013B5002814DD0C68E30711D5094B64107F
:105440000093094B0193072C0AD8084B1B78002BBB
:1054500001D1FFF7F9FD6B46054A1957054BD150AD
:10546000002016BDE2ECF0F4F8FC00040912002064
:10547000001000400C05000070B588B0002820DD49
:105480000124086804401CD104281AD90F2302689B
:105490001340042B15D1FEF761F9060006F082FDDA
:1054A0000500122800D912252A0002210D32684673
:1054B000FFF774FD6B465D73A54205DC6846FFF798
:1054C00025FF002008B070BD2300325D6B449A7345
:1054D0000134F1E7F0B50D008BB0012832DD08682A
:1054E0000122040014402DD104282BD90F23016878
:1054F0000B40042B26D16B68134223D0FEF72EF904
:105500006E6807007310019306F04CFD05000E282D
:1055100000D90E252A000121113202A8FFF73EFD15
:105520006A46127902AB5A7302AA73129373019BF3
:1055300076141B0ED67313745574A54205DC02A8AD
:10554000FFF7E4FE00200BB0F0BD3A5D02A963183E
:105550009A740134F1E730B589B0002814DD0C6885
:10556000E30711D5102268460021FFF717FD6B46AF
:105570006A4665105D73684663122D0E641493735A
:10558000D4731574FFF7C2FE002009B030BD0000CF
:10559000174B184A5968002903D00021596001317E
:1055A0009160196900291FD0002018618023DB0059
:1055B000D3581149012B18D1A923DB00D3585B42E2
:1055C0000B600E490B78032B01D801330B700320BD
:1055D0000B490B78013303400B700A495B015B18E0
:1055E000094953500123936070470860FAE7C046A9
:1055F000FC10004000100040240000209412002005
:10560000081200200A1200200405000010B5034A09
:105610001021034800F090F810BDC04644DA0000A5
:105620003BDA0000044A05491368C85401339B055E
:105630009B0D13607047C046C4160020C4120020A2
:1056400070B5114C114A2368834202DC00232360A9
:1056500016E0155C411C2E00FA3E012E05D8994239
:105660000FDA555C013D1F2D01D90800ECE7010060
:10567000151A565C6E5401318B42FADC181A206000
:1056800070BD1570FAE7C046D01A0020D016002071
:1056900010B5FDF7ABFD064B1A68824201D9002216
:1056A0001A601B68C31A034898428041404210BDEB
:1056B000C0120020204E000010B5094C094A236892
:1056C0001268934200D110BD074AD05CFDF7C8FFB5
:1056D0000028F8D0236801339B059B0D2360ECE77D
:1056E000C8160020C4160020C412002010B5040003
:1056F000064B074A1B6812689B1ADB439B059B0DF0
:10570000A34200DB10BDFFF7D7FFF1E7C41600206E
:10571000C816002070B5FFF741FAFF2504000028E5
:1057200001D1200070BD03681B142B401D2B00D13C
:105730000400FFF727F9F2E770B5074E33680B2B2B
:1057400008DC0C255D43054C013328516419616068
:10575000A260336070BDC046CC160020302F002000
:1057600010B5FBF7C7FCFFF76DF8FBF7EBFCFDF797
:105770000BFFFEF7C3FBFEF71FFCFFF747FF00F030
:1057800087FF01F08BF901F0D5FB10BD962210B513
:1057900012010021034806F07BF80022024B1A6038
:1057A00010BDC046381C0020CC050020064B074A1F
:1057B0001B6812689B1ADB439B059B0D01228342E9
:1057C00000DC002210007047C4160020C81600201C
:1057D000F8B505000C0016001F1E0ED10320FFF7C0
:1057E000E5FF002808D0FA20FFF71CFFE8B2FFF71A
:1057F00019FFE0B2FFF716FFF8BD501DFFF7D6FF07
:105800000028F9D0FB20FFF70DFFE8B2FFF70AFFF1
:10581000E0B2FFF707FFF0B2FFF704FF3012C0B2AB
:10582000FFF700FF3C00E31B9E42E5DD2078FFF719
:10583000F9FE0134F7E7000070B50024F0250B4BAA
:105840001B68A34202DCFFF7A1FF70BD2B0063437E
:10585000074A9B181A78002A05D05978002311208E
:105860001A00FFF7B5FF0134E9E7C046CC05002078
:10587000381C0020F8B507000024F0252B006343F6
:105880000C4A01349E18B74211D0317800290BD050
:105890000133D15C002311201A00FFF799FF2A0081
:1058A0000021300005F0F4FF0A2CE7D1F8BD024BCF
:1058B0001C60F9E7381C0020CC050020F0B515006D
:1058C00001222F007A4C1740A54401900291002F2D
:1058D00011D005AB1A706A105A70120E1A71052297
:1058E000691299706D140299DD70FFF771FFCF2373
:1058F0009B009D44F0BD042D2AD90F242868044044
:10590000042C32D1022304AA28001371FDF726FFCC
:10591000050006F047FBC82302009B00984200DD0B
:105920001A007C1C97420DD1984206D9614804ABFD
:1059300003226149C01805F08FFF220005AB0299D0
:105940000198D2E72700611E695C05ACE155E8E7E4
:10595000042D00D0A7E0032304AA043D13716B4279
:105960005D4105AB55710222E9E7092C7ED1042285
:1059700005AB1A706A685110009169465212097895
:105980009A70009A59701F2A01DD202200926A46FF
:10599000127806ACDA70009BBB4202DC05ABE21A5F
:1059A000CDE70126BB00EB189868064006D1042815
:1059B00037D90F210368194002290CD10123237024
:1059C0004310637042121B0E4014A270E0702371EA
:1059D00005340137DFE7042921D102232370FDF7C5
:1059E000BDFE039006F0DEFAA31C0C2809D86070F7
:1059F000864201D19C19ECE7039A925D9A550136D3
:105A0000F6E70C226270039A925D9A550136092ED0
:105A1000F9D12E23E372237363730E34D9E701297E
:105A200007D1032304382370434258416070023485
:105A3000CFE7092909D10423237043685A10627003
:105A40005B12A370E6700434C3E703290BD105236E
:105A500023700068020992B2430F92000B40D31AE0
:105A600063701B12EDE726700134B2E7032C00D0FF
:105A70003DE7052205AB01091A7089B2420F890082
:105A800022408A1A11125A709970642A00DD642229
:105A90000421DA70081F824201DC04324FE7685C9F
:105AA00058540131F6E7002D00D020E753E7C046F7
:105AB000C4FCFFFF220300003CCF000070B50200D1
:105AC0000024F0210D4E080060438019457895426E
:105AD00003D001340A2CF6D170BDF022002105F06C
:105AE000D7FE074A1368013BA34200D1146000238C
:105AF00029001A001120FFF76BFEEDE7381C00208B
:105B0000CC05002010B5B2B002236A460400137021
:105B100006F048FAC72800D9C7200023984207DCBE
:105B2000421C6B46FE211420FFF752FE32B010BD1E
:105B3000694601335A1EA25CCA54EFE730B5B3B0D0
:105B400002236A460500137006F02CFA0400C728E9
:105B500000D9C72400239C420BDC20003230FFF721
:105B6000C5FD621C6B46FF211420FFF731FE33B0E8
:105B700030BD694601335A1EAA5CCA54EBE70000E7
:105B8000F0B5BBB004900C00012803DC1B20FBF730
:105B90001BFC51E02A4B08680293C30709D4042870
:105BA00007D90F2302681340042B02D1FDF7D6FD5D
:105BB0000290234B60680393C30709D4042807D9D4
:105BC0000F2302681340042B02D1FDF7C7FD039099
:105BD00000271C4B1B680693069BBB420BDC039BF8
:105BE000194A0093C821029B08A806F063F908A887
:105BF000FFF7A4FFCAE70C267E43144B0299F61860
:105C0000306806F0C5F9051E05D17368B6680793BC
:105C1000079B9D4201DB0137DEE73068039905965B
:105C200006F0B6F90836002808D121000498059B33
:105C3000083102385B6898473BB0F0BD0135E7E7B3
:105C4000CBD30000CC160020A0DB0000302F0020BA
:105C5000F7B5234B06001B68F02100930023009A40
:105C60009A4211DC0024F0231A0062430192019948
:105C70001C4A55182F78002F12D001340A2CF3D16A
:105C80001948FFF75BFF29E00A005A4315488218BC
:105C90005078B04202D11278002A1FD10133DEE7DA
:105CA000F0223900280005F0F3FD02230D4A019986
:105CB000EB6053540D4AF1008A58009B6E70AE7031
:105CC000AA602F616F61A34202DC054B01341C60A6
:105CD000002331001A001020FFF77AFDF7BDC046FF
:105CE000CC050020381C0020E9DF000098250020AA
:105CF00010B5FFF7A1FDFF24084AE3005B429B18A3
:105D0000074AD35C043B012B03D8E043C0B2FFF742
:105D10009FFF013C002CEFD110BDC046FC070000E6
:105D200098250020F7B50F00FF247F2501901E4A1B
:105D3000E300D31A1D4A9A181278062A01D0032AC2
:105D400020D1FF22D2009B18186883682B401C2B9F
:105D500018D1C3681A002A40042A13D102692A40C4
:105D6000192A0FD11B0A01339B000C30C018FDF714
:105D7000F5FC03780600002B10D006F013F9002381
:105D8000B84209D0013C002CD1D1F7BD019AF15C99
:105D9000D25C9142F6D101339F42F7DCE043C0B2BE
:105DA000FFF756FFEEE7C04698250020FC070000ED
:105DB00070B50500FF24084AE3005B429B18074AC0
:105DC000D35CAB4203D1E043C0B2FFF741FF013CDB
:105DD000002CF0D170BDC046FC07000098250020C3
:105DE000F7B5FDF703FA574B1A68824201D9002232
:105DF0001A601A685449821A8A420DD9FF225349FF
:105E00001860D3005248CB1A1B181B78073B022B93
:105E10000CD9013A002AF4D1F7BD0720FFF7C8FFDB
:105E20004C4B27E00820FFF7C3FF38E0FDF7E8F907
:105E3000071E00D101270020FDF7DEFA01900020A7
:105E4000FDF7EEFA019B0090434C444D002B12D01D
:105E50002368002B6ED12B682760002B6ED0404B3F
:105E600001261B78002BD8D10920FFF7A1FF394B61
:105E70001E703B4B1E70009B002B12D02B68002B1A
:105E80000FD123682F60002B1ED0324B01261B78C8
:105E9000002BC7D10920FFF78BFF2E4B1E70304B14
:105EA0001E702368002B0FD02A4E3278002A0BD1A7
:105EB0009F4200D227602368FB1A312B04D90720A8
:105EC000FFF776FF012333702B68002B0FD0244E91
:105ED0003278002A0BD1BB4200D92F602B68FF1A01
:105EE000312F04D90820FFF763FF012333702368A3
:105EF000002B0CD0019B002B09D1164E3378002BC0
:105F000002D10720FFF754FF0023236033702B6872
:105F1000002B00D180E7009B002B00D07CE7104CC9
:105F20002378002B02D10820FFF742FF00232B60CB
:105F3000237071E7009A002AA0D1B5E7009B002BDF
:105F40009FD1AEE7BC1200200F270000982500204B
:105F5000FC070000B0120020AC120020B412002098
:105F6000B812002037B500240500FFF765FC01A832
:105F70000194FDF72FFA21002000FEF70BF9FEF740
:105F80000BFBFDF761FAFDF7DBFAFDF7F5FAFEF71B
:105F90004FFCFDF753F9A54204D0FDF78BFB0248F7
:105FA000FFF7CCFD37BDC046DADF0000002310B597
:105FB00001001A001120FFF70BFC10BD07B56B465E
:105FC000197069465A7013128B701314120ECB702D
:105FD0000A716B46010005221320FFF7F9FB07BD8C
:105FE00010B50A0001001220FFF768FC10BD70B563
:105FF00005000C00FDF70CF9002809D02000323014
:10600000FFF774FB2B00220000211B20FFF7E0FBB1
:1060100070BD10B50C000300110014202200FFF722
:10602000D7FB10BD012370B5FF24084A41185B421D
:10603000884201D3D84370BD06781D0A23407340BF
:106040009B009B5801306B40F2E7C046BCDB000070
:1060500013B50400FE2813D80A4BC200D0580028FC
:106060000ED0436808309900FFF7DCFF019009204B
:10607000FFF73CFB01AB042221001720FFF7A8FB30
:1060800013BDC04698250020F7B50190FFF742FBED
:1060900001250400FF276D42002C01D12800FEBD20
:1060A000266833143B40152B0DD12100019808318F
:1060B00005F06EFF002801D135123D402000FEF7AB
:1060C00061FC0400E8E71D2BF8D101256D42F5E7DE
:1060D000F0B580279FB0FFF7EFFAB54CB54D2068BB
:1060E000FF00391A4019FDF7A1FA23680600C3180A
:1060F0002360002B0ED11FB0F0BD2068391A28187C
:10610000FDF794FA236806001B182360FDF76EF86C
:10611000A94B1860002EF0DC2B78FA2B00D00EE192
:106120002368022B07DCFFF7B3FA0028E3D0012035
:10613000FFF786FADFE76B78AC78981E182800D94D
:10614000F2E003F0CDF90D2024282B34F13E707AD3
:106150007E94CDDEF1F1F1F1F1F1F1F1F1F1EC002C
:10616000FF2C0ED02000FFF7A9FC0022934BE1008A
:10617000CA505B181A712100009213001320FEF719
:1061800009FE0320D4E72000FFF762FDF9E72000B5
:10619000FFF794FCF5E7FFF7ABFDF2E7FFF74CFBE9
:1061A0000020FFF7DFFE8648FFF7C8FCE9E7632C15
:1061B000E7D8844BA200D25821001520FFF77EFBC0
:1061C000DFE7FFF7A7FAFF270400002CD9D02568E6
:1061D0002B143B40152B04D02000FEF7D3FB04000A
:1061E000F3E72000083005F0DDFE06000530FFF77C
:1061F0007DFAFB20FFF716FA2D121D20FFF712FA89
:10620000E8B2FFF70FFAF0B2FFF70CFA3012C0B2A3
:10621000FFF708FA25002B1B9E42DDDD287AFFF7E9
:1062200001FA0135F7E700211D2000910B000A005B
:10623000FEF7B0FDFDF73EFAA3E72000FFF708FFE9
:106240009FE7FCF7E7FF05AC5F4A642100905F4BD6
:10625000200005F02FFE02232000237005F0A2FE8F
:106260002300020000211620FFF7B2FA89E700267A
:10627000524AF3009B181C68002C28D01B7903930A
:10628000636808349F00B81D0293FFF72FFAFB20C4
:10629000FFF7C8F901207D1CFFF7C4F9F0B2FFF742
:1062A000C1F9E8B22D12FFF7BDF9E8B2FFF7BAF96C
:1062B0000398FFF7B7F9E719A7420CD8FFF7FCF9E5
:1062C00005230298584301F0F9FAFFF7F5F9013672
:1062D000FF2ECDD155E72078FFF7A4F90134EBE785
:1062E0000024FFF7A9FA2200210000942300DA20FD
:1062F000FEF750FDFF222100D200304805F0C8FA19
:1063000098E7012C02D1FEF767FB3AE7022C02D195
:10631000FEF73CFD35E70120FFF724FE31E70023BF
:1063200021001A001A209FE71A00C83A052A00D94E
:1063300027E7002218001100FAF710FF21E7FB2BD6
:1063400000D0F4E62268042A00DCECE62E79E87836
:106350001F4B360206439E4200DDE8E6331D9A429B
:1063600000DCE0E6EB5CFE2B00D0E0E66878AC7881
:10637000771E1B2800D17DE02ED8072863D008287F
:1063800038D001282DD1FF2C10D02000FFF796FB2C
:106390006D79104AB31E009221002A000A20FEF7F0
:1063A000F9FC064BE400E0501B191D71701DBFE69F
:1063B000D01A0020D0160020C012002098250020FE
:1063C000BCDF0000902D0020D3DF0000CEDF0000F6
:1063D000F6030000D61600201D285DD04FD31E28DE
:1063E00071D00300C83B052BE0D8404A3900FAF7CA
:1063F000B5FEDBE7632CD9D86A79022A13D0032AC9
:106400001BD0012AD2D1E979AB79090219432B7A41
:10641000A4001B0419436B7A1B060B435B00134358
:10642000334AA350C2E7002FC0DDB11E3148FDF74B
:10643000B5FB2F4BA400E050B8E7AB79A4005A1E7F
:1064400093419B00ECE7632FB0DC05AD3A00274990
:10645000280005F001FA00232800EB55FFF714FE91
:106460000028A3DB224B8000C25821001520FFF733
:1064700025FA9BE739001D48FFF754FC96E7FF2CEF
:1064800094D06A79022A91D81A490B2000912100F0
:10649000B31EFEF77FFC89E7632F00DD632700232F
:1064A00005A9BB420ADBFB430022DB173B40CB18AC
:1064B0001A70152000917B1C2100EAE7EA18527936
:1064C000CA540133EDE7012C00D06FE7002F00DC48
:1064D0006CE76B79002B03D01C00322B00DD3224DB
:1064E00064235C43044B1C6060E7C046D516002063
:1064F000902D0020D61600200400002001207047B7
:1065000010B5064C200000F045FE0549200000F0C3
:1065100075FE0122034B1A6010BDC046081B002007
:10652000801A0600D41A002010B501210D20FCF7B6
:1065300077FE01210E20FCF773FE00210F20FCF7EF
:106540006FFE044C200000F067FD1021200000F0D9
:106550007FFD10BDE81A0020F8B501250C682C421B
:1065600003D10D20FAF730FFF8BD64102DD4FCF7ED
:1065700055FEA04229DB00212000FCF751FEFA2243
:106580002900D200200001F0CBF900281DD0002501
:1065900000270726FA2201219200200001F0C0F90D
:1065A000002812D0282802DD0123B3401F43013EFA
:1065B000F0D20E4EAF550135052DE9D1012206214D
:1065C0000920FDF76DFA002801D10020CCE70B234C
:1065D000012443600023F25C9900520041182243D9
:1065E00001338A60052BF6D1BEE7C046D81A0020D9
:1065F00010B504680D20E30703D56410FF2C03D900
:106600001720FAF7E1FE10BDFFF78EFFE1B2024856
:1066100000F040FD0020F6E7E81A002010B5FFF773
:1066200083FF0021034800F035FD4300012018439B
:1066300010BDC046E81A0020A02101220B4BC90062
:106640005A500B480B4958500B491A604A68002AA7
:10665000FCD000224A60A121C9005858012159608C
:10666000A021C9005A50054BC01870470070004067
:106670006A10000004050000FC700040FBFDFFFFF5
:1066800010B5FFF7D9FF43000120184310BD0000EB
:1066900010B5034A0A210348FFF74EF810BDC04663
:1066A00000E0000050E00000F8B5012306681E423B
:1066B00005D045681D4202D084681C4203D10D20DC
:1066C000FAF782FEF8BD76101520802EF8D86D10EE
:1066D0001620FF2DF4D86410FF2C01D91720EFE706
:1066E0000B4B1B68002B01D1FFF70AFF094FF1B2DA
:1066F000380000F01AFEE9B2380000F017FDE1B2F0
:10670000380000F013FD380000F07AFE0020D9E7D1
:10671000D41A0020081B0020F7B501221400904273
:1067200022DD0D682A421FD01D4B15411B684C68A5
:10673000002B01D1FFF7E4FEE9B201272500194E35
:106740003D40300000F0F1FD002D0FD03C41300005
:10675000E1B200F0EBFC300000F052FE0024A04259
:1067600002D02320FAF730FE2000FEBD042CF2D91F
:106770000F2322681340092BEDD163685B1001934E
:10678000019BAB42E7DDAB00E3189968394204D0C6
:106790004910C9B2300000F0C9FC0135F0E7C0462D
:1067A000D41A0020081B0020154B70B51B6805008B
:1067B0000E00002B01D1FFF7A3FE124CEDB2290011
:1067C000200000F0B2FDF1B2200000F0AFFC00218B
:1067D000200000F0B5FD002801D0404270BD72B627
:1067E00001222900200000F09BFD62B6200000F08D
:1067F0008EFC0028F2D0200000F08EFCEEE7C046B0
:10680000D41A0020081B002010B50124036823427D
:1068100002D04168214203D10D20FAF7D5FD10BD09
:106820005810802801D91520F7E74910FF2901D910
:106830001620F2E7FFF7B8FF40002043EFE710B55E
:106840000400012814D105211820FFF7ADFF7F288F
:106850002BDC03007F3301DA7F204042C8235B42F8
:1068600058437F2102F0D0FE052C00D1404210BDDC
:10687000032811D101001820FFF796FF7F2814DCB0
:1068800003007F3301DA7F204042C8235B42584334
:106890007F2102F0B9FEEAE70020052CF5D107219F
:1068A0001830FFF781FF7F2802DD0138FF38D0E77D
:1068B00003007F3301DA7F204042C8235B42584304
:1068C0007F2102F0A1FED1E710B50120FFF7B7FF4D
:1068D00043000120184310BD10B50320FFF7AFFFA0
:1068E00043000120184310BD10B50520FFF7A7FF96
:1068F00043000120184310BD10B508211820FFF7F0
:1069000053FF0300C00FC018012340101530400092
:10691000184310BDF8B501231C0098422BDD0F6809
:106920003B4228D04E6835001D4024D1042E22D988
:106930000F2231680A40092A1DD173685C10202C8F
:1069400000DD2024144B1B68002B01D1FFF7D8FD7C
:1069500072B67F10F9B2114F2200380000F0E0FC4F
:1069600062B6A54214DA380000F0D1FB002804D149
:1069700001246D002C432000F8BD380000F0CCFB52
:106980000122AB004000F31810439860AD18E8E70F
:1069900064000125EEE7C046D41A0020081B002041
:1069A00070B52B4B86B01B68002B02D10120FFF77E
:1069B00046FF01AD14220021280004F069FF254E96
:1069C0001821300000F0B1FC0321300000F0AEFBD4
:1069D0000021300000F0B4FC041E13D172B6052271
:1069E0001821300000F09CFC62B6300000F08FFBF4
:1069F000002802D0300000F08FFBA3000134E850E3
:106A0000052CF2D1019B7F2B01DD013BFF3BAA68E6
:106A10007F2A01DD013AFF3A29697F2901DD013929
:106A2000FF39C820434342434843DB11D21152434C
:106A3000C0115B4340439B18181804F0F5FD01F0AA
:106A4000C9FA04F0BBFD43000120184306B070BD35
:106A5000E01A0020081B002000207047012070472A
:106A600000207047002070470020704701207047C9
:106A700000207047002070470020704700207047BA
:106A800000207047002070470020704700207047AA
:106A900000207047704770477047000010B5034AE8
:106AA0000F210348FEF748FE10BDC046B4E00000C9
:106AB0002CE100000378013B1F2B00D97047013007
:106AC000F8E710B5FFF7F6FF0378002B0BD0013085
:106AD000222B11D10378002B03D0421C222B03D18F
:106AE0001000FFF7E7FF10BD5C2B03D14378002BAC
:106AF00000D0821C1000EDE73A2BF2D02C2BF0D006
:106B00007B2B0BD1FFF7D6FF0378002BE9D07D2B31
:106B100001D10130E5E7FFF7D4FFF5E720225B2B39
:106B200014D1FFF7C7FF0378002BDAD05D2BF0D02C
:106B3000FFF7C7FFF7E7202BD3DD2C2BD3D01900AD
:106B400091435D29CFD0222BCDD001300378002B8B
:106B5000F1D1C6E7002210B5904216D0FFF7AAFF88
:106B600003780422222B10D0023A7B2B0DD0013A5D
:106B70005B2B0AD0190030390232092905D92D2B97
:106B800005D14178303909290AD8100010BD0522F5
:106B9000742BFAD00132662BF7D001326E2BF4D071
:106BA000581E83415A42F0E770B5FFF783FF037820
:106BB00001222D2B01D18018023A00230A2502E080
:106BC0006B430130CB1801783039CCB2092CF7D99E
:106BD0005A43100070BDF8B50C001500FFF76AFFAE
:106BE0000378222B02D000232370F8BD0D236A1EE8
:106BF000210008250C260A279C4601300378222B09
:106C000002D100230B70F0E7002BFAD0441C5C2B60
:106C10000BD14378841C622B0ED0662B0ED06E2BCA
:106C20000ED0722B0ED0742B0ED0002AE9DD0B7023
:106C3000013A01312000E1E72B00F6E73300F4E7E9
:106C40003B00F2E76346F0E70923EEE710B50400E6
:106C5000FFF737FFA04202D90378202B00D910BDDF
:106C60000138F7E710B5002815D00378002B13D0B2
:106C7000FFF720FF2021037802008B4300205D2BCB
:106C800009D01000FFF71DFF03782C3B5A425341F7
:106C9000C018FFF70FFF10BD1800FCE7030000202D
:106CA00070B50C0081420EDD1A785B2A0BD1581C9E
:106CB000FFF700FF0125AC4205D0FFF7D3FF002806
:106CC00001D00135F7E770BD70B50C001500002943
:106CD00001D000230B70002820D00378002B1ED099
:106CE000FFF7E8FE037806002C2B03D10130FFF7F5
:106CF000E1FE0600337800207D2B0FD0844204D0C3
:106D00002A0021003000FFF766FF3000FFF7D9FEB0
:106D100003783A2B02D10130FFF7CCFE70BD18008A
:106D2000FCE7F0B50D0004009DB02E78002E35D0A4
:106D30002E21280005F01EF9071E14D0431B0193D5
:106D4000303E092E14D82800FFF72EFF0100200046
:106D5000FFF7A4FF0400002C20D0002F1ED0019BC1
:106D60000133ED18E1E7280005F01CF90190E7E791
:106D700023787B2B11D1601C642203A9FFF7A4FFA9
:106D8000041E0BD0019A290003A805F012F900286F
:106D9000E1D02000FFF795FEEEE7002420001DB0B3
:106DA000F0BD70B5050000200C0081421DDD2800FB
:106DB000FFF7D0FE0300681C012B14D00020022B2B
:106DC00013D10022681C1100FFF77EFF012C0CD0AC
:106DD000FFF748FF00221100FFF776FF013CF5E7BF
:106DE000FFF740FF013C012CFAD170BDF8B505005A
:106DF00000200C0016001F0081420DDD2800FFF767
:106E0000A9FE03000020022B06D1681C3A003100C5
:106E1000FFF75AFF012C00D1F8BDFFF723FF3A001E
:106E20003100FFF751FF013CF4E710B50024A04208
:106E300018D0FFF73FFE03787B2B0AD101300022E8
:106E40001100FFF741FF00280CD0FFF73AFE013494
:106E5000F5E75B2B06D10130FFF704FF002801D0D6
:106E60000134F9E7200010BDF8B5002816DD0D68E3
:106E7000EB0713D56D10013D0124FDF78FFE0026B1
:106E8000FF27644200280CD1002E21D0300005F0ED
:106E900089F801003000FCF781FEF8BD01256D4244
:106EA000EAE703681A143A40152A0BD11B123B403B
:106EB0009C4200DA1C009D4201D106000836FDF715
:106EC00061FDDFE71D2AFAD1012400266442F6E7BE
:106ED0000120013464002043DFE7000010B508689A
:106EE0000C00FCF73BFCFFF7CFF8002803DB6268DF
:106EF000024B8000C250002010BDC046902D0020E3
:106F000010B50868FCF72AFCFFF7BEF8012300283B
:106F100002DB024B8000C358180010BD902D0020EA
:106F200010B50868FCF71AFCFFF7AEF8C043C00FB5
:106F3000800010BD10B5034A04210348FEF7FCFB96
:106F400010BDC046C8E10000C2E1000010B5FCF76A
:106F500027FBFCF7D5FBFEF703FC0448FEF7EEFD2C
:106F6000FDF77AFFFEF7C4FE10BDC04617E2000031
:106F700010B5FCF713F810BD70B5002504AC2478EB
:106F80000573A94205D10A4B0A4A25210A4804F093
:106F9000F5FB01600949920052589B0002715B5851
:106FA000A40083716358856043710223C37170BD6F
:106FB0002FE200008EE200003DE20000ECE2000063
:106FC000037B002B04D14373837303610133037389
:106FD000704700001FB50191A02100240068C9007E
:106FE000D2B24450012A10D0A24209D0032A0AD0BA
:106FF000074A8350074B019AC250012343501FBDDB
:1070000002221343F4E70422FBE70622F9E7C04615
:10701000540500002405000010B50400FFF7D0FF60
:10702000A1222368A179D20099506179064A2000F3
:107030009950217904329950044B19685A689B6819
:10704000FFF7C8FF10BDC0460C050000FC1A002069
:107050004BB2002B0FDB80233F290FD81F290FD8FD
:107060000F290FD807290FD803290FD81B0601684D
:10707000074A8B50704780239B04F8E7DB04F6E750
:107080001B05F4E75B05F2E79B05F0E7DB05EEE7A0
:10709000240500000368074A99501A00FC32D168A1
:1070A0000029FCD0A321C90058580023C0B2D360E6
:1070B0007047C0461C05000007B58022074BD2056B
:1070C0001A6000229A6002321A7111230E32009364
:1070D000034905330348FFF74FFF07BDFC1A0020A3
:1070E00000300040E81A0020F8B505000E00170037
:1070F0000024BC4208D02B68315D1B6828009847EB
:10710000002801D00134F4E72000F8BD704710B525
:107110001C3000F0AFF910BD10B51C3000F09CF928
:1071200010BD10B51C3000F0ABF910BD70B5437E3A
:107130000D00002B01D1002070BD6430040000F070
:10714000A8F90028F7D12000290000F076F90120E5
:10715000F2E70000F7B50193FA23002504009B0035
:1071600083600B4B4560083303601C300F00160032
:1071700000F058F92000643000F054F96B461B7998
:10718000276166756576A5762000A375FEBDC046AD
:10719000CCE20000012330B5A024C375837D1349E0
:1071A0009B005A58437DC132114DFF32E4059200D5
:1071B0009B005B581551CC22C133FF339B001D51FE
:1071C00004690C4B5204E25005220469243BE2504E
:1071D000837D04699B005A58A123DB00E250437D64
:1071E00002699B005958044BD15030BDECE20000BD
:1071F0000C060000240500000C050000A02200235E
:1072000010B50469D200A3500A4CA1420FD90A4C10
:107210008C425B4109495B420B40CD21C9045B189C
:1072200004690749635005210369995010BDCC23B7
:107230005B04F5E7A086010090D00300000098FDF4
:1072400024050000F7B5040000200D0001938242E0
:1072500065D01600402A00D9402627001C37380088
:1072600000F0F6F8B1232269DB00D550802201231B
:10727000216992008B50A27E002A03D122691362F9
:10728000226913600025731EAB4207D1019B002BBE
:1072900004D080220221236992009950012223699F
:1072A0001A622369FC33DA68002A02D19A6A002A3A
:1072B000F9D09A6A002A0BD1DA60A3232269DB0095
:1072C000D1583800C9B2013500F0B7F8B542DAD369
:1072D000019B2269002B0FD11300FC339B6A002B0A
:1072E0000AD10133A376D3612369FC33DA6C002A17
:1072F000FCD00022DA640AE000230121A376516168
:107300001A002369FC3399680029FCD09A6023692C
:10731000FC339A6A002A01D000229A62E8B2FEBDCC
:1073200010B50123FFF78EFF10BD0300AC3310B57D
:1073300004001970643000F08BF80123637610BDEF
:107340000023020070B5AC3243760D001178B122F3
:1073500004000069D20081508022216992008B5084
:10736000226901331362226993602600643630007B
:1073700000F080F8002812D0300000F06DF81E4BAD
:107380002269D0502369FC331A6A002A02D19A6A12
:10739000002AF9D09A6A002A01D11A62E5E7236926
:1073A0000122002D0DD11900FC31896A002908D174
:1073B000DA612369FC33DA6C002AFCD00022DA643B
:1073C00007E05A612369FC339A68002AFCD0002246
:1073D0009A6000202369FC339A6A82420BD098623B
:1073E0002169064A8B588B501800022B03D0181FB6
:1073F000431E9841033070BD1C050000C40400000A
:1074000010B50121FFF79CFF10BD000010B513233C
:10741000122202490248FFF79DFE10BD00400040C5
:10742000081B002010B540220021040004F030FAAF
:10743000002320002364636410BD10B53F24026C58
:10744000531C2340446C9C4201D08154036410BD02
:107450000023036443647047436C026C934206D07C
:107460003F21C25C01330B40436410007047012090
:107470004042FBE7036C406C181A00D5403070475F
:10748000436C026C934201D0C05C704701204042C3
:10749000FBE73F22036C406C01331340181A434250
:1074A0005841C0B27047000003210A4802680A43ED
:1074B0000260094802680A4302600849084A094B09
:1074C0009B1A03DD043BC858D050FBDC00F012F8D7
:1074D000F8F71AFE240500405405004030E800008B
:1074E0000000002064020020FEE7FEE7FEE7FEE762
:1074F000FEE7FEE7014B024A1A6070472C000020AD
:107500000024F4000120704710B503681322DB69E2
:10751000984710BD70470000054B0269D1500369C0
:10752000FC331A6A002AFCD0002201201A6270473C
:107530001C050000030010B55C331A781F231A40A5
:107540001E3B19009140114AD167C22204210469EF
:107550009200A150026953600269D360A023002207
:107560000169DB00CA5001230169094A5B428B5063
:107570000169084A8B5001690C3A8B500169083245
:107580008B501430FFF764FF10BDC04604E100E0EB
:107590000C0500001405000010B51430FFF76AFF59
:1075A00010BD10B51430FFF76BFF10BD10B51430CF
:1075B000FFF752FF10BD0000030070B55E331A786C
:1075C0000469724BE25003005D331A780469704B12
:1075D000E250030061331C7802696E4B012C00D02D
:1075E0009EE005005F352E78A225ED005651020081
:1075F00060321578A1220669D200B5500269D450D4
:107600009623DB00994200D88CE096231B01994217
:1076100000D88AE096235B01994200D888E096233F
:107620009B01994200D885E0E1239B01994200D853
:1076300082E09623DB01994200D880E0E123DB0160
:10764000994200D87DE096231B02994200D87AE047
:10765000E1231B02994200D877E096235B0299420E
:1076600000D874E0E1235B02994200D871E0E12385
:107670009B02994200D86EE0474B994200D86CE0DB
:10768000E123DB02994200D86AE0E12200231203E1
:107690008A425B41414A5B421340802252059B185B
:1076A00001693F4A8B50A02304220169DB00CA50C4
:1076B00000210369FC33D9600369FC33196201239B
:1076C00001690B6001698B60C12104698900625006
:1076D0001F215C3002780A4093406231314AFF3109
:1076E00053500021415600293CDA0F230B40083B40
:1076F0002D4C9B089B001B1903242140A140FC3406
:107700008C40DD69A5432C00C0258D402900214314
:10771000D9611F23017819401E3B8B40136070BD57
:1077200000246CE79E23DB02BAE79D231B03B7E727
:107730001E4BB5E71E4BB3E7EC239B03B0E71D4B95
:10774000AEE71D4BACE71D4BAAE71D4BA8E71D4B51
:10775000A6E71D4BA4E71D4BA2E78023DB049FE7B0
:107760001B4B9DE78C080F4BA400E41803230B4030
:10777000FF21C025DB009940AD0066598E433100E2
:10778000C0269E4033000B436351C2E70C05000046
:10779000140500006C05000090D0030000D0BEFE70
:1077A0002405000000E100E000ED00E000B013005F
:1077B0000050270000A04E0000F0750000509D0012
:1077C00000F0EB0000903A0100E0D70100B0AF03F9
:1077D00000705F07F7B5009308AB1B780025019395
:1077E000FA2304009B0083600E4B4560083303605E
:1077F00014300F001600FFF715FE23005C332761DD
:107800001E70009B084A9B00995823005D33197035
:10781000019B20009B009A5823005E33DD701A7094
:10782000FEBDC04668E30000ECE20000036910B54D
:107830001A00FC32D2680400002A0AD0A322D20027
:1078400099581430C9B2FFF7F8FD00222369FC33C0
:10785000DA6010BD10B50248FFF7E8FF10BDC04662
:10786000C01B00201D2307B50222009302490133EB
:107870000248FFF7AFFF07BD00200040C01B0020FB
:1078800010B5002801D004F0BFFA10BD0849094A1C
:10789000094B10B51B688858FA22190A1B061843B1
:1078A0009200002301F0E8FF4904C00B084310BD1B
:1078B0000010014004050000241C002070B5041EC7
:1078C00009D0FFF7E3FF050000F014F8FFF7DEFF33
:1078D000401BA042F8D370BD0022044B9A60044ABA
:1078E00013680133DBB213607047C046FC100140DF
:1078F000241C00207047704710B500F05FF8FFF7B8
:10790000FAFF0120FFF7DAFFFFF720FBFFF730FB5C
:10791000024B002BFAD000E000BFF7E700000000A8
:10792000F8B54C1EA1410125104B114F8000C358E2
:107930004C4238680F499D40160001F0DBFD0A21DA
:10794000704301F0D7FD2C400300220029000A48B3
:1079500000F016F8FA21094C89004443386801F018
:10796000C9FD0100200001F0C5FDF8BDECE20000FA
:107970002C00002040420F0010050050102700008E
:1079800030B504680C40944206D1013B002BF8D17D
:1079900012E0013B002B0FD004680C409442F8D158
:1079A000002405680D40954204D101349C42F8D171
:1079B000002002E0201C00E0181C30BDC420114B48
:1079C00080001A5810491140C02212020A431A506E
:1079D000C0218022490092025A501A608023A322BB
:1079E0000021DB05D20099500122F9309A60074B43
:1079F000FF301950C1200231800019504030195019
:107A00001A60704700E100E0FF00FFFF0010014036
:107A1000014B18607047C04678000020F7B500237E
:107A20001E285AD8384B8000C258042A5BD007D889
:107A3000022A54D055D80423012A09D000234CE04F
:107A4000062A54D051D31A2A53D002231B2AF5D127
:107A50002E4A116808294ED909294FD00A24022636
:107A6000A02001252A4AC00015502A482A4D07683F
:107A70001C20BF0007402948019700685759009013
:107A800027481B0207401F43C02300989B02034066
:107A9000FF2057515759000207401F43019B1F43C6
:107AA000009B58016023184007433E43565101256F
:107AB0001C4B156058680028FCD000205860A1239A
:107AC0000125DB00D3585560A025ED0050511BB2B5
:107AD000A14202D015D2611ACB401800FEBD082386
:107AE000B6E71023B4E72023B2E74023B0E78023B2
:107AF000AEE70123ACE708240026B1E70C0001261D
:107B0000AEE7091B8B40E8E7ECE2000074000020C0
:107B10000070004030000020040500003400002008
:107B2000FF00FFFFFC700040F0B51E285BD8364B0D
:107B30008000C258354B1E68002E30D1C227344B0E
:107B4000BF00D859334C03250440C0200002204315
:107B5000D851C02480206400800018512E4F186036
:107B60002E4B803CD859FF3CA043D8510437D859FC
:107B7000A8432043D8510837D8590C35A843844628
:107B8000072065462843D851A820C0001E50C120B8
:107B90008026800076021E501C601C4B1C60142541
:107BA00000202B001E4C2E0046433659771C1BD15B
:107BB0004343E250A0230325C132FF329200DB058C
:107BC000D550184B1A68082A14D114234343E318DC
:107BD0009A6812485132FF32920059601150DA68A7
:107BE000C1239B00C250F0BD9642E1D00130032872
:107BF000D9D1F8E7082A02D9083AD140E5E70823A5
:107C00009A1A9140E1E7C046ECE20000281C0020EF
:107C100000E100E0FF00FFFF0405000000900040CD
:107C200038000020780000202149F0B54A6C214836
:107C3000002A14D0A025A12600230124ED05F6007A
:107C4000C258571C06D0C7187F68002F02D02700E3
:107C50009740AF5114333C2BF2D100234B64A02347
:107C60000121DB0500260F009C4614234B43C3185B
:107C70001A1F1268104C0E4D920014195219526CB2
:107C8000002A10D01A00143A1268551C09D0103B73
:107C90001B68FF2B05D03B00934065461A00074B3D
:107CA000EA50FC34666401310429DED1F0BDC046DF
:107CB000FC90004038000020009000400C050000BF
:107CC00000B51E2810D80C4A8000835803290BD811
:107CD000A0220800C133FF33D2059B0001F000FC55
:107CE000020905070021D15000BD0C21FBE704214A
:107CF000F9E70321F7E7C046ECE200001E280AD8A6
:107D0000074B8000C25801239340A022D2050029CE
:107D100002D1044953507047A121C900FAE7C04677
:107D2000ECE200000C050000030000201E2B0AD826
:107D3000A021A222C905D2008858034A9B009B5863
:107D4000D840012318407047ECE20000F7B5060068
:107D50000D000C008B180193019B671B9C4207D000
:107D6000336821781B683000984701340028F3D12C
:107D70003800FEBDF0B5C64600B5CB0F9846404A68
:107D80004B005B0D9A1882B00D000400132A2FDC03
:107D9000002A49DB3B4F17413E000E40064323D0EB
:107DA0007F08390029400C430AD03749BD438C462F
:107DB00063445C425C418023DB021341E4071D43C2
:107DC0004146CE0031492B008E1922003468756877
:107DD0002000290001F0F6FE009001910098019921
:107DE00022002B0003F086F802B004BC9046F0BDE0
:107DF000332A08DD8023DB009A42F5D102000B0014
:107E000001F0E0FEF0E7224A944601226344524228
:107E1000DA400242E8D052080242D1D09443802294
:107E2000D2051A411443CBE74B005B080343DBD078
:107E30000B031B0B1C436342234380244D0C240380
:107E40001B0B23406D042B4319004346DA000F4BF4
:107E50009B181C685D6802000B002000290001F0DF
:107E6000B1FE009001910098019922002B0003F0CF
:107E700041F842464B005B08D60733431900B3E78D
:107E800001FCFFFFFFFF0F00EEFBFFFF98E3000088
:107E9000EDFBFFFFF8B5274A4B005B0D9A180C006D
:107EA0000700132A10DC002A36DB234B13410B4258
:107EB0003AD0802424031441002064189C43060017
:107EC000250030002900F8BD332A0EDD802306008E
:107ED000DB000D009A42F4D102000B0038002100B3
:107EE00001F070FE06000D00EBE7144D0600AC46F5
:107EF000012563446D42DD40AC4663460D000342FC
:107F0000DFD033239A1A323B93401818874200D9A6
:107F10004C1C63469843D2E7C90FCC070020531C82
:107F2000CDD1074B1C43CAE706000D000028C0D185
:107F3000C7E7C04601FCFFFFFFFF0F00EDFBFFFF9F
:107F40000000F03F30B5214A4B0087B05B089342F8
:107F50001EDD1F4A934205DD02000B0002F0CAFF3E
:107F600007B030BD02AA00F095F803231840049A28
:107F7000059B012813D002281DD0002814D0029898
:107F8000039900F06FFB80231B069C466144E7E7E2
:107F9000002300220093002301F0DEF8E0E70298BE
:107FA000039900F05FFBDBE701240298039900943A
:107FB00001F0D2F8D4E7012402980399009401F06B
:107FC000CBF880231B069C466144C9E7FB21E93FAF
:107FD000FFFFEF7FF0B54746CE4680B58DB0040079
:107FE0000D0000F067FA294B06001B780F005BB20A
:107FF0009846013310D022002B002000290003F006
:10800000C1FA8146002807D1002200232000290060
:1080100001F00AFC002806D1300039000DB00CBC7C
:1080200090469946F0BD01230293194B069407959B
:1080300003934B460A93434604940595002B15D0B1
:10804000002300221900100002F0D8F843460890DF
:108050000991022B0ED103F0AFFB212303600A9B91
:108060000193002B0CD1089E099FD5E70023002423
:108070000893099402A801F0C1F90028EFD1EAE7BA
:1080800003F09AFB0A9B01930360ECE77C0000205D
:10809000A8E30000F0B54E464546DE465746E0B53B
:1080A000E14B4C008FB09046894664089C4200DC4E
:1080B00087E0DE4B9C4222DCDD4A002900DC92E0B6
:1080C000DC4B02F017FFDB4B06000F009C4200D197
:1080D0007EE1D94AD94B02F00DFF02000B00414668
:1080E00030000A604B60390002F004FFD34BD24AE3
:1080F00002F000FF434601259860D9606BE0D04B49
:108100009C4200DC8FE0CF4B9C4200DD55E1CE4A23
:10811000231592469A4451460905631A19001D0019
:10812000040003F04BFA03F07FFA02000B0020007A
:1081300029000892099302F0DDFE0022C34B02F0F1
:1081400067FC0F00060003F039FA03F06DFA040033
:108150000D0002000B00300039000A940B9502F06C
:10816000C9FE0022B94B02F053FC002200230C9000
:108170000D9101F053FB002800D192E10023002271
:108180002000290001F04AFB434243410133B04A39
:1081900041460192022208A80092524600F07CFB60
:1081A0004B460500002B16DA802243461206944601
:1081B00042465B68454263445360D3686344D3607E
:1081C00009E00B00020041460A604B6000220023D8
:1081D00000258A60CB6028000FB03CBC90469946D1
:1081E000A246AB46F0BD934B01F0ECFC914B060070
:1081F0000F009C4200D13DE18F4A904B01F0E2FC20
:1082000002000B00414630000A604B60390002F06A
:1082100071FE894A894B01F0D5FC012543466D4228
:108220009860D960D7E701F049F88A4A8A4B06007E
:108230000F0002F0EDFB0022884B01F0C3FC03F0BD
:10824000BDF9050003F0F0F9794A7A4B04900591E5
:1082500002F0DEFB02000B003000390002F04AFEA3
:10826000754A06000F0004980599744B02F0D0FB84
:10827000029003911F2D00DCC7E0029A039B30009F
:10828000390002F037FE83468A4653465B002415C8
:108290005B0DE31A102B6CDD04980599D322674B14
:1082A000520502F0B5FB02000B00300039000292CB
:1082B000039302F01FFE0A000100130006910792CB
:1082C00002003900300002F015FE029A039B02F012
:1082D00011FE06000F0004980599614A614B02F0F7
:1082E00097FB32003B0002F005FE069E079F0B0045
:1082F0000200390030000292039302F0FBFD4B00B4
:108300005B0D83468A46E41A312C32DD04980599C8
:10831000B822544B920502F07BFB03000C000200D4
:10832000029303940B000698079902F0E3FD020004
:108330000B0006000F000698079902F0DBFD029A79
:10834000039B02F0D7FD484A0290039104980599D7
:10835000464B02F05DFB029A039B02F0CBFD02004C
:108360000B00300039000292039302F0C3FD8346F4
:108370008A465A465346414630000A604B603900EF
:1083800002F0B8FD029A039B02F0B4FD44460B00D4
:108390000200A260E3604B46002B00DB1BE75B465C
:1083A000236080231B065344636080231B069C4686
:1083B0006144A060E1606D420DE70B00020002F035
:1083C00099FD434600259860D9601860596002E71E
:1083D000D3221A4B520502F08DFD214A214B0D008C
:1083E000040002F087FD02000B00414620000A60F5
:1083F0004B60290002F07EFD1A4B194A02F07AFD0B
:10840000434601259860D960E5E602000B00300084
:10841000390002F06FFD6B1E154A9B009B58834686
:108420008A46A342A5D130E7FB21E93F7BD9024030
:1084300000004054FB21F93F3163621A61B4D03D22
:10844000FB213941FFFFEF7FEAFBFFFF0000704196
:1084500030E4000083C8C96D305FE43F0000E03FB6
:108460007370032E8A19A33BC14920259A837B3957
:10847000B0E30000D3220C4B520501F0A3FB0B4AE2
:108480000B4B04000D0001F09DFB02000B00414668
:1084900020000A604B60290002F02CFD034A044BC7
:1084A000B9E6032373E6C04661B4D03D7370032E72
:1084B0008A19A33BF8B54746CE46674B80B50A00FC
:1084C0000F00190005003940994200D19BE00400DB
:1084D0000100002F69DD3F1500D1B4E05F4B1203AE
:1084E0009C468023120B5B0313435B00CA0F674457
:1084F0009B184A00F80703D5D20F5B009B188A002F
:1085000079108C46002180201624894680030D189E
:108510009D4202DC29185B1B8144D50F5B00013CA6
:108520005B1952004008002CF1D1002080468020C9
:1085300020250027000609E08B425CD0D40F5B00A9
:10854000013DE31852004008002D16D0C4198B429B
:10855000F2DD27180E00002C49DB5B1AA24289418C
:1085600049425B1A121BD40F5B00013D804431006D
:10857000E31852004008002DE8D113434ED1434682
:108580005B0837494A468846494652104244C90763
:1085900002D5802109060B4361460F05BD1818005E
:1085A00029000CBC90469946F8BD7B005B0803434C
:1085B0003900002BF5D0002F3CD1E30A153A6405B1
:1085C000002BFAD08020400303423FD1002700E077
:1085D0000F005B00791C0342FAD0250020208D405B
:1085E000401A2900D71B2200C2401A4376E7FE43F7
:1085F000F60F8E19B1E79442A0D82718002CF6DBAD
:108600001E000023AEE702003B002800390002F004
:10861000FFF92A003B0001F0D5FAC2E743460133D7
:1086200003D0434601335B08ABE7012398460023A0
:10863000C144A6E73B00020002F05CFC02000B0014
:1086400001F0DCFDADE713000022BBE701272100AC
:1086500020207F42C6E7C0460000F07F01FCFFFFFC
:108660000000E03FF0B54746CE4680B587B00092A7
:108670000193754B4F00814688467F089F4263DC1B
:1086800002F09CFF002800D1D4E04A464346484609
:10869000414602F0BDF904000D006C4A6C4B02F03B
:1086A000B7F96C4A6C4B01F08DFA22002B0002F0F6
:1086B000AFF96A4A6A4B02F01DFC22002B0002F05F
:1086C000A7F9684A684B01F07DFA22002B0002F0FE
:1086D0009FF9664A664B02F00DFC22002B0002F067
:1086E00097F9644A644B01F06DFA22002B0002F006
:1086F0008FF9029003910022604B2000290002F0C4
:1087000087F9029A039B06000F002000290002F05F
:108710007FF9009A019B04000D004846414602F093
:1087200077F902000B002000290002F0E3FB0200B1
:108730000B003000390002F0DDFB02000B000020CE
:108740004F4902F0D7FB70E002000B0002F060F925
:1087500004000D003D4A3E4B02F05AF93D4A3E4BA3
:1087600001F030FA22002B0002F052F93B4A3C4B58
:1087700002F0C0FB22002B0002F04AF9394A3A4BC2
:1087800001F020FA22002B0002F042F9374A384B60
:1087900002F0B0FB22002B0002F03AF9354A364BCA
:1087A00001F010FA2B00220002F032F9354B029052
:1087B00003919F429FDD344B00229F423DDC3349B1
:1087C00000207B182E4916001F0002F093FB049036
:1087D00005910022294B2000290002F019F93200EE
:1087E0003B0002F087FB029A039B06000F0020006B
:1087F000290002F00DF9009A019B04000D00484683
:10880000414602F005F902000B002000290002F0A9
:1088100071FB02000B003000390002F06BFB02001C
:108820000B000498059902F065FB07B00CBC90465C
:108830009946F0BD00201249F7E7154B0026049237
:108840000593144FC5E7C046FFFF3F3ED43888BEAE
:10885000E9FAA8BDC4B1B4BD9EEE213EAD529C80E4
:108860004F7E923E9015CB19A001FA3E7751C1166A
:108870006CC1563F4C5555555555A53F0000E03F3E
:108880000000F03F3233D33F0000E93F0000E0FF3B
:108890000000E73F0000D23FF0B5DE464E464546B9
:1088A0005746E0B5DC4CA5440D9114001900A49A7C
:1088B0000993DA4B9200D6584D1E03901821E01E02
:1088C0000696029500F0A0FEC3430100DB17194095
:1088D0004B1C9A009B1ADB001B190B9105934C1B38
:1088E000771918D4A59BA5009C463F1922AE654474
:1088F000013707E0286802F097FE013403C604350B
:10890000BC4208D0002CF5DA00200021013403C657
:108910000435BC42F6D1069B002B01DA00F0FDFBCA
:10892000069B03990133DB009A46099BDA009446C3
:1089300000920022914672AA0492B94A6144934679
:1089400088469AAB63449B44029B002B00DABCE14F
:108950005D4600260027039C4D442A686B6803CCC3
:1089600002F056F802000B003000390001F02AF93D
:10897000083D06000F004445EFD1049B4B441E60A8
:108980005F6008239C46E144D145DDD10EA8042157
:108990008446494261448C46069A93009C44614651
:1089A00084460A910399083B63448C460C93009BD0
:1089B000009263449B46009A0498D10003008C46C1
:1089C000634408911E685F68002A33DD954980463C
:1089D0008C466244D300984470AB9A460EAB9946DD
:1089E0000022914B3000390002F012F802F0E6FD4F
:1089F00002F01AFE00228D4B04000D0002F008F870
:108A000002000B003000390002F074FA02F0D6FDCB
:108A10004B4601C39946434620001A685B6829000B
:108A200001F0D0F808235B429C46E04406000F00AA
:108A3000D045D5D1059B30001A003900984600F08A
:108A4000DFFCFF2300229B0504000D0001F0E0FF86
:108A500000F038FC0022764B01F0DAFF02000B0038
:108A60002000290002F046FA0D00040002F0A6FDE5
:108A7000814602F0D9FD02000B002000290002F01F
:108A800039FA060040460F00002800DCEEE0009BAB
:108A900018215A1E92000EAB9B58091A1D000D4159
:108AA000A9448D405D1B0EAB9D5017231B1A1D4121
:108AB000002D2DDD01239C46009BE144002B00DCB2
:108AC0001CE20E9C0123002C00D0B5E0009A012A84
:108AD00009D099000EAA54580133002C00D0ACE004
:108AE000009A9A42F5D1059B002B0EDD012B00D197
:108AF000A8E1022B09D1009B0EA95A1E92000EABD1
:108B00009B5807939B029B0A8B50022D00D1C1E01A
:108B1000002300223000390000F080FE009B002876
:108B200000D194E2069A591E8A4210DC414A0A9802
:108B300094460EAA6344944600229B0063441C683A
:108B4000043B22438342FAD1002A00D0C0E0069BB6
:108B50000EAA013B9B00D358002B00D0B3E00122AA
:108B60000C9B043B596801320029FAD0009B9C46BB
:108B70006244110007921A0001338B4246DC0B98C5
:108B800063468046A59C4344A046099C9B00A146A1
:108B90004A449844D30022AA9146049A99449446A0
:108BA000089BA59A63448446614494469A468B0088
:108BB000634400934346586802F036FD4B46186004
:108BC0005960029B002B24DB4D46039C00260027A6
:108BD00001E0286869680CCC01F01AFF02000B0064
:108BE0003000390000F0EEFF083D06000F005C4544
:108BF000EFD153469E60DF6004239C460433E0447B
:108C00009C46009BE144E2449845D3D1079B0093E6
:108C1000D1E600260027ECE794FDFFFF78E5000091
:108C200018FEFFFFFFFFFF1F0000703E00007041B5
:108C300000002040FFFFFF3F002180225204141B50
:108C40000EAA5450009999420EDD0EA884469B004E
:108C50000EAA8900D25861446344CF4800E01A68E4
:108C6000821A04C38B42FAD101243CE7059B002BF6
:108C700006D1009B0EAA013B9B00D558ED1517E7C6
:108C80000022C64B300000F0EDFD002800D024E1AA
:108C900000253DE732003B000020C14902F02AF9DF
:108CA00006000F00002C00D132E7059A0020BC49D5
:108CB00000F0A6FB02000B003000390002F01AF9A8
:108CC00006000F0024E7012250E70026002754E6A3
:108CD0004B46059A079388468B000EA9CB58183A45
:108CE00008950592002B0DD18C464146AD4B43446F
:108CF0009B006344043B58680139183A0028F9D0B6
:108D000088460592059A0020A54900F079FB434664
:108D100004000D00002B00DA05E29E000EAB9C461D
:108D20004346DB0066449C46059370AB9946049F1E
:108D300067440097306802F077FC22002B0001F0B6
:108D400067FE002238607960974B2000290001F00F
:108D50005FFE083F04000D00043EB945EAD14AAB6E
:108D600003939B4600239A46069B424699464346F8
:108D70000132029204934B46002B00DAAAE08020D5
:108D80008A4B009D9846C00589490026002700248B
:108D900008E008239C460835E044544511DC43466E
:108DA000186859682A686B6801F032FE02000B00EF
:108DB0003000390000F006FF013406000F00A14525
:108DC000E7DA5B46C0C39B4601239C46009BE24416
:108DD000083B0093029B9A45CDD1049B9846A49BE7
:108DE000022B00DD8EE0002B37DC1FD1059B002716
:108DF0001D00039B00249C461E006544083E2A6813
:108E00006B683800210000F0DDFE083D07000C0013
:108E1000AE42F4D1089B002B03D080231B069C4656
:108E200064443A0023000D990A604B600720079BB9
:108E300018409B239B009D443CBC90469946A2460B
:108E4000AB46F0BD009B0EA95A1E92000EAB9B587C
:108E500007935B025B0A8B5057E64346002B00DA10
:108E600070E100200021DB004AAAD61848AF326822
:108E70007368083E00F0A6FEB742F8D1089B002BAD
:108E800000D025E10B0002004A984B990D9C22600E
:108E9000636002F02FF8434607000C00002B13DD3F
:108EA00001254CAEB14638002E0021004C4601365B
:108EB0000CCC00F087FEA146B045F7DA089B07000E
:108EC0000C00002B00D015E13A0023000D998A60B8
:108ED000CB60ABE70026002773E701239C46009B8D
:108EE000E1440225002B00DDEBE532003B000020D1
:108EF0002B4901F0FFFF06000F0009E60024F2E510
:108F00004AAB0393A49B032B00D08FE74346002B6F
:108F100000DC14E1039ADB009B46130091465B449E
:108F20001E685F68234B43440293DB00994448ABBF
:108F30009A464B465C681B681800210032003B00D3
:108F40000090019100F03EFE04000D0002000B00B5
:108F50000098019901F0CEFF3B00320000F032FE94
:108F60004B469860D9601C605D6008235B429C465C
:108F7000E14426002F00CA45DBD14346012B00DC2B
:108F8000E3E0039A13005B441E685F68029BDB000A
:108F900099464A44904610E0FFFFFF000000E03F82
:108FA0000000F03FFFFFFF3F0000703E38E500008B
:108FB000FB21F93FFFFFFF1F984643465C681B6893
:108FC0001800210032003B000090019100F0FAFDF2
:108FD00004000D0002000B000098019901F08AFFC7
:108FE00032003B0000F0EEFD4346039A9860D960E2
:108FF0001C605D60083B26002F009A42DCD14D4684
:109000009446002600244746083565442A686B6864
:109010003000210000F0D6FD083D06000C00AF42F4
:10902000F4D1039B4A9F5D689968D868089B002B20
:1090300065D08022120694460D9B654460446444CA
:109040001F605D609960D8601E615C61EEE69A46C3
:109050004B460793059B30005A423900089500F0B3
:10906000CFF900223A4B06000F0000F0FBFB00286E
:1090700024D0384B00223000390001F0C9FC02F046
:109080009DFA52460400950002F0CEFA0022304BC1
:1090900001F0BEFC02000B003000390001F02AFF95
:1090A00002F08CFA0EAA50510122059B524418334B
:1090B0009046059393000EAAD45023E65346300001
:1090C00039009C0002F07AFA0EAB1851D04619E62E
:1090D00080230D9A1B06CB18106053600B00020012
:1090E0004A984B9901F006FF434607000C00002BFD
:1090F00000DDD5E680231B069C466444E4E62B0095
:109100003A000D9D2A606B600A000300AA60EB60C4
:10911000320023002A616B6188E6099BDB00009323
:1091200072AB049332E4A49B022B00DDE8E6002B33
:1091300000DD92E600D079E6002700246AE60026EA
:1091400000246EE70020002198E60026340068E73E
:10915000000070410000703EF0B5CE46474680B535
:1091600087B000920193474A4B00814688465B08CE
:10917000934207DC4146484602F020FA4146031E6E
:10918000484666D04A4643464846414601F040FCC0
:1091900004000D0002000B004846414601F038FC77
:1091A000394A3A4B06000F002000290001F030FC3C
:1091B000374A384B01F09EFE22002B0001F028FCBC
:1091C000354A364B00F0FEFC22002B0001F020FC5B
:1091D000334A344B01F08EFE22002B0001F018FCC4
:1091E000314B324A00F0EEFC0E9B02900391002BB3
:1091F00034D00098019900222D4B01F009FC029A0D
:10920000039B049005913000390001F001FC02003D
:109210000B000498059901F06DFE22002B0001F06F
:10922000F7FB009A019B01F065FE224A04000D0045
:10923000214B3000390001F0EBFB02000B00200055
:10924000290000F0BFFC02000B004846414601F037
:1092500051FE07B00CBC90469946F0BD02000B00D1
:109260002000290001F0D4FB124A134B01F042FE0A
:1092700032003B0001F0CCFB4A46434600F0A2FC22
:10928000E7E7C046FFFF3F3E7CD5CF5A3AD9E53DE0
:10929000EB9C2B8AE6E55A3E7DFEB157E31DC73EA7
:1092A000D561C119A0012A3F1111813FA6F8101103
:1092B0000000E03F495555555555C53F49004B08FD
:1092C00019007047474AF0B54F4691464B005B0D79
:1092D00099444646D6464A46C0B505000C000E00E5
:1092E00088460700132A27DC002A4BDB3E4B13413C
:1092F0009A460B0052461340034318D03B4A3C4B5E
:109300002800210000F05EFC0022002300F0A0FAFB
:10931000002847D0002C04DA80234A465B0313411F
:1093200098444646534600279E43380031001CBCF3
:1093300090469946A246F0BD332A08DD8023DB0023
:109340009945F4D102000B0000F03CFCEFE7294AFC
:109350009446012263445242DA4092460242E6D0E9
:10936000224A234B2800210000F02CFC002200237D
:1093700000F06EFA002815D0002C1EDB534646463E
:109380009F430FE0194A1A4B2800210000F01AFCF5
:109390000022002300F05CFA002803D0002C04DB3C
:1093A0000027002638003100C1E764006408254327
:1093B0000027002DF6D0104EF4E74B46142B0BD0AF
:1093C0003422D21A012393405D19BD4208D20123F1
:1093D0009C462F00E044D1E7133B9C46E044CDE798
:1093E0002F00CBE701FCFFFFFFFF0F009C750088FB
:1093F0003CE4377EEDFBFFFF0000F0BF002070472C
:109400004B0070B55B0D14000A00002B1AD14B0005
:109410005B08034315D0234B002201F0F9FA224BDD
:109420009C422DDB0A004B005B0D363B1F4DE318C1
:10943000AB422ADC002B0DDD1D4C1B0522401A43DC
:10944000110070BD1B4DAB42F0D102000B0000F0CB
:10945000B9FBF6E71D00353519DA174B02009C42BF
:1094600009DD0B001548164900F032F8134A144B79
:1094700001F0CEFAE5E70B001248134900F028F896
:10948000104A114B01F0C4FADBE70200E9E7084C8F
:10949000363322401B051343190000220B4B01F009
:1094A000B7FACEE700005043B03CFFFFFE070000D4
:1094B000FFFF0F80FF07000050C300009C7500886D
:1094C0003CE4377E59F3F8C21F6EA5010000903CC2
:1094D00030B54A00DB0FDB0752081A43110030BDDC
:1094E00002B4714649084900095C49008E4402BC37
:1094F0007047C046002243088B4274D303098B4255
:109500005FD3030A8B4244D3030B8B4228D3030C53
:109510008B420DD3FF22090212BA030C8B4202D3F5
:109520001212090265D0030B8B4219D300E0090A1D
:10953000C30B8B4201D3CB03C01A5241830B8B4226
:1095400001D38B03C01A5241430B8B4201D34B030F
:10955000C01A5241030B8B4201D30B03C01A524174
:10956000C30A8B4201D3CB02C01A5241830A8B42F9
:1095700001D38B02C01A5241430A8B4201D34B02E2
:10958000C01A5241030A8B4201D30B02C01A524146
:10959000CDD2C3098B4201D3CB01C01A52418309FA
:1095A0008B4201D38B01C01A524143098B4201D334
:1095B0004B01C01A524103098B4201D30B01C01A5F
:1095C0005241C3088B4201D3CB00C01A52418308D9
:1095D0008B4201D38B00C01A524143088B4201D306
:1095E0004B00C01A5241411A00D201465241104666
:1095F0007047FFE701B5002000F0F0F802BDC0465B
:109600000029F7D076E7704703460B437FD400224A
:1096100043088B4274D303098B425FD3030A8B4206
:1096200044D3030B8B4228D3030C8B420DD3FF2270
:10963000090212BA030C8B4202D31212090265D03E
:10964000030B8B4219D300E0090AC30B8B4201D3F1
:10965000CB03C01A5241830B8B4201D38B03C01A38
:109660005241430B8B4201D34B03C01A5241030BAF
:109670008B4201D30B03C01A5241C30A8B4201D360
:10968000CB02C01A5241830A8B4201D38B02C01A0B
:109690005241430A8B4201D34B02C01A5241030A82
:1096A0008B4201D30B02C01A5241CDD2C3098B4267
:1096B00001D3CB01C01A524183098B4201D38B01E4
:1096C000C01A524143098B4201D34B01C01A524187
:1096D00003098B4201D30B01C01A5241C3088B42CC
:1096E00001D3CB00C01A524183088B4201D38B00B7
:1096F000C01A524143088B4201D34B00C01A524159
:10970000411A00D201465241104670475DE0CA0F2F
:1097100000D04942031000D34042534000229C46EF
:1097200003098B422DD3030A8B4212D3FC228901F9
:1097300012BA030A8B420CD3890192118B4208D3CF
:10974000890192118B4204D389013AD0921100E031
:109750008909C3098B4201D3CB01C01A5241830945
:109760008B4201D38B01C01A524143098B4201D372
:109770004B01C01A524103098B4201D30B01C01A9D
:109780005241C3088B4201D3CB00C01A5241830817
:109790008B4201D38B00C01A5241D9D243088B426D
:1097A00001D34B00C01A5241411A00D20146634610
:1097B00052415B10104601D34042002B00D5494274
:1097C000704763465B1000D3404201B5002000F0B3
:1097D00005F802BD0029F8D016E770477047C0466B
:1097E000D0400B1C1141203A03D49C46134118432E
:1097F00063465242934018437047C0468446101C4B
:1098000062468C46191C634600E0C0461FB501F055
:1098100097F8002801D40021C8421FBD10B500F000
:10982000EFFF4042013010BD10B501F089F800286B
:1098300001DB002010BD012010BDC04610B501F0B5
:109840007FF8002801DD002010BD012010BDC046BA
:1098500010B501F011F8002801DC002010BD012036
:1098600010BDC04610B501F007F8002801DA00204D
:1098700010BD012010BDC046F0B5CE4647461504C8
:109880002D0C2E0080B50704140C3F0C9946030CD8
:109890007E435D43674363437F19340CE4199C4660
:1098A000A54203D980235B029846C4444B464343F8
:1098B0005143250C36046544360C2404A4195B1965
:1098C000591820000CBC90469946F0BDF0B54E46A4
:1098D00057464546DE46E0B543025B0A450083B085
:1098E0000F1C99462D0EC60F002D57D0FF2D24D0EA
:1098F0008020DB00C0041843002381469A469B4623
:109900007F3D7C027A00FB0F640A120E984623D03A
:10991000FF2A4BD0E30080240020E4047F3A1C435C
:10992000AD186B1C47460193534677403A000F2B06
:1099300048D87D499B00CB589F46002B00D085E03E
:1099400008339A46063B9B467C027A00FB0FFF25B4
:10995000640A120E9846DBD1002C00D090E05246EB
:1099600001231A4392460120DBE74C465846170074
:10997000022824D0032800D1CFE0002200230128B0
:109980004DD15802D205400AFF071043384303B0B7
:109990003CBC90469946A246AB46F0BD002B5BD13D
:1099A00004239A46033B00259B46AAE7FF35002C7B
:1099B00060D1524602231A4392460220B1E7FF22A9
:1099C0000023DEE74B461B0C9C464B462604360C18
:1099D000180461463300220C6446000C43434E4396
:1099E0005043544380191A0C1218964203D980210F
:1099F00049028C4664441B041B0C1004C0188301EC
:109A00005E1EB341800E1843130C1B199B010343C8
:109A10001C00230179D5012362081C401443019ADC
:109A20007F32002A4DDD630704D00F232340042B2F
:109A300000D00434230103D53C4B019A1C408032F2
:109A4000FE2ABCDCA3015B0AD2B29AE70C239A4639
:109A5000093BFF259B4654E7180001F071FE4A467A
:109A6000431F76259A4000236D4291462D1A9A464F
:109A70009B4646E7524603231A439246032050E78B
:109A8000200001F05DFE431F2D1A9C40763D002012
:109A900047E780230027DB03FF2272E7424666E7A1
:109AA0004C463200584662E780234A46DB031A429E
:109AB00022D01C4220D123435B025B0A4746FF228F
:109AC0005FE701239A1A1B2A21DC23000199D34066
:109AD0009E318C401A0023005C1EA34113435A0799
:109AE00004D00F221A40042A00D004335A0111D4A2
:109AF0009B015B0A002244E780234A46DB031343B1
:109B00005B025B0A3700FF223BE7019587E70022F3
:109B1000002336E70122002333E78023DB032343BE
:109B20005B025B0AFF222CE788E50000FFFFFFF7DE
:109B300070B500283DD0C317C5185D40C40F28007C
:109B400001F0FEFD9E22121A962A07DCD2B20828E6
:109B500033DD083885406802400A23E0992A0BDD8E
:109B6000052329001B1AD94003001B339D402B00FD
:109B70005D1EAB4119430D00052801DD431F9D40CB
:109B80002B000F490B406E0709D00F263540042DDE
:109B900005D004335D0102D59F220B40121A9B01B0
:109BA000580AD2B24002D205400AE40710432043CB
:109BB00070BD002400220020F4E76802400AF1E7AB
:109BC000FFFFFFFBF0B54F464646D6460C000903A3
:109BD000C0B5490A470F5E0039431F03DB0F9C469F
:109BE00065007B0A570F1F436D0DE40F760DA146EC
:109BF000C000B846D200AB1B64457BD0002B5FDDB4
:109C0000002E00D0A4E03E00164300D112E15E1EFB
:109C1000002E00D09EE1871A4346B84280410125BC
:109C2000C91A4042091A0B0200D431E149024E0A16
:109C3000002E00D16EE1300001F082FD0300083BF0
:109C40001F2B00DD61E120223900D21A9E40D14055
:109C50009F400E439D4200DD51E15D1B6B1C1F2B9D
:109C600000DD7CE12021C91A3D0030008F40884092
:109C7000DD40791E8F41310007222843D94000255D
:109C800007433A40002A09D00F233B40042B05D05C
:109C90003B1DBB42BF417F42C9191F000B0200D4CC
:109CA00026E26A1CC64B55056D0D9A4200D106E1AD
:109CB000C44AFF080A40530752023B43120B8EE08E
:109CC000002B00D0B8E06B1C5B055B0D012B00DCAA
:109CD00030E1871A4346B842B641CB1A76429E1B02
:109CE000330200D54CE13B003343A1D100220024D4
:109CF000002570E0002B00DCE5E0002E00D183E0C1
:109D0000AF4EB54260D0802636043743B846382B74
:109D100000DC3EE1434613431F007A1E97413F1883
:109D200087428041404209180B0200D4B0E0A44BA6
:109D300001359D4200D1C3E0A24A7B080A400121BF
:109D40000F401F435108D30707221F433A4099E7AA
:109D50009B4EB54238D0802636043743B846382B60
:109D600000DDDCE01F2B00DC30E11E004746203E1A
:109D7000F740BC46202B04D04026F31A46469E40AE
:109D80003243170063467A1E97411F43CCE0002BF5
:109D900000D104E24346134300D159E14B07C00808
:109DA00018438023C9081B03194208D04546ED0813
:109DB0001D4204D14346D008590708432900420FE9
:109DC000C9007F4D1143C0004B07CA087C49C00839
:109DD00003438D4268D012036D05120B6D0D0021F7
:109DE00012031800130B0A0D12051A43764B2D05AA
:109DF00013402B435B00E4075B08234319001CBCA2
:109E000090469946A246F0BD3E00164312D05E1E13
:109E1000002E00D000E18718874280414144404233
:109E2000091801250B0233D5022585E76446330066
:109E3000414610001D00C7E7002D00D0DAE00C00FD
:109E40000443F3D05C1C00D19FE15D4CA64200D1DD
:109E50002FE1DB43382B00DD66E11F2B00DD83E1C2
:109E600020240500E41A0F00DD40D940A0404346FD
:109E7000A7405B1A441EA04198462F433843171A47
:109E8000BA42924143465242991A64463500CAE6A4
:109E900007223A40002A00D0F6E64B07CA08484994
:109EA000FF083B438D4296D11900114300D19EE13A
:109EB000802109030A431203120B414D8FE715005D
:109EC000002200238BE7002B00D0C7E06B1C5F054E
:109ED0007F0D012F00DCF1E0394DAB4200D1B9E03C
:109EE00085180A0085428941424449425118072297
:109EF000CF076D082F4349083A401D00C2E60722EC
:109F00003049ED1A31403A40BCE63E0028388640E0
:109F100000279FE6380001F013FC20308EE6434610
:109F200013431F007A1E9741C71BB842804140422D
:109F3000091A78E60E003B0006431343002D61D159
:109F4000002E00D0F4E0002B00D11BE16446390064
:109F5000100039E71A4FBB427AD03300FFE63000D9
:109F60001F3DE840202B03D04021CB1A9E403743B1
:109F70007B1E9F41072207433A400021002589E7C5
:109F8000171A4346BA42B641591A76428E1B6446A6
:109F90004EE61F2B00DDADE020264746F61AB740FF
:109FA000B9461700B246DF404E463E43370056469C
:109FB000B240561EB24117434246DA408918AEE617
:109FC000FF070000FFFF7FFFFFFF0F8020264746AF
:109FD000F61AB740B9461700B246DF404E463E4338
:109FE00037005646B240561EB24117434246DA4049
:109FF000891A99E77F4CA6425BD0802424045B42F7
:10A00000214327E7002E0CD1002B00D1CBE0644682
:10A0100039001000774DD7E6764FBB4218D0330099
:10A0200075E6002B14D04B07C00818438023C908DD
:10A030001B03194207D0FC081C4204D17907D00841
:10A040000843E14621004C46420FC9001143C000BD
:10A05000684DB9E61D0000220023C0E6002D5BD14B
:10A060000D00054300D1E2E65D1C00D1B0E0614D7A
:10A07000AE421FD0DB43382B71DC1F2B00DD96E096
:10A0800020250F00ED1AAF40B9460700AA46DF4071
:10A090004D463D432F005546A840D940451EA84196
:10A0A00088440743BF1897429241514241443500CA
:10A0B0003AE6644635004146100085E60B0003434E
:10A0C000002D00D063E6002BF5D04346134300D1AA
:10A0D0007AE68718874280410722414440420918A6
:10A0E0003A400B0200D4D5E6434B01351940C9E58F
:10A0F000380069E61E004746203EF740BC46202B4C
:10A1000004D04026F31A46469E4032431700634669
:10A110007A1E97411F4302E6364DAE42CAD08025D3
:10A120002D045B422943A6E70843411E8841A6E669
:10A13000002B00D148E6871A4346B842B641CB1AF5
:10A1400076429E1B33024BD5171A4346BA429241C0
:10A15000591A5242891A072264463A4092E501434D
:10A160000F00791E8F419DE71C000F00203CE74047
:10A17000202B03D04024E31A99400843411E884114
:10A1800038437CE60022002425E6171A4346BA42EB
:10A190009241591A5242891A6446350043E54146B4
:10A1A0001000144D10E680220024120380E61D00EA
:10A1B0000F00203DEF40BC46202B03D04025EB1A7A
:10A1C0009940084307006346781E87411F4369E7AB
:10A1D000871897429B4141445B42C9183500A3E56B
:10A1E0003B003343CED0072231003A4052E60023F1
:10A1F0001A00F4E5FF070000FFFF7FFFF0B55746A8
:10A20000DE464E464546E0B5834607000E0348004D
:10A2100085B092461C00360B400DCD0F002800D1B2
:10A220009DE0954B984239D08023F6001B041E43D5
:10A23000924A7B0F3343994694460300634400934C
:10A2400000230026FF00029323031B0B98466300A4
:10A25000E40F52465B0D019400D1B3E086498B4276
:10A2600000D19EE04246D100802212040A435146AA
:10A27000490F11438B46814952468C4600996344ED
:10A28000CB1A0021D20000932B0063409A460F2E78
:10A2900000D905E17A4BB6009B599F465B46334394
:10A2A000994600D0B8E002230826002700900293C8
:10A2B000CAE7CB463A0002990195019B9A460229CA
:10A2C00027D0032900D180E2012944D06D49009BA9
:10A2D0008C4663441C00002C38DD530700D013E289
:10A2E000D2085B46DB0109D55946674B19408B46BE
:10A2F0008021C9008C46009B63441C00634B9C4238
:10A3000007DC5B4664055F075B0217431B0B620DAE
:10A3100002E000230027584A00211B031C0B0B0DF1
:10A320001B05234314055A4A380013401C43534667
:10A330006400DB0764081C43210005B03CBC904668
:10A340009946A246AB46F0BD0122524201231B1B97
:10A35000382B00DCADE1002200230027DCE75B4660
:10A36000334399465ED0002E00D18AE1300001F0DF
:10A37000E7F903000B3B1C2B00DD7BE11D22D31A08
:10A380005A460100DA4008398E4013005F463343D5
:10A3900099468F403F4B00261B1A009300230293DF
:10A3A00052E7414653460B433B499B468C46009B34
:10A3B000634400935B46002B3BD1022300221E43E3
:10A3C000022161E7434613439B4637D04346002BA7
:10A3D00000D162E1404601F0B3F903000B3B1C2BB6
:10A3E00000DD53E102004146083A914088461D21B4
:10A3F000CB1A5146D9400B0041460B439B4653466E
:10A4000093401A00009B25499C46604403008C46FB
:10A4100063440093002137E70323B14600900C26E4
:10A42000029311E7002300930133042600270293CF
:10A430000AE70323C3461E43032125E701331E43D6
:10A440000022012120E700239A46802300271B03D6
:10A45000094A61E7802349461B03194200D1E2E023
:10A460005946194200D0DEE00B431B0317001B0BBB
:10A47000A246014A50E7C046FF07000001FCFFFF6B
:10A48000C8E50000FF030000FFFFFFFEFE0700001D
:10A49000FFFF0F800DFCFFFF01F8FFFFF30300003B
:10A4A000D94500D9CBE000D1C6E03C0048460027A2
:10A4B000009B013B00935B46160E1B021E431302DA
:10A4C000984633041B0C9946310C0191FFF798F81C
:10A4D0004A4642430B04210C050019438A4207D91E
:10A4E0008919013D8E4203D88A4201D9851E8919F6
:10A4F000881A0199FFF784F809048C464A4621041A
:10A5000064464243090C030021438A4204D9891955
:10A51000013B8E4200D8F1E02D041D43AB4643467B
:10A52000891A4246280C12041D0C5B46140C2200AA
:10A530001B041B0C5A4303946B434443029568432A
:10A540001B19150CEB189C4203D980246402A44605
:10A5500060441C0C15041B042D0C20185D1981424D
:10A5600077D373D00C1AA24A7D1BAF42BF419446E9
:10A57000009B7F426344E01B1C00864200D1DBE06D
:10A580000199FFF73DF84A4642430B04290C0700A6
:10A5900019438A4207D98919013F8E4203D88A425A
:10A5A00001D9871E8919881A0199FFF729F809042A
:10A5B0004A46894629044D464243090C0300294373
:10A5C0008A4207D98919013B8E4203D88A4201D9B0
:10A5D000831E89193F04891A3A00039F1A433800E1
:10A5E00013041B0C584381460298150C6F434343D8
:10A5F00045434846000C8446DB1963449F4203D917
:10A60000802040028446654448461F0C00041B0419
:10A61000000C7D191818A94200D284E000D17FE017
:10A6200001231A4357E680234A461B0313431B03A7
:10A630001B0BAA466F4A6FE6BA4200D935E74B4674
:10A64000DC0758087B081C43FF0734E70024AF42AF
:10A6500089D247444745A4415B466442A419641823
:10A66000013BA6421ED2A0426DD800D1B6E0241A0A
:10A670009B4678E703005A46283B9A4000279146BC
:10A6800088E6584601F05CF8203072E60300524636
:10A69000283B9A4093460022B4E6504601F050F819
:10A6A00020309AE6A642E2D1B845DCD9341A9B465E
:10A6B00059E71F2B65DC504C0099A4465C46614469
:10A6C00008008C4011008240D940501E82410C434A
:10A6D00014435A46DA401300620709D00F22224081
:10A6E000042A05D02200141D9442894149425B1876
:10A6F0001A0262D50122002300270DE68A4200D803
:10A700000AE7831E891907E70F231340042B00D1A2
:10A71000E6E5171D9742924153429B44FA08E0E553
:10A72000002800D1D7E57118531EB14227D3A942A2
:10A7300015D358D01A0073E7002B00DC04E6012380
:10A7400000229B44CDE502234744474589415B42B3
:10A750009C46494289190C19E344241A03E74346ED
:10A760005F0047459B41B8465B429E19023A8919F2
:10A77000A94200D054E7404500D051E7ABE51A00AC
:10A78000F6E71F215F4649420C1BE740202B07D00C
:10A790001A49009B8C46634418005B4683401A4369
:10A7A000501E82413A4307270023174009D00F214A
:10A7B000002311401400042995D122005F075B0299
:10A7C0001B0BD20817430022A6E5802359461B0322
:10A7D0000B431B0317001B0B064A9DE5BD42B2D875
:10A7E0009B460024BFE68045B9D31A00C3E7C046A4
:10A7F000FF030000FF0700001E0400003E040000ED
:10A80000F0B54F464646D6468446C0B58046194EFA
:10A8100018030F034D00000B5C0082463F0B6D0DCB
:10A82000C90F9146640DDB0F0120B5420AD0B44236
:10A8300003D0A54201D157450CD01CBC9046994687
:10A84000A246F0BD66463E43F7D1AC42F5D1544630
:10A850001443F2D10120C845EFD1994207D0002D11
:10A86000EBD163461F433800471EB841E5E700209F
:10A87000E3E7C046FF070000F0B54F464646D64620
:10A880004D00C0B50E03C90F8A462C491F035C005A
:10A890008046360B6D0D91463F0B640DDB0F8D42EC
:10A8A0001ED08C4216D0002D1ED130438446002C81
:10A8B00001D13A4323D06246002A1AD09A4529D0C2
:10A8C000514602200139084001381CBC9046994687
:10A8D000A246F0BD39001143E5D002204042F4E722
:10A8E0003043FAD1AC420FD0002C0FD13A43E7D01D
:10A8F0000CE00122013B934318000130E5E7634679
:10A900000020002BE1D0DBE73A43E6D19A45D7D1CE
:10A91000A542D5DCA54205DBBE42D1D808D0002037
:10A92000BE42D2D250460123013898430130CCE7D1
:10A93000C845C5D80020C845F4D3C6E7FF070000C6
:10A94000F0B54F464646D6464D00C0B50E03C90F7A
:10A950008A462E491F035C008046360B6D0D9146DA
:10A960003F0B640DDB0F8D4218D08C4211D0002DAF
:10A9700018D130438446002C1ED13A431CD1634683
:10A980000020002B30D05146022001390840013808
:10A990002AE039001143EAD0022025E03043FBD100
:10A9A000AC4226D0002C26D13A4324D15146022075
:10A9B00001390840013817E06246002A0FD09A4555
:10A9C000E1D1A54205DBBE42DDD819D00020BE4250
:10A9D0000AD25046012301389843013004E0012295
:10A9E000013B9343180001301CBC90469946A24697
:10A9F000F0BD3A43D0D19A45C5D1A542C3DCE0E7CA
:10AA0000C845C0D80020C845E3D3EDE7FF070000E4
:10AA1000F0B55746DE464E464546E0B5834606004D
:10AA20000F03480087B092461D003F0B400DCC0F2E
:10AA3000002800D16FE0DE4B984238D08023FF0021
:10AA40001B041F43730F3B430193DA4B00279946C6
:10AA500000239B46F60081442B0369001B0B5246E2
:10AA60009846490DED0F002900D185E0D04B994261
:10AA700000D173E04346DA0080231B04134352469F
:10AA8000CC48520F84461343524600206144D20002
:10AA900089442100694000918C46012149448A463D
:10AAA0000F2F00D990E0C449BF00CF59BF465B4685
:10AAB0003B43019300D06AE1022308270026814628
:10AAC0009B46C9E732005846019B61460091022827
:10AAD00000D175E0032800D1FEE1012800D02CE16F
:10AAE00000230027002600253F032A0D3F0BB34813
:10AAF00012053A4302401B051343009A5B00D1073D
:10AB00005B080B433000190007B03CBC90469946E7
:10AB1000A246AB46F0BD5B463B43019300D12FE11B
:10AB2000002F00D1A5E1380000F00AFE03000B3B26
:10AB30001C2B00DD96E11D22D31A5A460100DA4093
:10AB40005E4608398F4013008E403B4301939C4B77
:10AB500000271B1A994600239B467DE74146534632
:10AB60000B4393498C46E144002B00D01AE10222AA
:10AB70000220174300228CE7134300D10DE1434626
:10AB8000002B00D181E1404600F0DAFD02000B3AD3
:10AB90001C2A00DD72E10100434608398B409846CB
:10ABA0001D239A1A5346D3401A0043461343524674
:10ABB0008A404946081A824989468144002068E74C
:10ABC0007B4B002700268EE7140C1204120C110098
:10ABD000370C3604350C794328008C462E00604330
:10ABE0006044834656432100300C804658467943E2
:10ABF00040440291844506D98846802149028C460A
:10AC0000E044414602913604010C360C00048B46A8
:10AC100081191E0C1B041B0C0391190079438C46EF
:10AC2000280075436544A8465843050C45447743BE
:10AC3000A94203D9802149028C466744290C8C46DD
:10AC400039000004000C2D042D186144AB4405911B
:10AC50005946049101990F043F0C080C39005143E7
:10AC60004243904602008C46090C8B4662437C436B
:10AC700044445C44A04503D98021490288464244AB
:10AC8000210C884661460904090C8C463900594359
:10AC9000434370437E430F0CF6182404BE196444EA
:10ACA00042448C46B34203D980235B029846404419
:10ACB000029B61469846049B370443449B46AB4540
:10ACC000AD416B420D0405992D0C8C467F196744EC
:10ACD000FD18A8465D462D19A542A441934664423D
:10ACE000A446C344DC448F42BF4198459B419345F1
:10ACF0009241A445A4415B427F421F43360C52421D
:10AD00006442BF192243BF18624638184302D20D6D
:10AD1000039913436A020A43501E82416146ED0DB6
:10AD20002A434E023243D90100D4B3E00126500831
:10AD300032400243DE0732435B08224C5444002C6D
:10AD400062DD510709D00F201040042805D0101DE6
:10AD50009042924152429B180200D90104D58024AE
:10AD60001948E400034054441848844200DD27E7B2
:10AD70005E075B02D2081F0B630516435B0DB2E64C
:10AD8000002399460133042700269B4664E60323EB
:10AD9000019781460C279B465EE60122012017435E
:10ADA000002276E6032303201F43434671E6C04694
:10ADB000FF07000001FCFFFF08E60000FFFF0F8017
:10ADC0000DFCFFFFFF030000FFFFFFFEFE0700007A
:10ADD0000023802700933F030026434B83E6019B1B
:10ADE0003200A446584670E6AC466EE680270199CC
:10ADF0003F0339422DD03B422BD11F433F033F0B32
:10AE000000951600384B6EE601252D1B382D00DD10
:10AE100066E61F2D40DC35481C0050441600824079
:10AE20008440EE40501E824134431443EB4062079D
:10AE300009D00F222240042A05D02200141D94427A
:10AE4000804140421B181A023ED5012300270026EC
:10AE500049E68027019B3F031F433F033F0B0094BC
:10AE6000214B40E603005A46283B9A4000260192B7
:10AE70006DE6584600F064FC203057E60300524669
:10AE8000283B9A401300002293E6504600F058FCFD
:10AE900020307BE6CA4650E71F201E004042041BBC
:10AEA000E640202D03D0124C5444A3401A43501EB8
:10AEB0008241324307260027164009D00F20002385
:10AEC000104014000428B9D122005E075B021F0B5A
:10AED000D2081643002306E680273F031F433F03A3
:10AEE0003F0B1600004BFEE5FF0700001E040000AC
:10AEF0003E040000F8B557464E464546DE460C0077
:10AF00000903E0B5490A460F5F0031431E03DB0F1A
:10AF1000760A9B46530F3343C84E6500C000E40FCA
:10AF2000D2006D0DA24681467F0D9C469046B742E9
:10AF300000D1B9E05B46012673409B46EE1BA3455A
:10AF400000D183E0002E63DD002F00D0B1E0634626
:10AF5000134300D123E1731E002B00D0BAE1861AFF
:10AF60006346B04280410125C91A4042091A0B02CA
:10AF700000D447E149024B0A98464346002B00D1D2
:10AF800089E1404600F0DCFB0300083B1F2B00DD9D
:10AF90007CE120223000D21A4146D0409940020084
:10AFA0009E400A439D4200DD6AE15D1B6B1C1F2B26
:10AFB00000DD94E1202110003500C91A8E40DA40EE
:10AFC0008840DD40711E8E41110007222843002574
:10AFD00006433240002A09D00F233340042B05D00A
:10AFE000331DB342B641764289191E000B0200D4CC
:10AFF0003DE26A1C914B55056D0D9A4200D119E155
:10B000008F4AF6080A40570752023743120B9BE05B
:10B01000002E00D0C5E06E1C7605760D012E00DCFA
:10B0200048E16746861ACB1BB042BF417F42B84613
:10B030001F004346FF1A3B00B8461B0200D55FE1E4
:10B0400037439AD100220024002579E0002E00DC4D
:10B05000FAE0002F00D18DE0784B9D4267D080232D
:10B0600067461B041F43BC46382E00DC52E1634692
:10B0700013435A1E93411E188642804140420918CC
:10B080000B0200D4BEE06D4B01359D4200D1D2E0F1
:10B090006B4A73080A4001210E401E435108D30732
:10B0A00007221E43324095E71E00164300D045E7B5
:10B0B00040E7624B9D423AD0802367461B041F4302
:10B0C000BC46382E00DDEBE01F2E00DC3AE13300F9
:10B0D0006746203BDF403B00202E05D04027BF1BAA
:10B0E0006646BE40324390464646721E9641334302
:10B0F000DAE0002B00D114E26346134300D168E18B
:10B1000080234E07C008C9081B030643194208D014
:10B110006046C008184204D163460100D2085E07A9
:10B120001643F3009946C900720F444D11434B4634
:10B13000DE08424B4F073743CA089D4200D16EE0FC
:10B1400012036D05120B6D0D00211203130B0A0D76
:10B1500012051A433B4B2D0513402B435B00E407BC
:10B160005B082343380019003CBC90469946A24630
:10B17000AB46F8BD6346134311D0731E002B00D0BD
:10B1800007E1861886428041614440420918012542
:10B190000B0237D502257BE73E006146914635001C
:10B1A000C5E75C46002D00D0E1E00B000343F3D07F
:10B1B000731C00D1ACE1214B9F4200D13AE1F34333
:10B1C000382B00DD6FE11F2B00DD8CE120250E0008
:10B1D000ED1AAE40B0460600AA46DE40454635436D
:10B1E0002E005546D940A8406346451EA8415B1A2B
:10B1F0009C463043161AB242924163465242991A13
:10B200003D00B4E607223240002A00D0E4E60B4BB2
:10B21000F6084F073743CA089D4200D090E73B002D
:10B22000134300D1A6E180231B031A431203120B20
:10B23000024D89E715000022002785E7FF0700007F
:10B24000FFFF7FFFFFFF0F80002E00D0C7E06B1CC9
:10B250005E05760D012E00DCF0E0C84DAB4200D15A
:10B26000B9E085180A008542894162444942511873
:10B270000722CE076D082E43490832401D00A9E67B
:10B28000BF49ED1A114007223240A3E632002838A8
:10B290008240002686E6300000F052FA203073E645
:10B2A000634613435A1E9341C61AB042804140423E
:10B2B000091A5CE60E00674606431743002D5ED16F
:10B2C000002E00D0F3E0002F00D11EE15C46614665
:10B2D00091462CE7A94FBE427BD01E00F1E610003C
:10B2E0001F3DE840202B03D04021CB1A9A40164343
:10B2F000731E9E410722064332400021002583E74A
:10B30000161A6346B2428041591A40420B1A9846B7
:10B310005C4632E61F2E00DDABE02027BB1B9A46C1
:10B3200063465746BB40994613004F46F3401F43C0
:10B330003B005746BA40571EBA4113436246F2409B
:10B34000891898E62027BB1B9A4663465746BB40A0
:10B35000994613004F46F3401F433B005746BA40FF
:10B36000571EBA4113436246F240891A9CE7834B49
:10B370009F425FD080252D047342294320E7002E91
:10B380000CD1002F00D1D0E05C46614691467B4D48
:10B39000CDE67A4FBE421CD01E0065E6002F18D0C5
:10B3A000C0084E0706438020C9080003014208D0A8
:10B3B0006346DC08044204D12100DA46D2085E0765
:10B3C0001643F300994601245346C900720F1143F6
:10B3D0001C406A4DABE61D0000220027B4E6002D9C
:10B3E00059D10B00034300D1D6E6731C00D1B2E063
:10B3F000624B9F421ED0F343382B6FDC1F2B00DDC6
:10B4000097E020250E00ED1AAE40B0460600AA4691
:10B41000DE40454635432E005546A840D940451EDE
:10B42000A8418C440643B618964292415142614469
:10B430003D0025E63D006146914678E60B0003435A
:10B44000002D00D055E6002BF5D06346134300D104
:10B450006DE6861886428041614440420918002208
:10B460000B0200D4D0E6464B01351940B2E5B14697
:10B470005DE633006746203BDF403B00202E05D0D1
:10B480004027BF1B6646BE40324390464646721E6A
:10B4900096413343EFE5394B9F42CBD080252D04B5
:10B4A00073422943A8E70843411E8841A2E6002FC2
:10B4B00000D13CE66346861ACF1AB0429B415B42FC
:10B4C000FB1A98461B024ED5161A6346B2429241A9
:10B4D000591A5242891A5C4600227BE501430E004C
:10B4E000711E8E419FE71D000E00203DEE40B046CC
:10B4F000202B04D04025EB1A99400843814648464A
:10B500004346411E8841184374E60022002417E692
:10B51000161A6346B2429241591A5242891A3D00A4
:10B5200025E561469146154D01E68022002412036F
:10B5300079E61D000E00203DEE40B046202B04D0E1
:10B540004025EB1A9940084381464E464346711EFA
:10B550008E411E4367E7861896429B4161445B42D9
:10B56000C9183D008CE547463743CED007224146F7
:10B57000324049E600273A00E6E5C046FF070000F2
:10B58000FFFF7FFF70B50C4E0D031C0349005B00ED
:10B590002D0B490D240B5B0DB14208D0064900204C
:10B5A0008B4203D114432000441EA04170BD0543CB
:10B5B0000120002DFAD1F1E7FF07000030B5144D4E
:10B5C0000A034B00120B5B0DC90F0024AB4211DDC7
:10B5D000104CA34210DC8024640322430E4CE41A76
:10B5E0001F2C0CDD0D48C31ADA4013005C42002901
:10B5F00000D11C00200030BD094BCC18FAE7094DE2
:10B60000E040AC4663449A4013000343EEE7C04673
:10B61000FE0300001D0400003304000013040000BA
:10B62000FFFFFF7FEDFBFFFF70B500282DD0C31794
:10B63000C5185D40C40F280000F082F8154B1B1A96
:10B640005B055B0D0A2815DD0B38854000222D03B4
:10B650002D0B002110002D030A0D2D0B12052A437E
:10B660000D4D1B052A4013435B00E4075B08234391
:10B67000190070BD02002900153291400A000B210B
:10B68000081AC5402D032D0BE3E7002400230025F5
:10B690000022DEE71E040000FFFF0F804100090EBC
:10B6A0004B1C70B5DBB24602750AC40F012B14DDCA
:10B6B000E0239B006D07360BCB1800210A0D2800F4
:10B6C00012051C4D32435B052A405B0813435B00A7
:10B6D000E4075B082343190070BD002914D1002D35
:10B6E0001ED0280000F02CF80A281CDC0B232A00AE
:10B6F0001B1ADA40030015339D400F4B12031B1A2F
:10B700005B05160B5B0DD8E7002D06D0320B8026AB
:10B7100036036D071643094BCFE7084B0026CCE7ED
:10B7200000230026C9E703002A000B3B9A400025AE
:10B73000E3E7C046FFFF0F8089030000FF0700001A
:10B740001C2101231B04984201D3000C10391B0A51
:10B75000984201D3000A08391B09984201D3000915
:10B76000043902A2105C40187047C046040302026C
:10B7700001010101000000000000000030B51C00C4
:10B78000094B05001B6885B0D868084B002A01D119
:10B79000074B1A000292019300912B0022000549E9
:10B7A00000F026F800F0A6FD8000002048E600002A
:10B7B000CBD3000055E60000014B18687047C04627
:10B7C00080000020084B10B50400002B02D000219F
:10B7D00000E000BF054B1868836A002B00D0984733
:10B7E000200001F05DFBC0460000000084E6000080
:10B7F0000EB403B5010003AB044804CB0068019309
:10B8000000F076F802B008BC03B0184780000020B2
:10B8100070B500260C4D0D4C641BA410A64209D136
:10B82000002601F03FFB0A4D0A4C641BA410A642FF
:10B8300005D170BDB300EB5898470136EEE7B30071
:10B84000EB5898470136F2E75002002050020020E2
:10B850005002002060020020002310B59A4200D15F
:10B8600010BDCC5CC4540133F8E710B5884202D94E
:10B870008B18984203D3002307E08B5C8354013A72
:10B88000FBD210BDCC5CC45401339A42FAD1F8E724
:10B8900003001218934200D1704719700133F9E781
:10B8A000936810B5013B9360002B04DA9469A342BE
:10B8B00007DB0A2905D01368581C106019700800AE
:10B8C00010BD00F04BFC0100F9E7F8B506000F00D1
:10B8D0001400D518AC4201D1002007E021783A00CD
:10B8E0003000FFF7DDFF0134431CF3D1F8BD000049
:10B8F000F0B59FB002900F0016000593002805D008
:10B9000083690493002B01D100F0F4FD7B4B9F422F
:10B910005BD1029B5F68BB891B0762D53B69002B2B
:10B920005FD0002306AC6361203363761033A376C7
:10B9300035002B78002B01D0252B5CD1AB1B049359
:10B940000CD0320039000298FFF7BFFF431C00D132
:10B95000C4E06269049B9446634463612B78002BC6
:10B9600000D1BBE0012200235242626002A954329E
:10B9700052186E1C2360E360A3601370A3653178D6
:10B9800005225F4800F0D4FE751C002835D12268DE
:10B99000D30604D5532302A95B182021197013077D
:10B9A00004D5532302A95B182B21197033782A2B55
:10B9B0002CD0350000210A20E3682A786E1C303A2A
:10B9C000092A64D900292ED026E04E4B9F4202D18D
:10B9D000029B9F689FE74C4B9F429CD1029BDF6874
:10B9E00099E73900029800F00FFC002899D0012057
:10B9F00040421FB0F0BD01359BE7414B2268C01AA1
:10BA000001238340134323602E00B8E7059B191DD3
:10BA10001B680591002B01DB099304E05B42E360A6
:10BA20000223134323602B782E2B0AD16B782A2B09
:10BA300035D1059B02351A1D1B680592002B2BDBA7
:10BA40000793324E29780322300000F071FE00285F
:10BA500006D04023801B83402268013513432360B6
:10BA6000297806222A486E1C217600F061FE002803
:10BA70003AD0284B002B25D10722059B073393434F
:10BA8000083305936369039A9B18636150E7434346
:10BA900001219B18350090E701235B42D0E700238A
:10BAA0000A201A000135636029786E1C3039092993
:10BAB00003D9002BC5D00792C3E742430123521894
:10BAC0003500F1E705AB00933A00134B21000298D3
:10BAD00000E000BF0390039B0133D3D1BB895B0619
:10BAE00000D584E70B9884E705AB00933A000A4B36
:10BAF0002100029800F080F8ECE7C046DCE6000088
:10BB000088E60000FCE60000BCE600008EE60000CF
:10BB100092E6000000000000CBB80000F7B5150069
:10BB200001938A680B6900900C00934200DA1300BD
:10BB300022002B6043321278002A01D001332B609F
:10BB400023689B0602D52B6802332B6006272368E7
:10BB50001F4027D0230043331B785A1E934122688D
:10BB6000920630D42200019943320098089EB047D3
:10BB7000431C25D0062320682A68E168034000257D
:10BB8000042B03D18D1AEB43DB171D40A3682269F8
:10BB9000934201DD9B1AED180027BD4220D1002001
:10BBA00010E00137E3682A689B1ABB42D2DD22000D
:10BBB0000123193201990098089EB047431CF0D127
:10BBC00001204042FEBD3020E118433108702100C1
:10BBD0005A1C45310978A218433202331170C1E76B
:10BBE000220001231A3201990098089EB047431C95
:10BBF000E6D00137D1E70000F0B589B004920A0021
:10BC000043320593039002920A7E0C000E9B6E2A2B
:10BC100000D186E01FD8632A33D008D8002A00D18B
:10BC20008CE0582A4DD0250042352A7030E0642A35
:10BC300001D0692AF7D1196825680A1D280629D577
:10BC400008681A60002803DA2D23029A4042137014
:10BC50006B4E0A274FE0732A74D008D86F2A1FD082
:10BC6000702AE0D1202209680A43226003E0752A85
:10BC700016D0782AD7D12200782145321170614E32
:10BC800022E025001A684235111D196013682B70D7
:10BC9000012365E008681A606906D3D500B2D1E7D0
:10BCA00019682568081D186008682E0605D5544EC9
:10BCB00008276F2A1BD00A2719E06D06F7D580B236
:10BCC000F5E745314E4E0A7018682268011D00687C
:10BCD0001960150621D5D30702D520231A43226007
:10BCE0001027002803D1202322689A4322602300D2
:10BCF000002243331A706368A360002B58DB0422D0
:10BD0000216891432160002854D1029D002B5AD014
:10BD10002500337842352B7055E05506DBD580B2CF
:10BD2000D9E71A680D68101D4969186013682E0656
:10BD300001D5196002E06D06FBD519800023029D34
:10BD400023614FE01A68111D1960156800216268AF
:10BD5000280000F0EDFC002801D0401B6060636803
:10BD600023610023029A13703CE023692A0004999E
:10BD70000398059DA847431C3ED023689B0715D414
:10BD8000079BE068984239DA180037E02200012367
:10BD9000193204990398059EB047431C2CD00135F5
:10BDA000E368079A9B1AAB42F0DCE9E70025F7E766
:10BDB0000028ADD0029D3900FDF722FC735C013DE7
:10BDC0002B700028F7D1082F09D12368DB0706D58F
:10BDD00063682269934202DC3023013D2B70029B91
:10BDE0005B1B2361059B07AA00932100049B03981A
:10BDF000FFF794FE431CB8D10120404209B0F0BDCA
:10BE000099E60000AAE600000D4B70B51C6805001D
:10BE1000A36B002B0FD1182000F06EFC094BA06320
:10BE20000360094B01224360084B83600B2383812D
:10BE30000023026143610022A36B1D615A6170BD42
:10BE4000800000200E33CDAB34126DE6ECDE050031
:10BE5000124B10B51C68A36B002B0FD1182000F0FB
:10BE60004BFC0F4BA06303600E4B012243600E4B53
:10BE700083600B238381002302614361A46B0B4A1F
:10BE8000206961690A4BFDF7F7FC01220023801845
:10BE90005941206161614800400810BD80000020C8
:10BEA0000E33CDAB34126DE6ECDE05002D7F954CE4
:10BEB0002DF451580CB430B5164B9DB00C1E1D68B6
:10BEC00008DA8B2301202B6040421DB030BC08BC37
:10BED00002B01847822302A99B008B8100230290A5
:10BEE00008619C4200D0631E8B604B6101235B4262
:10BEF000CB81209A21AB2800019300F055FD431C13
:10BF000001DA8B232B60002CDFD00023029A137000
:10BF1000DBE7C046800000200EB400B50B499CB0A2
:10BF20001DAB02900690079104910948094904CB82
:10BF30000591006802A9019300F036FD0023029AE2
:10BF400013701CB008BC03B01847C046FFFFFF7F4A
:10BF5000800000200802FFFF020010B51378541C77
:10BF6000002B05D1CC5CD4540133002CFAD110BD88
:10BF70002200F3E7C9B20378002B04D08B4200D132
:10BF800070470130F7E74B42594149420840F7E713
:10BF900002780B78002A03D0013001319A42F7D0A1
:10BFA000D01A70470023C25C0133002AFBD1581E0F
:10BFB0007047002330B59A420AD0013AC45CCD5C88
:10BFC000AC4204D1934202D00133002CF6D1631B62
:10BFD000180030BD30B50500002A00D130BD0C7806
:10BFE000013A6B1C2C700131002C05D19A189A4231
:10BFF000F4D01C700133FAE71D00EDE710B50378AB
:10C00000002B0FD10B785A4253415B42184010BDB0
:10C010000023CA5C002AFAD0C45C944201D10133E7
:10C02000F7E701300378002BF2D11800EFE70000AA
:10C03000F0B51F000E0087B00590019102920C9898
:10C04000347800F0EAFA082200194378751C13408E
:10C0500036D12D2C36D1B51C74780126002F62D034
:10C06000102F09D1302C07D120222B789343582B45
:10C0700054D110276C7802352D4B3900F318180075
:10C080000393FDF7BDFA0491012100234942020008
:10C090008C4618002100303909291AD80C00A74213
:10C0A00023DD591C09D06346824206D302D104998C
:10C0B000A14202DB0123784320182C780135E9E7FF
:10C0C0002E00BCE72B2C01D01E00C7E7B51C7478EE
:10C0D000FAE721004139192901D8373CDFE721006F
:10C0E0006139192901D8573CD9E75A1C08D1059A5A
:10C0F00023331360029B0398002B09D107B0F0BDD6
:10C10000002E00D04042029A002AF7D0002B01D026
:10C110006B1E0193029B019A1A60EFE73024002FF7
:10C12000AAD10827A8E7302C9ED00A27A4E7C0464A
:10C13000FFFFFF7F37B51300064A05001068046A49
:10C14000002C00D1044C0A0000942900FFF770FF76
:10C150003EBDC04680000020E4000020F8B5050088
:10C160000E001400002804D08369002B01D100F0D8
:10C17000C1F9224B9C422DD16C68A369A360A389AD
:10C180001B0731D52369002B2ED023682269F7B213
:10C19000981A6369F6B2834205DC2100280000F09A
:10C1A0003BF9002826D1A3680130013BA360236836
:10C1B0005A1C22601F706369834204D0A389DB0785
:10C1C0001AD50A2E18D12100280000F025F90028E0
:10C1D00012D00FE00A4B9C4201D1AC68CDE7094B6D
:10C1E0009C42CAD1EC68C8E72100280000F00CF896
:10C1F0000028CAD0012676423000F8BDDCE60000F7
:10C20000FCE60000BCE60000364B70B51D68060079
:10C210000C00002D05D0AB69002B02D1280000F0E6
:10C2200069F9314B9C420FD16C680C23E25E93B2EA
:10C2300019072DD4D90611D40923012033603733CF
:10C240001343A381404270BD284B9C4201D1AC688E
:10C25000EBE7274B9C42E8D1EC68E6E75B0713D598
:10C26000616B002908D023004433994202D030008A
:10C2700000F06AFA002363632422A3899343A38115
:10C2800000236360236923600823A2891343A381E9
:10C290002369002B0BD1A0218022A3898900920061
:10C2A0000B40934203D02100300000F0E1F901235C
:10C2B000A289134011D00023A36063695B42A3618C
:10C2C000002023698342BED10C23E25E1306BAD557
:10C2D00040231343A3810138B5E7920700D4636973
:10C2E000A360EDE780000020DCE60000FCE6000033
:10C2F000BCE6000010B5062000F090FC012000F024
:10C30000CFFD0000F7B58A8905000C00130760D443
:10C310004B68002B04DC0B6C002B01DC0020FEBD05
:10C32000E76A002FFAD000232E682B6080235B0180
:10C33000216A1A4034D0606DA3895B0706D5636813
:10C34000C01A636B002B01D0236CC01A0200216A53
:10C3500000232800E76AB847A189431C06D12B684F
:10C360001D2B30D82B4ADA40D3072CD5002363602D
:10C3700023692360CB0405D5431C02D12B68002B15
:10C3800000D16065616B2E600029C7D02300443363
:10C39000994202D0280000F0D7F900206063BEE780
:10C3A00001232800B847431CC6D12B68002BC3D0FB
:10C3B0001D2B01D0162B01D12E60AFE74023A2899F
:10C3C0001343A381ABE740230B430120A3814042E9
:10C3D000A5E70F69002FA1D00B680F60DB1B01934D
:10C3E0000023920700D14B69A360019B002B00DC66
:10C3F00094E7019B3A00216A2800A66AB04700280A
:10C4000003DC4023A2891343DFE7019B3F181B1A7B
:10C410000193EAE7010040200B6970B505000C00AC
:10C42000002B01D1002070BD002804D08369002BAF
:10C4300001D100F05FF80B4B9C4209D16C680C22D3
:10C44000A35E002BEED021002800FFF75BFFEAE798
:10C45000054B9C4201D1AC68F1E7044B9C42EED104
:10C46000EC68ECE7DCE60000FCE60000BCE600005F
:10C47000002310B50400036043608360818143663C
:10C48000C281036143618361190008225C30FFF7B8
:10C49000FFF9054B24626362044BA362044BE36221
:10C4A000044B236310BDC0465DCC000085CC00006A
:10C4B000BDCC0000E9CC000010B5024900F08CF8BA
:10C4C00010BDC04619C4000070B568254A1E55430A
:10C4D0000E002900743100F081F9041E08D00021FB
:10C4E0002A00016046600C30A0606832FFF7D0F986
:10C4F000200070BD836913B50400002B28D183642C
:10C50000C3640365134B144A1B688262019398420B
:10C5100001D101238361200000F020F86060200039
:10C5200000F01CF8A060200000F018F80022E06085
:10C5300004216068FFF79CFF01220921A068FFF732
:10C5400097FF02221221E068FFF792FF0123A36107
:10C5500013BDC04684E60000B9C40000F8B51C4B0A
:10C5600007001E68B369002B02D13000FFF7C2FF3D
:10C570004836B4687368013B04D53368002B07D094
:10C580003668F6E70C22A55E002D0DD06834F2E780
:10C5900004213800FFF798FF30600028F0D10C2309
:10C5A00004003B602000F8BD20000A4B6566256052
:10C5B0006560A560E36025616561A56108222900C9
:10C5C0005C30FFF765F96563A563A564E564E9E799
:10C5D00084E600000100FFFFF7B504000700002615
:10C5E00001914834002C01D13000FEBD6368A5687C
:10C5F0000093009B013B009301D52468F2E7AB89CF
:10C60000012B08D90E22AB5E013304D0290038007B
:10C61000019B984706436835EBE7EC3000687047AC
:10C6200070B50E001D000E23C95E96B014000029DF
:10C6300007DA00232B60B3891B0611D48023DB00AB
:10C640000FE06A4600F088FB0028F2DBF022019B35
:10C6500012021340054A9B185A4253412B60EDE7E2
:10C6600040230020236016B070BDC04600E0FFFFED
:10C67000F7B502268B8905000C00334206D0230053
:10C6800047332360236101236361F7BD01AB6A4631
:10C69000FFF7C6FF00990700280000F09FF8002868
:10C6A00008D10C22A35E9A05EFD4032293431E43C4
:10C6B000A681E4E70F4BAB628023A289206013437D
:10C6C000A381009B20616361019B002B0DD00E2391
:10C6D000E15E280000F052FB002806D00322A38967
:10C6E00093431A0001231343A381A0893843A081F7
:10C6F000CBE7C046B9C4000010B5034B0100186871
:10C7000000F06CF810BDC0468000002082B0002907
:10C7100000D101A9101E06D0002B06D013780B60A3
:10C720001078431E984102B0704702204042FAE759
:10C73000C9B28218904201D10020704703788B4221
:10C74000FBD00130F6E7000070B50500002910D0DD
:10C750000C1F2368002B00DAE418280000F034FBDB
:10C760001D4A1368002B05D163601460280000F097
:10C770002CFB70BDA34209D9216860188342F3D114
:10C7800018685B6841182160EEE713005A68002AB8
:10C7900001D0A242F9D919685818A0420BD12068DB
:10C7A0000918581819608242E0D11068526841187F
:10C7B00019605A60DAE7A04202D90C232B60D5E752
:10C7C00021686018824203D11068526841182160C4
:10C7D00062605C60CAE7C0462C1C0020032370B571
:10C7E000CD1C9D43083506000C2D1ED20C25A942F8
:10C7F0001DD8300000F0E8FA254A1468210000290D
:10C8000019D1244C2368002B03D1300000F0CAF961
:10C8100020602900300000F0C5F9431C2BD10C2307
:10C820003000336000F0D1FA03E0002DDFDA0C2392
:10C830003360002070BD0B685B1B19D40B2B03D930
:10C840000B60CC18256003E04B688C420DD113605F
:10C85000300000F0BAFA200007220B30231D90436D
:10C86000C31AE7D05A42E250E4E763600C00EFE7F6
:10C870000C004968C3E70323C41C9C43A042E1D0D9
:10C88000211A300000F08EF9431CDBD1C7E7C04607
:10C890002C1C0020301C0020F8B507000D001600ED
:10C8A000002905D11100FFF799FF04002000F8BD11
:10C8B000002A03D1FFF748FF3400F7E700F086FABB
:10C8C0002C00B042F2D231003800FFF787FF041E7F
:10C8D000ECD029003200FEF7BFFF29003800FFF737
:10C8E00033FFE3E7F0B58E6885B007000C000392D4
:10C8F00001939E423CD890238A89DB001A4234D0AF
:10C900000325096923685B1A0293636902985D43F2
:10C91000EB0F5D19019B6D1001331B18AB4200D961
:10C920001D00530532D529003800FFF757FF061EBA
:10C9300009D10C233B6040230120A28940421343CC
:10C94000A38105B0F0BD029A2169FEF785FFA38996
:10C95000144A1A4080231343A381029B2661F618D0
:10C9600026606561019EED1AA560019B9E4200D97B
:10C97000019E320003992068FEF777FFA36800202C
:10C980009B1BA36023689E192660DAE72A00380003
:10C99000FFF782FF061EE0D121693800FFF7D4FEC1
:10C9A000C7E7C0467FFBFFFFF0B59FB0029005933D
:10C9B0008B890F0016001B0611D50B69002B0ED1B9
:10C9C0004021FFF70BFF38603861002805D10C23A8
:10C9D000029A013813601FB0F0BD40237B61002331
:10C9E00006AC6361203363761033A37635002B7871
:10C9F000002B01D0252B46D1AB1B04930CD0320069
:10CA000039000298FFF76EFF431C00D1AEE0626967
:10CA1000049B9446634463612B78002B00D1A5E00E
:10CA2000012200235242626002A9543252186E1C45
:10CA30002360E360A3601370A36531780522544836
:10CA4000FFF776FE751C00281FD12268D30604D597
:10CA5000532302A95B1820211970130704D553230F
:10CA600002A95B182B21197033782A2B16D03500B8
:10CA700000210A20E3682A786E1C303A092A4ED930
:10CA8000002918D010E00135B1E7414B2268C01AE7
:10CA900001238340134323602E00CEE7059B191D1D
:10CAA0001B680591002B01DB099304E05B42E36006
:10CAB0000223134323602B782E2B0AD16B782A2B69
:10CAC00035D1059B02351A1D1B680592002B2BDB07
:10CAD0000793304E297803223000FFF729FE002803
:10CAE00006D04023801B8340226801351343236016
:10CAF0002978062228486E1C2176FFF719FE0028A7
:10CB00003CD0264B002B25D10722059B07339343AE
:10CB1000083305936369039A9B18636166E743438F
:10CB200001219B183500A6E701235B42D0E70023D3
:10CB30000A201A000135636029786E1C30390929F2
:10CB400003D9002BC5D00792C3E7424301235218F3
:10CB50003500F1E705AB00933A00114B2100029834
:10CB600000E000BF0390039B0133D3D1BB890B9836
:10CB70005B0600D42FE7012040422CE705AB009371
:10CB80003A00074B21000298FFF736F8EAE7C04663
:10CB900088E600008EE6000092E60000000000003B
:10CBA000E5C80000002370B5064C050008002360AE
:10CBB00000F060F9431C03D12368002B00D02B60E8
:10CBC00070BDC046C02F002070B504000D001F29A5
:10CBD00004D9162303600120404270BD436C002B32
:10CBE00004D08A009B181A68002A08D1200000F09F
:10CBF00031F82A000100200000F01AF8EDE70020CB
:10CC0000012AEAD0511C03D1162301302360E4E746
:10CC1000002428001C6090472000DEE710B5034B7D
:10CC200001001868FFF7D0FF10BDC046800000204B
:10CC3000002370B5064C050008001100236000F0C9
:10CC400001F9431C03D12368002B00D02B6070BD79
:10CC5000C02F002010B500F0E5F810BD70B50C0035
:10CC60000E25495F00F0BAF8002803DB636D1B183E
:10CC7000636570BDA389024A1340A381F9E7C046EA
:10CC8000FFEFFFFFF8B51F008B8905000C001600B1
:10CC9000DB0505D50E23C95E0022022300F080F8D3
:10CCA000A389054A28001340A38132000E23E15EC8
:10CCB0003B0000F02BF8F8BDFFEFFFFF70B50C0054
:10CCC0000E25495F00F06CF8A389421C03D1054A88
:10CCD0001340A38170BD802252011343A38160657C
:10CCE000F8E7C046FFEFFFFF10B50E23C95E00F066
:10CCF00021F810BD0B1E04D0FF2A04D98A2303603B
:10CD00008B3B180070470A700123FAE770B50500E5
:10CD1000080011000022064C22601A0000F0B8F84A
:10CD2000431C03D12368002B00D02B6070BDC0468C
:10CD3000C02F0020002370B5064C050008002360BA
:10CD400000F060F8431C03D12368002B00D02B6057
:10CD500070BDC046C02F0020002370B5064C0500F2
:10CD600008001100236000F055F8431C03D123682C
:10CD7000002B00D02B6070BDC02F0020002370B5A9
:10CD8000064C05000800236000F054F8431C03D152
:10CD90002368002B00D02B6070BDC046C02F002040
:10CDA00070B50500080011000022064C22601A0030
:10CDB00000F050F8431C03D12368002B00D02B60F7
:10CDC00070BDC046C02F0020704770470B1F1B6806
:10CDD000181F002B01DA0B58C018704770B50500FA
:10CDE000080011000022064C22601A0000F03AF8F8
:10CDF000431C03D12368002B00D02B6070BDC046BC
:10CE0000C02F002058220120014B40421A60704779
:10CE1000C02F002058220120014B40421A60704769
:10CE2000C02F002058220120014B40421A60704759
:10CE3000C02F00205822024B00201A607047C046C5
:10CE4000C02F002058220120014B40421A60704739
:10CE5000C02F002058220120014B40421A60704729
:10CE6000C02F002058220120014B40421A60704719
:10CE7000C02F0020044A1368002B00D1034B181860
:10CE8000106018007047C046341C0020C82F0020D6
:10CE900058220120014B40421A607047C02F0020E9
:10CEA000FEE7C046F8B5C046F8BC08BC9E467047D1
:10CEB000F8B5C046F8BC08BC9E4670476461746112
:10CEC0000000000040CF0000EF01000049CF00004B
:10CED000E302000051CF00001909000058CF000004
:10CEE000290A00005DCF00004105000068CF000066
:10CEF000530300006DCF0000810C000079CF0000CB
:10CF00001F02000083CF00002108000091CF000025
:10CF1000CD0600009ECF00000305000072616E6424
:10CF20006F6D00616C6C006C6173740066616C7392
:10CF300065007472756500252E3135732E2E2E0016
:10CF40006D616B654C697374006164644C617374EA
:10CF50000064656C657465006A6F696E00636F706C
:10CF60007946726F6D546F0066696E64006A6F690E
:10CF70006E537472696E677300756E69636F646572
:10CF8000417400756E69636F6465537472696E678E
:10CF9000006E6577427974654172726179006672DC
:10CFA00065654D656D6F72790000000011D000005D
:10CFB0000D11000016D000002B11000051CF000011
:10CFC0002F1100001CD000001111000026D000001D
:10CFD000331100002FD000003711000039D00000BD
:10CFE0003B11000044D000003F11000050D0000071
:10CFF0001511000059D000002311000063D000007B
:10D00000191100006ED000002711000066696C65E0
:10D01000006F70656E00636C6F736500656E644FC2
:10D020006646696C6500726561644C696E65007284
:10D03000656164427974657300617070656E644CFB
:10D04000696E6500617070656E6442797465730025
:10D0500066696C6553697A650073746172744C69B2
:10D060007374006E657874496E4C697374007379DB
:10D070007374656D496E666F00000000481400000F
:10D080005814000072140000F0140000281500006D
:10D090005E15000096150000BC150000F815000094
:10D0A0003A16000090160000D41600004017000049
:10D0B00088170000AE170000E61700002C180000CB
:10D0C0005218000080180000AE180000F018000090
:10D0D00074190000461A0000D01A0000261B000038
:10D0E000721B0000921B0000B41B00000C1D00000E
:10D0F000501D0000C81D0000F61D0000441E000069
:10D100007A1E0000E41E00004E1F0000AA1F00004F
:10D11000082000007E200000F420000050210000C4
:10D12000B4210000EA210000302200007622000035
:10D13000BE2200001223000066230000A42300008A
:10D140000C240000422400008A240000D2240000A5
:10D150001A25000054250000A4250000EC2500003D
:10D160004E27000080180000E6170000542600003B
:10D17000481400008A260000B6260000EC260000B5
:10D18000182700004814000048140000481400004C
:10D1900048140000C82700000A280000502800009A
:10D1A000A0280000CC28000078290000CA2900002F
:10D1B000F829000048140000481400001C2A000050
:10D1C0004C2A00007C2A0000B22A0000DC2A000061
:10D1D000122B00003C2B0000642B00008C2B000065
:10D1E000BC2B0000EC2B0000162C0000402C000093
:10D1F000702C00009A2C0000481400004814000015
:10D20000481400004814000048140000CA2C000014
:10D21000F62C0000222D0000602D00008C2D000057
:10D22000C22D0000F82D00002E2E0000642E0000FC
:10D23000902E0000BC2E0000F22E000048140000CA
:10D24000481400004814000048140000481400006E
:10D25000481400004814000048140000481400005E
:10D26000481400004814000048140000481400004E
:10D27000481400001E2F0000542F00005B2564207E
:10D280006974656D206C6973745D00282564206283
:10D29000797465732900286F626A656374207479F4
:10D2A00070653A2025642900537461636B20756EA4
:10D2B000646572666C6F7700626F6F6C65616E009B
:10D2C0006E756D62657200737472696E67006C6969
:10D2D0007374006279746520617272617900000074
:10D2E000070000000300000041D30000753000007B
:10D2F00049D300002531000052D30000CF31000097
:10D300005BD300007930000064D30000D33100000B
:10D310006CD30000BD3100001C00000001000000C3
:10D3200002000000040000000500000006000000EC
:10D33000100000001100000043616C6C696F7065A3
:10D3400000686173546F6E6500706C6179546F6E24
:10D350006500686173536572766F00736574536519
:10D3600072766F00646163496E697400646163572B
:10D370007269746500474320746F6F6B20256420C9
:10D3800075736563733B206672656520256420773D
:10D390006F726473003C496E74656765723E003C51
:10D3A0004C6973743E003C4F626A6563743E003C96
:10D3B0004279746541727261793E000D0A564D20C2
:10D3C00050616E69633A2025730D0A006D697363BD
:10D3D0000000000009D40000A93E000012D40000A3
:10D3E000393E000016D400008D3D00001ED4000020
:10D3F000333D000028D40000C93C000034D40000B4
:10D40000CB3B00006E756C6C00686578546F496E9C
:10D41000740073696E006A736F6E476574006A7397
:10D420006F6E436F756E74006A736F6E56616C75C4
:10D43000654174006A736F6E4B657941740000003A
:10D44000CCD40000153F0000D4D40000193F0000E8
:10D45000DED40000373F0000E7D40000413F000069
:10D46000F2D400004B3F0000FED40000553F000006
:10D470000CD500005F3F000014D50000693F00009C
:10D480001AD50000733F00002FD500007D3F00003B
:10D4900044D50000873F000050D50000913F0000B8
:10D4A00060D500009B3F00006CD50000A53F000048
:10D4B00079D50000AF3F000088D50000233F000071
:10D4C0009BD500002D3F00006E65740068617357A6
:10D4D00069466900737461727457694669007374B0
:10D4E0006F7057694669007769666953746174752E
:10D4F00073006D794950416464726573730073748D
:10D50000617274535349447363616E006765745369
:10D51000534944006D794D414300687474705365FC
:10D5200072766572476574526571756573740072C1
:10D530006573706F6E64546F487474705265717562
:10D540006573740068747470436F6E6E6563740005
:10D55000687474704973436F6E6E656374656400BC
:10D560006874747052657175657374006874747052
:10D57000526573706F6E736500776562536F636B8E
:10D580006574537461727400776562536F636B6581
:10D59000744C6173744576656E7400776562536F81
:10D5A000636B657453656E64546F436C69656E7428
:10D5B000000D0E0F04050C0B0A06070809000000F9
:10D5C000000008080800080A4A4000000A5FEA5FF5
:10D5D000EA0ED92ED36E19324489330C924C924DF7
:10D5E00008080000000488080804080484848800EF
:10D5F0000A448A4000048EC48000000004880000B1
:10D600000EC000000000080001224488100C925255
:10D61000524C048C84848E1C824C901E1EC24492F8
:10D620004C06CA525FE21FF01EC13E02448ED12E4C
:10D630001FE24488100ED12ED12E0ED12EC48800A8
:10D640000800080000048004880244880482000E58
:10D65000C00EC008048244880ED126C0040ED13505
:10D66000B36C0C925ED2521C925C925C0ED0101085
:10D670000E1C9252525C1ED01C901E1ED01C90108C
:10D680000ED013712E12525ED2521C8808081C1F35
:10D69000E242524C1254981492101010101E113B7A
:10D6A00075B131113935B3710C9252524C1C925CE8
:10D6B00090100C92524C861C925C92510ED00C82AF
:10D6C0005C1FE4848484125252524C1131312A443A
:10D6D000113135BB7112524C9252112A4484841E6E
:10D6E000C488101E0EC808080E10080482410EC21D
:10D6F00042424E048A400000000000001F080480DF
:10D700000000000ED2524F10101C925C000ED01080
:10D710000E02424ED24E0C925C900E06C81C880837
:10D720000ED24EC24C10101C92520800080808027B
:10D730004002424C10149814920808080806001B76
:10D7400075B131001C925252000C92524C001C9246
:10D750005C90000ED24EC2000ED010100006C8041D
:10D760009808080EC807001252524F0011312A447F
:10D7700000113135BB00124C8C9200112A449800E4
:10D780001EC4881E06C48C84860808080808180869
:10D790000C881800000C83600000000001000000ED
:10D7A000020000000300000004000000050000006B
:10D7B000060000000700000008000000090000004B
:10D7C0000A0000000B0000000C0000000D0000002B
:10D7D0000E0000000F00000010000000120000000A
:10D7E0001400000016000000180000001A000000DD
:10D7F0001C0000001E0000002000000023000000AC
:10D8000026000000290000002C0000002F0000006E
:10D8100032000000360000003A0000003E00000028
:10D8200042000000460000004B00000050000000D5
:10D83000550000005A000000610000006800000070
:10D840006F000000760000007D00000084000000F2
:10D850008B0000009200000099000000A000000072
:10D86000A7000000AE000000B5000000BC000000F2
:10D87000C3000000CA000000D1000000D800000072
:10D88000DF000000E6000000ED000000F4000000F2
:10D89000FB000000FF000000E8D80000D13F0000BE
:10D8A000F3D800006D450000FDD800009541000050
:10D8B0000AD90000DD43000011D900002D4400000A
:10D8C0001AD900007D44000026D9000075430000ED
:10D8D00037D900000542000044D90000054300008C
:10D8E000646973706C6179006C696768744C657603
:10D8F000656C006D62446973706C6179006D62449F
:10D900006973706C61794F6666006D62506C6F74FC
:10D91000006D62556E706C6F74006D624472617759
:10D920005368617065006D625368617065466F721F
:10D930004C6574746572006E656F506978656C53E0
:10D94000656E64006E656F506978656C53657450E0
:10D95000696E004E6F7420656E6F75676820726F18
:10D960006F6D206576656E20616674657220636FE9
:10D970006D70616374696F6E00436F6D7061637485
:10D98000656420466C61736820636F6465207374FE
:10D990006F72650A256420627974657320757365FA
:10D9A0006420282564252529206F662025640042EF
:10D9B0006164207265636F726420666F756E6420A7
:10D9C000647572696E6720696E697469616C697AE1
:10D9D0006174696F6E002564202564202564202809
:10D9E000256420776F726473290025642072656353
:10D9F0006F7264732C20256420776F7264732C20FF
:10DA00006D617849442025642C20636F6D706163DB
:10DA100074696F6E206379636C65732025640052AE
:10DA20006573746F72656420256420736372697016
:10DA30007473005374617274656400726164696F19
:10DA400000000000D4DA0000454F0000E1DA0000D9
:10DA5000E1510000F1DA000061510000FFDA00003E
:10DA6000755300000ADB00006D4F00001ADB000058
:10DA7000F54F00002EDB0000DD4F00003DDB000015
:10DA80005755000049DB0000D554000052DB000070
:10DA9000795400005DDB0000C153000068DB00002A
:10DAA000FD53000071DB0000315400007ADB000000
:10DAB0007D4F000089DB00005D4F000092DB00001D
:10DAC0008D4F00006E6F6E65006F74686572007038
:10DAD0006169720064697361626C65526164696F47
:10DAE000006D65737361676552656365697665642A
:10DAF000007061636B65745265636569766500707B
:10DB000061636B657453656E640072656365697605
:10DB10006564496E746567657200726563656976F0
:10DB200065644D65737361676554797065007265EE
:10DB3000636569766564537472696E670073656EB8
:10DB400064496E74656765720073656E64506169DF
:10DB5000720073656E64537472696E6700736574E6
:10DB60004368616E6E656C0073657447726F7570A3
:10DB700000736574506F776572007369676E616CCE
:10DB8000537472656E67746800646576696365498D
:10DB900044006C6173744D6573736167654944003B
:10DBA000556E6B6E6F776E207072696D69746976F1
:10DBB00065205B25733A25735D00000000000000BE
:10DBC000963007772C610EEEBA51099919C46D078A
:10DBD0008FF46A7035A563E9A395649E3288DB0EE5
:10DBE000A4B8DC791EE9D5E088D9D2972B4CB609C8
:10DBF000BD7CB17E072DB8E7911DBF906410B71DA5
:10DC0000F220B06A4871B9F3DE41BE847DD4DA1ADD
:10DC1000EBE4DD6D51B5D4F4C785D38356986C130E
:10DC2000C0A86B647AF962FDECC9658A4F5C011487
:10DC3000D96C0663633D0FFAF50D088DC8206E3B65
:10DC40005E10694CE44160D5727167A2D1E4033C77
:10DC500047D4044BFD850DD26BB50AA5FAA8B5359E
:10DC60006C98B242D6C9BBDB40F9BCACE36CD8328D
:10DC7000755CDF45CF0DD6DC593DD1ABAC30D92634
:10DC80003A00DE518051D7C81661D0BFB5F4B42137
:10DC900023C4B3569995BACF0FA5BDB89EB8022834
:10DCA0000888055FB2D90CC624E90BB1877C6F2FB9
:10DCB000114C6858AB1D61C13D2D66B69041DC76B4
:10DCC0000671DB01BC20D2982A10D5EF8985B1718D
:10DCD0001FB5B606A5E4BF9F33D4B8E8A2C907783C
:10DCE00034F9000F8EA8099618980EE1BB0D6A7FD3
:10DCF0002D3D6D08976C6491015C63E6F4516B6B8C
:10DD000062616C1CD83065854E0062F2ED95066C40
:10DD10007BA5011BC1F4088257C40FF5C6D9B065B5
:10DD200050E9B712EAB8BE8B7C88B9FCDF1DDD6212
:10DD3000492DDA15F37CD38C654CD4FB5861B24D78
:10DD4000CE51B53A7400BCA3E230BBD441A5DF4A42
:10DD5000D795D83D6DC4D1A4FBF4D6D36AE9694305
:10DD6000FCD96E34468867ADD0B860DA732D0444B0
:10DD7000E51D03335F4C0AAAC97C0DDD3C710550DB
:10DD8000AA41022710100BBE86200CC925B5685782
:10DD9000B3856F2009D466B99FE461CE0EF9DE5ECB
:10DDA00098C9D9292298D0B0B4A8D7C7173DB3597C
:10DDB000810DB42E3B5CBDB7AD6CBAC02083B8ED0D
:10DDC000B6B3BF9A0CE2B6039AD2B1743947D5EA1A
:10DDD000AF77D29D1526DB048316DC73120B63E349
:10DDE000843B64943E6A6D0DA85A6A7A0BCF0EE4A8
:10DDF0009DFF099327AE000AB19E077D44930FF063
:10DE0000D2A3088768F2011EFEC206695D5762F759
:10DE1000CB67658071366C19E7066B6E761BD4FE96
:10DE2000E02BD3895A7ADA10CC4ADD676FDFB9F973
:10DE3000F9EFBE8E43BEB717D58EB060E8A3D6D635
:10DE40007E93D1A1C4C2D83852F2DF4FF167BBD163
:10DE50006757BCA6DD06B53F4B36B248DA2B0DD866
:10DE60004C1B0AAFF64A0336607A0441C3EF60DF09
:10DE700055DF67A8EF8E6E3179BE69468CB361CBF2
:10DE80001A8366BCA0D26F2536E2685295770CCC17
:10DE900003470BBBB91602222F260555BE3BBAC558
:10DEA000280BBDB2925AB42B046AB35CA7FFD7C249
:10DEB00031CFD0B58B9ED92C1DAEDE5BB0C2649B3A
:10DEC00026F263EC9CA36A750A936D02A906099C6D
:10DED0003F360EEB8567077213570005824ABF95E0
:10DEE000147AB8E2AE2BB17B381BB60C9B8ED29263
:10DEF0000DBED5E5B7EFDC7C21DFDB0BD4D2D386BA
:10DF000042E2D4F1F8B3DD686E83DA1FCD16BE812C
:10DF10005B26B9F6E177B06F7747B718E65A0888FD
:10DF2000706A0FFFCA3B06665C0B0111FF9E658F8E
:10DF300069AE62F8D3FF6B6145CF6C1678E20AA038
:10DF4000EED20DD75483044EC2B30339612667A7BE
:10DF5000F71660D04D476949DB776E3E4A6AD1AE0D
:10DF6000DC5AD6D9660BDF40F03BD83753AEBCA99C
:10DF7000C59EBBDE7FCFB247E9FFB5301CF2BDBD09
:10DF80008AC2BACA3093B353A6A3B4240536D0BA12
:10DF90009306D7CD2957DE54BF67D9232E7A66B3AF
:10DFA000B84A61C4021B685D942B6F2A37BE0BB45C
:10DFB000A18E0CC31BDF055A8DEF022D416C6C2026
:10DFC0007461736B732073746F7070656400763165
:10DFD000303900202573202573004D656D6F7279EF
:10DFE00020636C6561726564004E6F2066726565C2
:10DFF000207461736B20656E747269657300000034
:10E0000058E00000A169000065E00000F968000028
:10E0100071E00000C968000077E00000D9680000E6
:10E020007DE00000E968000083E00000FD6400007E
:10E030008DE000001569000095E000001967000000
:10E040009EE0000059650000A6E000008166000027
:10E0500073656E736F727300616363656C65726183
:10E0600074696F6E0074656D706572617475726548
:10E070000074696C74580074696C74590074696C2C
:10E08000745A00746F756368526561640069326325
:10E090005265616400693263577269746500726524
:10E0A0006164444854006D6963726F70686F6E6597
:10E0B0000000000030E10000596A00003EE100006D
:10E0C000696A00004BE100005D6A000054E1000055
:10E0D0006D6A00005EE10000716A000067E1000007
:10E0E000756A00006CE10000796A000071E10000CF
:10E0F0007D6A00007DE10000816A000084E100008B
:10E10000856A00008DE10000896A000092E100004C
:10E110008D6A00009DE10000916A0000A7E1000007
:10E12000616A0000B1E10000656A00007466740075
:10E13000656E61626C65446973706C6179007365CA
:10E14000744261636B6C69676874006765745769D2
:10E15000647468006765744865696768740073650E
:10E1600074506978656C006C696E650072656374E3
:10E1700000726F756E6465645265637400636972E2
:10E18000636C6500747269616E676C6500746578B4
:10E190007400746674546F756368656400746674A3
:10E1A000546F7563685800746674546F756368596A
:10E1B00000746674546F756368507265737375721A
:10E1C0006500766172730000E8E10000216F0000D5
:10E1D000F2E10000016F0000FBE10000DD6E0000D5
:10E1E00007E20000696E0000766172457869737419
:10E1F00073007661724E616D65640073657456617B
:10E20000724E616D6564007661724E616D65466F38
:10E2100072496E6465780057656C636F6D65207434
:10E220006F204D6963726F426C6F636B7321007076
:10E230005F73706920213D204E554C4C002F686F54
:10E240006D652F6769742F2E706C6174666F726DC7
:10E25000696F2F7061636B616765732F6672616DA3
:10E2600065776F726B2D61726475696E6F6E6F7218
:10E270006469636E7266352F6C696272617269657A
:10E28000732F5350492F5350492E637070005350D1
:10E2900049436C6173733A3A535049436C617373E9
:10E2A000284E52465F5350495F547970652A2C209E
:10E2B00075696E74385F742C2075696E74385F747C
:10E2C0002C2075696E74385F74290000000000000E
:10E2D000000000002D710000E97000000F710000C7
:10E2E00019710000237100000D7100000000000092
:10E2F0000100000002000000160000000400000001
:10E3000005000000060000000700000008000000F3
:10E31000090000000A0000000B0000000C000000D3
:10E320000D0000000E0000000F0000001A000000A9
:10E330001B0000001400000013000000110000008A
:10E3400017000000100000001C0000001D0000006D
:10E350001E00000012000000150000000300000075
:10E36000180000001900000000000000000000007C
:10E37000197500004D7D000099750000AD75000015
:10E38000A37500001575000009750000B97500003F
:10E3900035750000057500000000000000003043E6
:10E3A00000000000000030C37371727400000000B0
:10E3B000FB21F93FFB2109407CD91240FB21194088
:10E3C0007A6A1F407CD92240BBFD2540FB212940B1
:10E3D0003A462C407A6A2F405C4731407CD9324023
:10E3E0009C6B3440BBFD3540DB8F3740FB2139400F
:10E3F0001BB43A403A463C405AD83D407A6A3F40C6
:10E400004C7E40405C4741406C1042407CD94240C9
:10E410008CA243409C6B4440AC344540BBFD45401E
:10E42000CBC64640DB8F4740EB584840FB21494074
:10E4300083F9A200444E6E00FC291500D157270035
:10E44000DD34F50062DBC0003C999500419043004B
:10E450006351FE00BBDEAB00B761C5003A6E24001D
:10E46000D24D42004906E00009EA2E001C92D1007C
:10E47000EB1DFE0029B11C00E83EA700F535820027
:10E4800044BB2E009CE98400B4267000417E5F00EE
:10E49000D6913900538339009CF439008B5F840096
:10E4A00028F9BD00F81F3B00DEFF97000F9805001C
:10E4B000112FEF000A5A8B006D1F6D00CF7E3600C2
:10E4C00009CB2700464FB7009E663F002DEA5F004C
:10E4D000BA277500E5EBC7003D7BF100F73907006F
:10E4E00092528A00FB6BEA001FB15F00085D8D004D
:10E4F000300356007BFC4600F0AB6B0020BCCF0025
:10E5000036F49A00E3A91D005E619100081BE60045
:10E5100085996500A0145F008D40680080D8FF00D9
:10E5200027734D0006063100CA561500C9A87300AE
:10E530007BE260006B8CC00000000040FB21F93FD3
:10E54000000000002D44743E000000809846F83C16
:10E550000000006051CC783B00000080831BF03944
:10E560000000004020257A38000000802282E33637
:10E57000000000001DF369350200000003000000E8
:10E580000400000006000000C49900006E9900001D
:10E590006E9900009C9A00006A9900006A99000038
:10E5A000929A00009C9A00006A990000929A0000DA
:10E5B0006A9900009C9A0000A09A0000A09A0000AE
:10E5C000A09A0000A89A0000A0A4000012A30000D6
:10E5D00056A30000BAA2000056A3000046A4000003
:10E5E00056A30000BAA2000012A3000012A300006C
:10E5F00046A40000BAA20000B2A20000B2A200002D
:10E60000B2A2000054A40000C8AB0000CAAA0000D7
:10E61000CAAA0000E8AD0000C4AA0000C4AA000015
:10E62000D0AD0000E8AD0000C4AA0000D0AD0000ED
:10E63000C4AA0000E8AD0000DEAD0000DEAD0000C1
:10E64000DEAD0000ECAD00002C2066756E637469D1
:10E650006F6E3A2000617373657274696F6E202269
:10E66000257322206661696C65643A2066696C6571
:10E6700020222573222C206C696E65202564257369
:10E6800025730A0084000020232D302B2000686CA5
:10E690004C006566674546470030313233343536C5
:10E6A00037383941424344454600303132333435FE
:10E6B0003637383961626364656600000000000027
:10E6C000000000000000000000000000000000004A
:10E6D000000000000000000000000000000000003A
:10E6E000000000000000000000000000000000002A
:10E6F000000000000000000000000000000000001A
:10E700000000000000000000000000000000000009
:10E71000000000000000000000000000504F5349BE
:10E7200058000020202020202020202028282828D1
:10E7300028202020202020202020202020202020D1
:10E740002020208810101010101010101010101021
:10E750001010100404040404040404040410101031
:10E7600010101010414141414141010101010101DD
:10E77000010101010101010101010101010110106B
:10E7800010101010424242424242020202020202B1
:10E79000020202020202020202020202020210103D
:10E7A0001010200000000000000000000000000029
:10E7B0000000000000000000000000000000000059
:10E7C0000000000000000000000000000000000049
:10E7D0000000000000000000000000000000000039
:10E7E0000000000000000000000000000000000029
:10E7F0000000000000000000000000000000000019
:10E800000000000000000000000000000000000008
:10E8100000000000000000000000000000000000F8
:08E820000000000000000000F0
:08E82800E018FF7F0100000071
:10E83000FFFFFFFFE803000001000000E803DC0524
:10E84000DC05DC05DC050000FFFFFFFFFFFFFFFF2D
:10E850001800000019FCFFFFFFFFFFFF0024F40079
:10E860000200000003000000FFFFFFFF00000000A7
:10E87000010000000000020001000000FFFFFFFF98
:10E880000000000002000000000004000200000080
:10E89000FFFFFFFF00000000030000000000080071
:10E8A000030000000A000000080000000100000052
:10E8B0008400002000000000DCE60000FCE6000010
:10E8C000BCE60000000000000000000000000000A6
:10E8D0000000000000000000000000000000000038
:10E8E0000000000000000000000000000000000028
:10E8F0000000000000000000000000000000000018
:10E900000000000000000000000000000000000007
:10E9100000000000430000000000000000000000B4
:10E9200000000000000000000000000000000000E7
:10E930000000000043000000000000000000000094
:10E9400000000000000000000000000000000000C7
:10E950000000000043000000000000000000000074
:10E9600000000000000000000000000000000000A7
:10E970000000000043000000000000000000000054
:10E980000000000000000000000000000000000087
:10E990000000000043000000000000000000000034
:10E9A0000000000000000000000000000000000067
:10E9B0000000000043000000000000000000000014
:10E9C0000000000000000000000000000000000047
:10E9D00000000000430000000000000000000000F4
:10E9E0000000000000000000000000000000000027
:10E9F00000000000F5CC00000DC700000000000082
:10EA000022E700003ECF0000CBD30000CBD30000B4
:10EA1000CBD30000CBD30000CBD30000CBD300007E
:10EA2000CBD30000CBD30000CBD30000FFFFFFFF10
:10EA3000FFFFFFFFFFFFFFFFFFFF0000010041534B
:10EA400043494900000000000000000000000000F1
:10EA50000000000000000000000000000000415322
:10EA600043494900000000000000000000000000D1
:10EA70000000000000000000000000000000000096
:10EA8000E9000000B97000000D7400006578000016
:04EA9000C1000000C1
:04000003000074A9DC
:00000001FF
